:020000040800F2
:10000000000002208D860008918400089984000871
:100010009B8400089D8400089F8400080000000065
:10002000000000000000000000000000A1840008A3
:10003000A384000800000000A5840008A78400082D
:10004000DD860008DD860008DD860008DD86000804
:10005000DD860008DD860008DD860008DD860008F4
:10006000DD860008DD860008DD860008DD860008E4
:10007000DD860008B1840008DD860008DD86000802
:10008000C1840008DD860008DD860008000000004D
:10009000000000000000000000000000DD860008F5
:1000A000DD860008DD860008D1840008DD860008B2
:1000B000E1840008DD860008DD860008DD86000892
:1000C000DD860008DD860008DD860008DD86000884
:1000D000DD860008DD860008DD86000800000000DF
:1000E000DD860008DD860008DD86000800000000CF
:1000F000000000000000000000000000DD86000895
:1001000000000000DD86000851850008DD8600083B
:1001100000000000000000000000000000000000DF
:10012000DD860008DD860008DD860008DD86000823
:10013000DD86000800000000000000000000000054
:10014000000000000000000000000000BD85000865
:10015000DD860008DD860008DD860008DD860008F3
:10016000DD860008DD8600080000000000000000B9
:10017000000000000000000000000000000000007F
:1001800000000000DD860008000000000000000004
:08019000DD860008DD86000891
:1001C0000348044B834202D0034B03B118477047E6
:1001D000A40A0020A40A00200000000005480649E7
:1001E0000B1AD90F01EBA301491002D0034B03B145
:1001F00018477047A40A0020A40A0020000000004D
:1002000010B5064C237843B9FFF7DAFF044B13B15E
:100210000448AFF300800123237010BDA80A00201A
:1002200000000000E4CB000808B5044B1BB10449F2
:100230000448AFF30080BDE80840CFE700000000AD
:10024000AC0A0020E4CB000853B94AB9002908BF22
:1002500000281CBF4FF0FF314FF0FF3000F074B9A1
:10026000ADF1080C6DE904CE00F006F8DDF804E00D
:10027000DDE9022304B070472DE9F047089E0D46E2
:1002800004468846002B4DD18A42944668D9B2FA7A
:1002900082F252B101FA02F3C2F1200120FA01F117
:1002A0000CFA02FC41EA030894404FEA1C45210C79
:1002B000B8FBF5FE1FFA8CF705FB1E8341EA0343EA
:1002C0000EFB07F199420BD91CEB03030EF1FF3033
:1002D00080F01E81994240F21B81AEF1020E634410
:1002E0005B1AA4B2B3FBF5F005FB103344EA0344F8
:1002F00000FB07F7A7420AD91CEB040400F1FF3307
:1003000080F00881A74240F2058164440238E41B72
:1003100040EA0E4000211EB1D4400023C6E900434C
:10032000BDE8F0878B4208D9002E00F0EE80002156
:10033000C6E900050846BDE8F087B3FA83F1002955
:100340004AD1AB4202D3824200F2F980841A65EBB3
:10035000030301209846002EE2D0C6E90048DFE7FB
:1003600002B9FFDEB2FA82F2002A40F09180A1EBDE
:100370000C054FEA1C471FFA8CFE0121B5FBF7F371
:1003800007FB1350250C45EA00450EFB03F0A8427D
:1003900008D91CEB050503F1FF3802D2A84200F290
:1003A000CB8043462D1AA4B2B5FBF7F007FB1055DE
:1003B00044EA05440EFB00FEA64508D91CEB0404E4
:1003C00000F1FF3502D2A64500F2BB802846A4EB1F
:1003D0000E0440EA03409EE7C1F120078B4022FA59
:1003E00007FC4CEA030C20FA07F405FA01F31C435E
:1003F000FD404FEA1C4900FA01F3B5FBF9F8200C67
:100400001FFA8CFE09FB185540EA054508FB0EF063
:10041000A84202FA01F20BD91CEB050508F1FF3ADC
:1004200080F08880A84240F28580A8F102086544E7
:100430002D1AA4B2B5FBF9F009FB105544EA0545A5
:1004400000FB0EFEAE4508D91CEB050500F1FF349C
:100450006CD2AE456AD90238654440EA0840A0FB38
:100460000294A5EB0E05A542C846A64656D353D026
:100470005EB1B3EB080265EB0E0505FA07F722FA49
:1004800001F3CD401F43C6E900750021BDE8F087A8
:10049000C2F1200320FA03F10CFA02FC25FA03F35F
:1004A00095400D434FEA1C471FFA8CFEB3FBF7F152
:1004B00007FB11302B0C43EA004301FB0EF098427E
:1004C00004FA02F408D91CEB030301F1FF382FD220
:1004D00098422DD9023963441B1AADB2B3FBF7F031
:1004E00007FB103345EA034500FB0EF3AB4208D986
:1004F0001CEB050500F1FF3816D2AB4214D90238C7
:100500006544ED1A40EA014138E73146304607E7D5
:100510008646E5E61846FAE64B45A9D2B9EB02084D
:1005200064EB0C0E0138A3E74046EAE7204694E767
:100530004146D1E7D0467BE7023B654432E70846B7
:1005400009E76444023842E7704700BF00230146D0
:100550001A46184601F0FABA014B1868704700BFF6
:100560000000002038B5084B084D5B1B9C1007D0DD
:10057000043B1D44013C55F804399847002CF9D13F
:10058000BDE838400CF034BB7CD0000878D00008BF
:1005900070B50D4E0D4D761BB61006D0002455F8E3
:1005A000043B01349847A642F9D1094E094D761B08
:1005B0000CF018FBB61006D0002455F8043B0134AB
:1005C0009847A642F9D170BD70D0000870D00008DD
:1005D00078D0000870D00008830730B548D0541E8A
:1005E000002A3FD0CAB2034601E0013C3AD303F8E7
:1005F000012B9D07F9D1032C2DD9CDB245EA052554
:100600000F2C45EA054536D9A4F1100222F00F0C53
:1006100003F1200EE6444FEA121C03F1100242E9F6
:10062000045542E9025510327245F8D10CF101022D
:1006300014F00C0F03EB021204F00F0C13D0ACF10A
:10064000040323F003030433134442F8045B93428E
:10065000FBD10CF003042CB1CAB21C4403F8012BEB
:100660009C42FBD130BD64461346002CF4D1F9E71F
:1006700003461446BFE71A46A446E0E70CB410B59B
:100680009CB01EAB6FF00044CDE9061402910849FE
:1006900053F8042B059102A90193049400F02AF861
:1006A000029B00221A701CB0BDE8104002B07047D7
:1006B0000802FFFF0EB410B59DB06FF000411FABF4
:1006C000CDE906010491094953F8042B0290084C26
:1006D0000868019302A9059400F00CF8029B00221F
:1006E0001A701DB0BDE8104003B070470000002034
:1006F0000802FFFF2DE9F04FBFB0884691460D93E9
:100700000C9002F04DFA03681493184603F038FB7E
:10071000B8F80C301390180604D5D8F81030002B18
:1007200000F0CA860023CDE922330F93129315936C
:10073000099300240023CDE910342EAA2192924679
:1007400099F80030002B00F080814C4604E014F84A
:10075000013F002B00F0C580252BF8D1B4EB090533
:1007600040F0C3802378002B00F06F8100234FF00E
:10077000FF3265788DF8673004F101091846089258
:100780000A939B4609F10109A5F12002582A00F2BB
:10079000D380DFE812F05302D100D1004E02D10025
:1007A000D100D100D100D100D10001024902D10015
:1007B0000C021102D100440259005900590059009D
:1007C00059005900590059005900D100D100D100F9
:1007D000D100D100D100D100D100D100D1002B0235
:1007E0006401D1006401D100D100D100D1005B02CD
:1007F000D100D1007800D100D100D100D100D100CA
:100800006800D100D1006E02D100D100D100D1002A
:10081000D100D100D100D100D100D1006002C401CB
:100820006401640164018F02C401D100D10003039B
:10083000D100ED027A00D202CD02D100AB02D1008C
:100840006A00D100D1009402A5F13002002119F80C
:10085000015B01EB810102EB4101A5F13002092AA4
:10086000F5D90A9190E74BF0100B1BF0200100F036
:1008700048810D9B073323F00703596853F8080B91
:100880000D9301230EE04BF0100B1BF0200100F044
:100890002B810D9B073323F00703596853F8080B8E
:1008A0000D93002300248DF86740089A561C00F031
:1008B00084822BF08006069650EA010640F07B8287
:1008C000002A40F00383002B40F024851BF0010335
:1008D0000B9300F0908530238DF8B7300DF1B706FB
:1008E00090E2B4EB090500F0B080239B2B442393E6
:1008F000229B0133072BCAE90095229305DC0AF1FC
:10090000080A099B2B4409932CE70C9821AA41461D
:1009100003F0A4FA18B90DF1B80AF2E7B846B8F82E
:100920000C3013F0400F099B18BF4FF0FF330993B1
:1009300009983FB0BDE8F08F002B40F0C587002D2F
:1009400000F0838000238DF8673001238DF89050EC
:1009500007930B9324AE0023CDF818B008930E93A1
:10096000069B13F0020302D0079A02320792069AFE
:1009700012F0840B05D10A9A0799571A002F00F339
:100980009883239C9DF867208AB1229A0DF1670114
:1009900001320134CAF80010072A4FF001012394F4
:1009A0002292CAF8041000F3CD830AF1080A83B139
:1009B000229B1AAA01330234CAF80020072B4FF0F9
:1009C000020223942293CAF8042000F3C9830AF197
:1009D000080ABBF1800F00F09582089B0B9AA3EBED
:1009E000020BBBF1000F00F3CF82069BDF0500F185
:1009F00012820B9BCAF804301C44229BCAF8006088
:100A00000133072B2394229300F347830AF1080A4A
:100A1000069B5B0705D50A9B079A9D1A002D00F3DC
:100A2000AB83DDE9093207998A42ACBF9B185B189A
:100A30000993002C40F0E2820023229399F80030C1
:100A40000DF1B80A002B7FF480AE239B002B3FF4FE
:100A500066AF0C9821AA414603F000FA5FE7002B2D
:100A600040F0D4870D9B073323F00702F2E80234ED
:100A7000CDE91034DDE9103424F000440D921E4617
:100A800018462146B54B4FF0FF3207F013F9002806
:100A900040F0B884B14B304621464FF0FF3207F0AA
:100AA000EBF8002840F0AE84DDE9100100220023BD
:100AB00007F0D8F8002840F0E0869DF86740A84E7F
:100AC0002BF080030693A74B0022472DC8BF1E467C
:100AD0000323CDE907320B930E92002C3FF440AF75
:100AE000079B013307933BE71BF0100348D11BF032
:100AF000400145D00D9A52F8040B0D92194680B270
:100B0000D0E61BF0100341D11BF040013ED00D9AFE
:100B100052F8040B0D92194680B20123C2E6002B55
:100B200040F07C871BF0200F0D9B68D0073323F02B
:100B300007031A465B6852F8080B0D921946002B02
:100B4000C0F23084089B013300F06B852BF08003EA
:100B5000069350EA01039DF8674000F0D783DDF863
:100B600018B00A2871F1000380F0FC8430300123B2
:100B70008DF8B700CDF818B00B930DF1B70641E131
:100B80000D9B53F8040B0D930B468BE60D9B53F80E
:100B9000040B0D93012385E60D9A52F8041B0A916C
:100BA000002980F223840A990D9249420A9199F80A
:100BB00000504BF0040BE5E5494611F8015B2A2D86
:100BC00000F0A387A5F13002092A894698BF0021C9
:100BD00000F2208719F8015B01EB810102EB410172
:100BE000A5F13002092AF5D90891CDE5002B40F096
:100BF00019874BF0100B1BF0200F0D9B96D153F86B
:100C0000040B0D931BF0100F40F0C7831BF0400F37
:100C100000F0C38340F3C0310B4600B28FE799F870
:100C200000504BF0800BADE599F8005001232B20CC
:100C3000A8E599F800504BF0010BA3E599F8005096
:100C400000287FF49FAD012320209BE599F80050F8
:100C50004BF0080B96E50D9B00228DF8672053F8AA
:100C6000042B0D9301238DF8902007930B9324AE52
:100C700071E6002B40F0DA863B4B12931BF020010B
:100C800025D00D9B073323F00703596853F8080B51
:100C90000D931BF0010F0BD050EA010308D0302355
:100CA0008DF868308DF869504BF0020B0223F9E59E
:100CB0000223F7E599F800504BF0400B62E5002B5A
:100CC00040F0A086294B12931BF02001D9D11BF0D4
:100CD000100340F05D831BF0400100F059830D9A32
:100CE00052F8040B0D92194680B2D2E70D9C089B76
:100CF00054F8046B00278DF86770002E00F0C8844C
:100D00005A1C00F0E9831A463946304602F000FAD0
:100D1000002800F05F86831B0B9323EAE3730D9496
:100D200008979DF86740CDF818B007930E97D4E662
:100D300099F800504BF0200B24E50D9B53F8040B61
:100D40000D93302378258DF86830084B12934BF0C3
:100D5000020B8DF8695000210223A3E5FFFFEF7F0E
:100D600048CF00084CCF00086CCF000858CF0008CF
:100D7000002B40F05F861BF0200F40F087831BF0B4
:100D8000100F40F0E1831BF0400F00F0DD830D9B5E
:100D9000099953F8042B0D931180D1E499F8005070
:100DA0006C2D03BF99F801504BF0200B09F101099C
:100DB0004BF0100BE6E4DDF818B0012B3FF4D1AE98
:100DC000022B00F08B802EAE00F00703C00840EA33
:100DD0004170C908303350EA0107324606F8013D38
:100DE000F2D11BF0010F00F08780302B00F08480DF
:100DF0003023023A06F8013C2EAB9B1ACDF818B00E
:100E00000B931646089B0B9A9342B8BF1346079361
:100E100000230E9361E6652D40F3F980DDE91001B2
:100E20000022002306F014FF002800F0DE81229B40
:100E3000C14ACAF80020013301340122072B239450
:100E40002293CAF8042000F3FC830AF1080A1B9BD2
:100E50000F9A934203DB069BD8077FF5D9AD139B0E
:100E6000149A1C44CAE90023229B23940133072BC4
:100E7000229300F300840AF1080A0F9B5D1E002DE7
:100E80007FF7C6AD102D229BAC4F40F3CE83DDF82B
:100E900030B0102605E00AF1080A103D102D40F38D
:100EA000C48301331034072BCAE90076CDE922341C
:100EB000F1DD21AA4146584602F0D0FF00287FF418
:100EC0002EADDDE922340DF1B80AE6E7012B00F082
:100ED0004C85022BDDF818B07FF475AF129A2EAE58
:100EE00000F00F030009D35C06F8013D40EA0170F1
:100EF000090950EA0103F3D12EAB9B1BCDF818B0C2
:100F00000B937FE70A9B079AA3EB020BBBF1000F41
:100F10007FF763ADBBF1100F229A884F26DD214683
:100F200010230C9C06E0ABF1100BBBF1100F0AF183
:100F3000080A1ADD01321031072ACAE90073CDE927
:100F40002221F0DD21AA414620460DF1B80A02F027
:100F500085FF00287FF4E3ACABF1100BBBF1100F61
:100F6000DDE922214FF01003E4DC0C4601325C4441
:100F7000072ACDE92224CAF80070CAF804B000F3A9
:100F80006D830AF1080A28E5BBF1100F229A6B4F16
:100F900026DD214610230C9C06E0ABF1100BBBF1C3
:100FA000100F0AF1080A1ADD01321031072ACAE9C6
:100FB0000073CDE92221F0DD21AA4146204602F04E
:100FC0004DFF00287FF4ABACABF1100BBBF1100F61
:100FD000DDE922210DF1B80A4FF01003E4DC0C46E4
:100FE00001325C44072ACDE92224CAF80070CAF80D
:100FF00004B000F3C0810AF1080AF6E40C9821AAB3
:10100000414602F02BFF00283FF416AD87E40F9B0A
:10101000012B40F35D81229DCAF800600135013447
:101020000123072D23942295CAF8043000F3C481CC
:101030000AF1080A139B149A01351C44072DCAE9CA
:101040000023CDE9225400F3C4810AF1080ADDE946
:1010500010010022002306F0FBFD002840F05F8114
:101060000F9B0135013B01361C44072DCAF8006077
:101070002295CAF80430239400F33B810AF1080A50
:10108000159BCAF8043001351C44072D1DABCDE972
:101090002254CAF800307FF7B9AC0C9821AA414617
:1010A00002F0DCFE00287FF43AAC239C0DF1B80A74
:1010B000AEE4102FDDE922212FDDCDE916354B46B8
:1010C0000C9DB14610243E4608464746984604E02B
:1010D000103E102E0AF1080A17DD0132184B1030AD
:1010E000072ACAE90034CDE92220F1DD21AA3946D8
:1010F00028460DF1B80A02F0B1FE00287FF40EACCC
:10110000103E102EDDE92220E7DCDDE91635014630
:101110004046B84637464E46814601327C18072A7B
:101120000749CAF80470CDE92224CAF8001000F378
:1011300035820AF1080A25E488CF000814CC00089B
:1011400004CC00080C98169321AA414602F086FEB2
:1011500000287FF4E4AB239C169B0DF1B80A26E42B
:101160000C9821AA414602F079FE00287FF4D7AB03
:10117000239C0DF1B80A2CE4102D229B1FDD0C9F3F
:10118000102604E0103D102D0AF1080A17DD013386
:101190009A4A1034072BCAE90026CDE92234F1DD42
:1011A00021AA414638460DF1B80A02F057FE002840
:1011B0007FF4B5AB103D102DDDE92234E7DC0133BF
:1011C0008E4ACAF804502C44072BCDE92234CAF8C1
:1011D00000207FF726AC0C9821AA414602F03EFE83
:1011E00000287FF49CAB239C1BE41B99002940F34F
:1011F000E481DDE90E379F42A8BF1F46002F0BDDBB
:10120000229B01333C44072BCAE9006723942293B5
:1012100000F3C2830AF1080A0E9D002FA8BFED1B40
:10122000002D00F369811B9D0F9B9D4280F2388148
:10123000139B149A1C44CAE90023229B2394013374
:10124000072B229300F31E830AF1080A0F9B0E9AC4
:101250005D1B9F1AAF42A8BF2F46002F0EDD229BB9
:10126000CAF80470013316443C44072BCAF80060E6
:101270002394229300F39F830AF1080A002FA8BF4A
:10128000ED1B002D7FF7C4AB102D229B5C4F40F36C
:10129000CC81DDF830B0102605E00AF1080A103DD7
:1012A000102D40F3C28101331034072BCAE90076B8
:1012B000CDE92234F1DD21AA4146584602F0CEFDA7
:1012C00000287FF42CABDDE922340DF1B80AE6E703
:1012D000069BDA073FF59FAE229DCAF800600135F4
:1012E00001340123072D23942295CAF804307FF797
:1012F000C5AE0C9821AA414602F0B0FD00287FF44B
:101300000EABDDE922540DF1B80AB9E6089B002BBB
:1013100040F02B83002308930B932EAE72E50F9BB6
:101320005E1E002E7FF7ACAE102E354F40F3F081DD
:10133000CDF820904FF0100BC146DDF8308005E06D
:101340000AF1080A103E102E40F3DF8101351034F7
:10135000072DCAE9007BCDE92254F1DD21AA4946D7
:10136000404602F07BFD002840F06883DDE922540E
:101370000DF1B80AE6E70C9821AA414602F06EFD8D
:1013800000287FF4CCAA239C0DF1B80AFFF72DBBEF
:101390000D9B53F8040B0D937BE4C1170B46002BF8
:1013A000BFF6D0AB40424FF02D0461EB41018DF808
:1013B00067400123FFF779BA0C9821AA414602F051
:1013C0004DFD00287FF4ABAADDE922540DF1B80AE7
:1013D00030E60C9821AA414602F040FD00287FF437
:1013E0009EAADDE922540DF1B80A30E699F80050C2
:1013F0000D92FFF7C7B92EAE04E500BF04CC00087C
:1014000014CC0008DDE9100102460B4606F052FC40
:10141000002840F03C83089B013325F020030B9308
:1014200000F0C682472B00F09780DDE910124BF4E4
:101430008073171E0693C0F23F82109B0793002310
:101440001693662D00F07081462D00F06D810B9B88
:10145000079A0C98452B1FA908BF089B04911CA94B
:1014600003911BA90CBF5C1C089C029102213B4606
:101470000194009100F032FC672D064640F0828214
:101480001BF0010F00F09881344464E10D9B099832
:1014900053F8041B0D93C217C1E90002FFF750B9BE
:1014A000069BD9073FF5C4AEDDE90E239F1A5D1BED
:1014B000AF42A8BF2F46E1E60C98402101F078FB2F
:1014C000C8F80000C8F81000002800F02D83402361
:1014D000C8F81430FFF726B930460D940897CDF8B8
:1014E00018B002F04DFC20EAE0739DF867400B90C5
:1014F00007930E97FFF7F1BA102D229BAB4F40F3E5
:10150000AF813A46089647460C9E4FF0100B904626
:1015100005E00AF1080A103D102D40F39D810133CA
:101520001034072BCAE9008BCDE92234F1DD21AA62
:101530003946304602F092FC00287FF4EFA9DDE93D
:1015400022340DF1B80AE6E70D9B099953F8042BF4
:1015500011600D93FFF7F4B8089B002B08BF01231F
:10156000089362E72EAE06950A22002307460D4631
:10157000FEF76AFE303206F8012D00233846294670
:101580000A22FEF761FE0A2F75F10003ECD22EABA2
:101590009B1B069D0B93CDF818B033E40C98169363
:1015A00021AA414602F05AFC00287FF4B8A9239CE6
:1015B000169B0DF1B80AFFF7E5B9229B7C4ACAF8E1
:1015C0000020013301340122072B23942293CAF80F
:1015D000042000F364810AF1080A002961D1069B06
:1015E0000F9A03F0010313433FF412AA139B1499BB
:1015F0001A19CAE90013229B23920133072B229365
:1016000000F366810AF1080A0F99CAF800600133F5
:101610008C18072BCDE92234CAF804107FF7F6A9FD
:101620003BE59DF86740FFF79CBA01332C44072B3C
:10163000CAF80070CAF80450CDE922347FF7E6A951
:101640002BE50C9821AA414602F008FC00287FF403
:1016500066A9239C0DF1B80AFFF7F9BB0C9821AAE3
:10166000414602F0FBFB00287FF459A9239C0DF1B1
:10167000B80AFFF7B2B90C9821AA414602F0EEFB76
:1016800000287FF44CA9239C0DF1B80AFFF7F5BBA5
:10169000062B28BF0623474E0B930D940793FFF7A5
:1016A0005AB9139B14981A19CAE90003229B239272
:1016B0000133072B229300F30B810AF1080A00295A
:1016C000A2DA4D421031394F80F2BB81DDF830B0E3
:1016D000102405E00AF1080A103D102D40F3B181F5
:1016E00001331032072BCAE90074CDE92232F1DD53
:1016F00021AA4146584602F0B1FB00287FF40FA909
:10170000DDE922320DF1B80AE6E7C846DDF820909F
:10171000CAF8007001353444072DCDE92254CAF8C7
:1017200004607FF7ABACE4E51FA904911CA9039109
:101730001BA9089C029103213B460194079A0C982F
:10174000009100F0CBFA064604193378302B00F0F4
:1017500090811B9B1C44079839460022002306F009
:1017600077FA002840F0AE801F9BA34206D23021BA
:101770005A1C1F9219701F9B9C42F9D89B1B0F93F8
:101780000B9B472B1FD0662D40F0D6811B9B0E93E1
:10179000002B0BF0010B40F3EC8008995BEA01028F
:1017A00040F098810E9B07930B9321E014CC000826
:1017B00088CF000880CF00081F9B9B1B0F930B9BBB
:1017C000472B40F0B9811B9B0E93D91C1BDB089A59
:1017D000934218DCDDE90E329342C0F207811BF020
:1017E000010F40F06E8123EAE37207920B936725A5
:1017F000169B002B00F0CA802D238DF86730002344
:101800000893FFF76DB9023D0E9A8DF87450531E80
:10181000002B1B93B6BFC2F101032B222D22092BF3
:101820008DF875206EDC30338DF8773030238DF8ED
:101830007630042315930F9A159B012A13440B93BA
:1018400040F336810B9B139A13440B9323EAE37303
:10185000079300230E93CBE74246089EB8461746EF
:1018600001332C44072BCDE92234CAF80070CAF8A2
:1018700004503BDC0AF1080AD5E42D248DF86740BA
:10188000FFF71DB90C9821AA414602F0E7FA00289B
:101890007FF445A81B9D239C0DF1B80AD6E40C9853
:1018A00021AA414602F0DAFA00287FF438A81B99F1
:1018B000239C0DF1B80A90E62D23079102F1004711
:1018C0001693BEE5234659E78DF86700FFF737B852
:1018D0000C9821AA414602F0C1FA00287FF41FA803
:1018E000DDE922321B990DF1B80AE8E60C9821AA2D
:1018F000414602F0B3FA00287FF411A8239C0DF1B1
:10190000B80A90E40DF183048D4F2246104687FB00
:101910000321DA17C2EBA10202EB8201A3EB410122
:10192000303100F8011C19466329134600F1FF32DB
:10193000ECDC3033D9B2831E9C4202F8011C40F229
:10194000F08013460DF1760201E013F8011B02F856
:10195000011B9C42F9D10DF185030DF176021B1A92
:1019600013441DAA9B1A159365E7DDF818B0FFF71D
:10197000FDB8089A5BEA020340F0B48001230793A4
:101980000B9335E7472D3FF47BAD7DE5169B9DF826
:1019900067400893FFF7A1B80C9821AA414602F0CE
:1019A0005DFA00287EF4BBAF239C0DF1B80A33E446
:1019B0000623089339E50C9821AA414602F04EFA15
:1019C00000287EF4ACAF1B9D0F9B239C5D1B0DF18B
:1019D000B80A53E4089B0D94CDF818B09DF8674001
:1019E00007930B9308900E90FFF777B8139A0F9B0D
:1019F00013440E9A0B93002A7CDD23EAE3730793CA
:101A00006725F5E68DF86700FFF75CB98DF867008C
:101A1000FFF728B800220892FEF7B6BE8DF86700DF
:101A2000FFF780B88DF86700FFF7E3B88DF867001F
:101A3000FFF722B98DF86700FFF79DB9C846FEF79A
:101A40006EBF01332A44072BCDE92232CAF8007059
:101A5000CAF804507FF7D6AD0C9821AA414602F08F
:101A6000FDF900287EF45BAFDDE922320DF1B80A02
:101A7000CAE5079839460022002306F0E9F8002855
:101A80007FF467AE089BC3F101031B9362E6119BD1
:101A90002C4E002BB8BF2D242BF080030693A8BF3B
:101AA0009DF86740284BB8BF8DF86740FFF70CB82A
:101AB0001BF001020E927FF4C5AE23EAE373079395
:101AC00096E60E9B139A13440B9323EAE373079352
:101AD00067258DE6139A1344194421EAE1730B91AB
:101AE000079385E6139B01331A4422EAE2730B92B3
:101AF00007937DE60E9B0B9AC3F101031A4422EA79
:101B0000E2730B920793672572E60D9A99F80150DC
:101B1000894652F8041B0D9241EAE1710891FEF7E3
:101B200031BE0223159386E60C9A0C2313604FF006
:101B3000FF330993FEF7FCBE1B9B0E9364E600BFC8
:101B40006766666650CF000854CF000870B4184C22
:101B50002568D5F848411CB365681F2D25DC38B9C8
:101B6000AB1C0135656044F82310002070BC704741
:101B700004EB850C0228CCF88820D4F888614FF05B
:101B8000010202FA05F246EA0206C4F88861CCF8BE
:101B90000831E5D1D4F88C311343C4F88C31DFE738
:101BA00005F5A674C5F84841D6E74FF0FF30DDE7EC
:101BB00000CC0008000000002DE9F04F03690C691B
:101BC000A34283B0C0F28680013C01F11405A3005A
:101BD00000F11408009355F8243058F824200133FC
:101BE0008A469A4208EB8401814605EB84070191FD
:101BF000B2FBF3F638D30023AE4640469B465EF870
:101C0000041B02681FFA81FC06FB0C33090C4FEA27
:101C1000134C06FB01CC99B2ABEB01011FFA8CF31C
:101C200011FA82F1C3EB124202EB214289B241EA7E
:101C30000241774540F8041B4FEA1C434FEA224B10
:101C4000DDD2009B58F8033073B9019B043B9845E3
:101C500004D307E0984504F1FF3403D253F8042974
:101C6000002AF7D0C9F810405146484601F01AFE44
:101C700000282BDB01364046002355F8041BD0F822
:101C800000C08AB29A1A0B0C12FA8CF2C3EB1C43F6
:101C900003EB224392B242EA0342AF4240F8042BE4
:101CA0004FEA2343E9D258F8242008EB84036AB9A9
:101CB000043B984504D307E0984504F1FF3403D270
:101CC00053F80429002AF7D0C9F81040304603B071
:101CD000BDE8F08F002003B0BDE8F08F2DE9F04F94
:101CE000016C99B090469946CDE90489259D04463A
:101CF00041B1426C4A60012393408B6001F01CFBB0
:101D000000232364B9F1000AB4BF012300232B6030
:101D1000754BBCBF2AF0004ACDF814A033EA0A0381
:101D200000F0AA80DDE904231046194600220023B2
:101D3000CDE90A0105F08CFF074670B1249A012312
:101D40001360269B002B00F0E28268481860431E57
:101D50000393039819B0BDE8F08F16AB019317AB4E
:101D600000932046DDE90A2301F0ECFE5FEA1A56F3
:101D7000054640F09780DDE916763E4406F2324093
:101D8000202840F3B383C0F140000AFA00FA06F2BB
:101D9000124028FA00F04AEA000005F077FC01231F
:101DA000013EA1F1F8710F93514B002205F030FB79
:101DB00047A3D3E9002305F0E3FC47A3D3E90023BD
:101DC00005F028FB80463046894605F06FFC44A3A9
:101DD000D3E9002305F0D4FC02460B4640464946B1
:101DE00005F018FB8046894605F07AFF00228346FD
:101DF00000234046494605F035FF002840F07A822E
:101E0000BBF1160F00F269823A4B03EBCB03D3E927
:101E10000023DDE90A0105F025FF002870D000232A
:101E2000BE1B0E93731E0BF1FF3B069300F15C8209
:101E300000230993BBF1000F69DA099BCDF81CB0B0
:101E4000A3EB0B030993CBF100030D93229B092B0A
:101E50004FF0000B64D8052B40F34683043B2293DC
:101E60000026229B023B032B00F26686DFE813F07C
:101E70005A0457044E043104249A42F20F73CAF3F1
:101E8000130A13605AEA08031AD1269B002B00F0AC
:101E90006286194B03930833269A0398136019B08E
:101EA000BDE8F08FDDE90A12C2F31303084643F0E0
:101EB0007F510F97A6F2FF36169F41F4401173E74A
:101EC000269B002B40F0E8830C4B039341E700BFB7
:101ED00061436F63A787D23FB3C8608B288AC63F30
:101EE000FB799F501344D33F0000F07F89CF000857
:101EF0000000F83F38CC000890CF00088CCF0008D5
:101F0000BE1B731E069300F185840E900990069BFC
:101F10005B44CDE9063B00230D93229B092B9AD904
:101F20000023CDE9223301264FF0FF330C960893AE
:101F3000089B129300216164204601F0D7F90390B9
:101F4000002800F00186039B2364089B0E2B00F2FF
:101F50001381002E00F010810799002940F35C8462
:101F6000AE4B01F00F0203EBC2034FEA2118C90583
:101F7000D3E9006740F11484A94BDDE90A01D3E9F4
:101F8000082305F027FDCDE9100108F00F084FF0F8
:101F9000030AB8F1000F13D0DFF8849218F0010F94
:101FA00009D030463946D9E9002305F0E9FB0AF1AA
:101FB000010A06460F465FEA680809F10809EDD1F3
:101FC000DDE9100132463B4605F004FD80468946B6
:101FD0000E9B43B1934B00224046494605F042FE1A
:101FE000002840F03085504605F060FB42464B46E5
:101FF00005F0C6FB8C4B002205F00CFAA1F15073E2
:10200000CDE910011193089B002B00F09780079BEE
:102010001493089B13930C9B002B00F0A584139A38
:102020007E4B8249039E03EBC20353E90223002047
:1020300005F0D0FCDDE9102305F0EAF9CDE9100147
:102040004946404605F04CFE074605F02FFB024688
:102050000B464046494605F0DBF93037DDE91023F1
:1020600006F8017B8046894605F0FCFD002840F01B
:102070002985CDF854B00027DDE910AB1095139DEC
:1020800013942AE00137AF4280F22C85684B50460A
:102090005946002205F074FB654B002282468B46B0
:1020A0004046494605F06CFB8946804605F018FE1F
:1020B000044605F0FBFA02460B464046494605F049
:1020C000A7F9303406F8014B52465B4680468946F4
:1020D00005F0C8FD002840F0F38442464B465149C4
:1020E000002005F095F952465B4605F0BBFD00283F
:1020F000C8D0DDE91343109D039A079302E096428E
:1021000000F0C884B24616F8013D392BF7D00133F0
:10211000DBB23370079B01330793C8E1504605F0EB
:10212000C5FA42464B4605F02BFB3F4B002205F01B
:1021300071F9A1F15073CDE9100111933D4B404667
:102140004946002205F064F9DDE910894B46424614
:1021500006460F4605F0A4FD8146002840F0AA84FB
:10216000DDE91001024601F100433046394605F031
:1021700079FD002840F04583179B002BC0F28C802E
:10218000079A0E2A00F38880244B03EBC203D3E99D
:1021900000AB239B002B1BDA089B002B18DC40F0C4
:1021A0002E83244B00225046594605F0E9FA024698
:1021B0000B46DDE90A0105F05FFDDDF820904E4693
:1021C000002800F0C782239BDDF80C80DF43C9E2C2
:1021D000DDE90A7852465B463846414605F0FAFB8F
:1021E00005F07EFD8146099005F060FA52465B4697
:1021F00005F0C6FA039E0B4602464146384605F0F6
:1022000007F909F1300306F8013B089B012B00F0A8
:102210005C830694012704951C462AE038CC00080C
:1022200028CD00080000F03F00001C400000E03F07
:10223000000024400000144052465B464046494698
:1022400005F0C8FB05F04CFD054605F02FFA524697
:102250005B4605F095FA01370B4602464946404673
:1022600005F0D6F805F13003A74206F8013B00F06F
:102270002983AC4B002205F083FA0022002380461C
:10228000894605F0E5FC0028D6D0049D069C079BF6
:1022900001330793B2460AE10C9A002A3DD0229AF4
:1022A000012A40F39C82089B03F1FF380D9B4345B4
:1022B000C0F26D82A3EB0808089B002BC0F23C83A0
:1022C000069A1A440692099A17461A44099201215D
:1022D000204601F033F9064623E00123BE1B0E938E
:1022E000731E06937FF5A4ADC6F101030993002385
:1022F00006939FE5584605F0D9F942464B4605F04E
:10230000A7FC00287FF47CAD0BF1FF3B78E5864B02
:102310000393039819B0BDE8F08FDDF83480099F6E
:102320000C9E002F0CDD069900290B4608DD099A4A
:10233000B942A8BF3B46D21AFF1ACB1A099206939C
:102340000D9BDBB10C9B002B00F05D82B8F1000F00
:102350000FDD31464246204601F0CCF92A460146BF
:102360000646204601F018F929460546204600F0A9
:10237000E3FF0D9BB3EB080240F0D8820121204619
:1023800001F0DCF8BBF1000F814600F3B480229B22
:10239000012B40F386814FF0000A0120BBF1000FB2
:1023A00040F0B580069A104410F01F0000F09380B2
:1023B000C0F12003042B40F3D283099BC0F11C0021
:1023C00003440244099307440692099B002B05DD50
:1023D00029461A46204601F0EDF90546069B002BDA
:1023E00005DD49461A46204601F0E4F981460E9B78
:1023F000002B40F03681089B002B40F31D810C9B85
:10240000002B40F0A080079B01330793DDF80C8080
:10241000DDF820A0012707E0294600230A222046F4
:1024200000F094FF0137054649462846FFF7C4FBF4
:10243000574500F1300308F8013BEDDB089A002A0C
:10244000C8BF9346039AD8BF4FF0010B93440027AF
:10245000294601222046049301F0ACF9494605467D
:1024600001F020FA002840F3A8811BF8013C039AF0
:102470000BF1FF3B04E05A4500F0AA811BF8013D37
:10248000392B0BF1010AF6D001338BF800304946A5
:10249000204600F051FF56B12FB1B74203D0394664
:1024A000204600F049FF3146204600F045FF29460E
:1024B000204600F041FF00238AF80030249B079A51
:1024C0001A60269B002B3FF444AC0398C3F800A08D
:1024D00019B0BDE8F08F1C20099B03440993069BAB
:1024E00003440744069370E70126BAE4C0F12000D4
:1024F00008FA00F051E401465A46204601F0FAF885
:10250000229B012B814640F3B3814FF0000AD9F89A
:10251000103009EB8303186900F0C2FFC0F12000FE
:1025200040E700BF0000244088CF00083146002368
:102530000A22204600F00AFF129B002B064640F3B9
:10254000E782CDE90783002F00F31A81BAF1000F6B
:1025500040F0D581B046049B039F089903F0010227
:102560007B1E1944229B0C92134309910A934946FE
:102570002846FFF721FB31468346284601F092F9B1
:10258000424649468246204601F0ACF9C2680146FF
:102590000BF13003002A42D106902846089301F03F
:1025A00081F906990490204600F0C6FE049A089B23
:1025B0001AB90A99002900F09B82BAF1000FC0F203
:1025C000638122994AEA010A0C9951EA0A0100F052
:1025D0005B81002A00F3B481099A3B7007F1010A7C
:1025E0009742D34600F0B281294600230A222046B2
:1025F00000F0ACFE4645054631464FF000034FF073
:102600000A02204612D000F0A1FE414606460023F1
:102610000A22204600F09AFE57468046A7E7204649
:10262000049300F089FE049B0122C6E700F08EFEB1
:102630005746064680469AE7229B022B79DC0C9B84
:10264000002B80D1079B4946013328460793FFF7AB
:10265000B3FADDF80CB000F130030BF8013B0027B2
:10266000F6E64946284601F01DF90028BFF6C3AE3C
:10267000294600230A22204600F068FE079B03F14A
:10268000FF380C9B0546002B7FF450AF129B002BAC
:1026900040F335820893B9E6AF4B03930333FFF75A
:1026A000FBBBDDE9041200297FF475AEC2F313030E
:1026B000002B7FF470AEA94B1340002B00F0FE817D
:1026C000099B01330993069B013306934FF0010ADE
:1026D00063E601230C93239B079A1344129301335F
:1026E000012B1F460893B8BF01270021172F6164F3
:1026F0007FF722AC012204235B0003F11400B842EF
:10270000114602F10102F7D9616415E401230C932B
:10271000239B002B4CDD129308931F46E5E7002313
:102720000C93D8E700230C93F2E7129BCDF81C80A2
:102730000893089B002B7FF446AD494605222046AE
:1027400000F004FE01468146284601F0ABF800285F
:102750007FF739AD0398079F3123804600F8013B8E
:10276000013703904946204600F0E6FD7B1CDDF86A
:102770000CA00793CDF80C80002E7FF494AE96E663
:1027800031463A46204601F015F80646DEE60D9B36
:10279000CDF83480A8EB03039B444FF000088BE591
:1027A000DDE90A234FF0020ACDE91023FFF7F1BB60
:1027B000012323930893FFF7BBBB03D1049BDB07E3
:1027C0003FF553AEDA461BF8013D302BFAD05EE6FA
:1027D000079B039A013307933123137057E60F9A2F
:1027E000002A00F0268103F23343069ADDF8348094
:1027F0001A440692099A17461A44099267E54FF05F
:1028000000094E46DFE429460D9A204600F072FF8B
:102810000546B3E50E9067E500F00F81079A504B2F
:10282000564206F00F0203EBC203D3E90023DDE9B1
:102830000A0104F0A5FF36118046894600F0718137
:10284000484F00234FF0020AF20706D5D7E90023CC
:1028500004F096FF0AF1010A0123761007F1080738
:10286000F2D1002B3FF4B4AB80468946FFF7B0BBF2
:10287000049B002B7FF449AEDDE90412C2F313037D
:10288000002B3FF418AF40E6002A12DD2946012252
:102890002046049300F08EFF4946054601F002F8F9
:1028A0000028049B40F31881392B00F0F9800BF1CC
:1028B0003103BA460AF8013B079B013337460793B9
:1028C0004646E4E50995069C049D02460B4604F045
:1028D000A1FD52465B468046894605F0E1F960B9A4
:1028E00052465B464046494605F0B2F900283FF49F
:1028F000CEAC099BD9077FF5CAAC039A02E4716894
:10290000204600F0F3FC0746002800F00E813369F2
:1029100002339A0006F10C010C3000F049FC3946F4
:102920000122204600F046FF804614E62946204654
:1029300000F0E0FE054621E5DDE908239F1AC6E424
:10294000392B00F0AD80BA460133B3E7079A013264
:102950003746079246467BE58CCF00080000F07FA3
:1029600038CC000828CD0008DDF84CA0844901EBE4
:10297000CA01DDE9102351E9020104F001FFCDE9AC
:1029800010014946404605F0ABF9064604F08EFEBC
:102990000B4602464946404604F03AFD039F534623
:1029A0003036012B07F8016B8046894600F0AE8077
:1029B000139E039B1E44734B00224046494604F07D
:1029C000DFFE8946804605F08BF9824604F06EFEF4
:1029D0000AF1300A02460B464046494604F018FD0B
:1029E00007F801ABB74280468946E4D1664B002226
:1029F000DDE9100104F00EFD42464B4605F032F9C8
:102A0000002864D1DDE910235F49002004F000FDB7
:102A100042464B4605F044F900283FF4ADABB246C0
:102A2000013E1AF8013C302BF9D0149B0133079377
:102A30003DE5169BC3F13603D7E6DDE90A894FF081
:102A4000020AFFF7C5BA089B002B3FF467AB129B45
:102A5000002B7FF791AB079A013ACDE9133240463C
:102A6000484B0022494604F08BFE804689460AF115
:102A7000010004F01BFE42464B4604F081FE434B2E
:102A8000002204F0C7FCA1F15073CDE910011193AD
:102A9000FFF7C1BA079B013307933123FFF739BB17
:102AA000079BBB4601330793392337460BF8013B9D
:102AB0004646DCE44FF000094E464BE69A466CE48D
:102AC000109D139C149B01330793B246EFE4149BB3
:102AD000039A0793FFF716BB7FF4EBAEDA077FF597
:102AE000E8AEE1E6DDF854B0109D139CFFF744BB5F
:102AF000392BD5D0BAF1000F3FF7D9AED9E6229BDA
:102B0000022B3FF712AECDF81C809BE53E466DE7E9
:102B1000229B022B3FF709AE129BCDF81C80089335
:102B200011E54FF0020AFFF753BA194B19483A461C
:102B300040F2EA2101F03CFF00266664314620465F
:102B400000F0D4FB039078B9114B124800224FF4E7
:102B5000D57101F02DFF104B0393FFF7FAB83FF446
:102B600034ACC0F13C00B7E4039B236401224FF076
:102B7000FF33239612930C920893FFF7FDBA00BF20
:102B800038CC0008000024400000E03F00001C405A
:102B90009CCF0008B0CF000890CF0008F0307047FD
:102BA0000048704730090020004870473009002075
:102BB0002DE9F04F01F10B06162E83B0044624D800
:102BC000102900F2BA8000F08DFB10261822022096
:102BD000B74F3A44A2F1080153688B4200F0BA8023
:102BE0005A68D96822F003021A449D68E9608D6032
:102BF000516841F001012046516003F1080500F0E1
:102C000073FB284603B0BDE8F08F36F0070600F1ED
:102C10009480B14200F2918000F064FBB6F5FC7F35
:102C2000C0F09681730A00F08F80042B00F26B8154
:102C3000B30903F1390003F1380CC3009C4F3B4446
:102C4000A3F108055B689D4206D10CE0002980F2E3
:102C50002B81DB689D4206D05A6822F00302911B4B
:102C60000F29F3DD60463D69DFF848C265457CD039
:102C70006A6822F00302931B0F2B00F37781002B6D
:102C8000C7E904CC80F26881B2F5007F80F016813C
:102C9000D308796801334FEA521E012202FA0EF27C
:102CA0000A4357F833E0C5F808E007EBC3010839D9
:102CB000E9607A6047F83350CEF80C508310012158
:102CC0009940914257D8114206D120F003004900A3
:102CD000114200F10400FAD007EBC0094D468646C8
:102CE000D5F80C80454508D119E1002B80F22081F0
:102CF000D8F80C80454500F01281D8F8042022F065
:102D00000302931B0F2BF0DD2046D8E9025408EB99
:102D1000060146F00106C8F80460EC60A56043F0C7
:102D20000104C7E90411C1E902CC4C6048F8023043
:102D300000F0DAFA08F1080502E00C232360002510
:102D4000284603B0BDE8F08F4FF4007340204FF0E9
:102D50003F0C73E7D3689A4208BF02307FF440AF5C
:102D60003D69DFF850C1654582D17A688310012141
:102D700099409142A7D9BD686B6823F00308464586
:102D800003D8A8EB06030F2B7EDCDFF82C91D7F8D5
:102D90000824D9F800300132334405EB080A00F06A
:102DA0002F8103F580530F3323F47F6B2BF00F0B30
:102DB0005946204600F0D0FF411C024600F0EF804B
:102DC000824500F2EA80D9F804105944C9F8041089
:102DD0000B4600F04B81D7F8081401311BBFA2EB62
:102DE0000A0A5344C7F80824C9F8043012F007034C
:102DF00000F01281C3F108010A44C3F580519344E5
:102E00000831A1EB0B01C1F30B0A51462046019298
:102E1000009300F0A1FF421CDDE9003200F04B817D
:102E2000831A03EB0A0BD9F80400BA604BF00103D4
:102E30000AEB0001BD425360C9F8041000F0228182
:102E4000B8F10F0F40F220816B68A8F10C0020F060
:102E5000070003F0010303436B604FF0050C2B18D0
:102E60000F28C3E901CC00F22D8153681546D9F82B
:102E70002C208A42D9F8302038BFC9F82C108A4259
:102E800038BFC9F830108CE0AA1943F0010346F0AE
:102E900001066E602046BA60536000F025FA0835DE
:102EA000284603B0BDE8F08FD9681A449DE600BFFC
:102EB0003004002038040020C40A0020B2F5206F3E
:102EC0004FEA522363D3142B00F2B88003F15C0164
:102ED000C9005B3307EB010E7958AEF1080E8E4541
:102EE00000F091804B6823F00303934202D9896874
:102EF0008E45F7D1D1F80CE07A68C5E9021ECEF80C
:102F00000850CD60DAE6142B59D9542B00F29E807C
:102F1000330B03F16F0003F16E0CC3008EE60EF16C
:102F2000010E1EF0030F05F108057FF4D9AE51E044
:102F3000424445465368D8F80C1043F001035360EF
:102F400055F8083F2046D9608B6000F0CDF9F7E6D0
:102F5000F00806F108023BE62A442046536843F095
:102F600001035360083500F0BFF9E9E6A9192046CE
:102F700046F0010643F001046E60C7E90411C1E99F
:102F800002CC4C60AB5000F0AFF90835D8E693099D
:102F900003F13901C90038339CE7BD4260D0BD68F8
:102FA0006B6823F0030B5E45ABEB060302D80F2BD7
:102FB0003FF76AAF204600F097F90025C0E603F11D
:102FC0005C0003F15B0CC30038E659F808394B4547
:102FD00040F0968010F0030F00F1FF30F5D17B68D0
:102FE00023EA01037B60490099423FF6C4AE19B958
:102FF000C1E649000EF1040E1942FAD070466BE6A4
:1030000003F1100BD4E69A104FF001087B6808FA20
:1030100002F21A437A6070E702EB0B014942C1F3F6
:103020000B0A514620460193009200F095FE431C86
:10303000DDE900237FF4F4AE9A46F4E6542B26D85B
:10304000130B03F16F01C9006E3343E7B3F5AA7F99
:1030500026D8F30B03F1780003F1770CC300EDE5FC
:10306000D9F804305B44C9F80430B4E6CAF30B0065
:1030700000287FF4B0AEBD6808EB0B0343F00103FA
:103080006B60F4E61546F2E60123536092E7B3F570
:10309000AA7F21D8D30B03F17801C900773319E750
:1030A00040F25452934221D8B30C03F17D0003F156
:1030B0007C0CC300C2E5083B9B44ABEB020B4FF01A
:1030C000000AB0E605F10801204601F039FDBD68AF
:1030D000D9F804106B68CAE640F254518B420BD801
:1030E000930C03F17D01C9007C33F3E64FF47E734A
:1030F0007F204FF07E0CA1E54FF47E717E23E9E640
:103100007B6870E700000000000000000000000085
:1031100001F0FF01102A2BDB10F0070F08D010F888
:10312000013B013A8B422DD010F0070F42B3F6D18C
:10313000F0B441EA012141EA014122F007047FF0A5
:1031400000070023F0E80256083C85EA010586EAFC
:10315000010685FA47F5A3FA87F586FA47F6A5FA38
:1031600087F68EB9EED1F0BC01F0FF0102F0070244
:1031700032B110F8013B013A83EA010313B1F8D1EF
:103180000020704701387047002D06BF35460338D0
:10319000073815F0010F07D1013015F4807F02BF09
:1031A000013015F4C03F0130F0BC0138704700BF5A
:1031B000844641EA000313F003036DD1403A41D342
:1031C00051F8043B40F8043B51F8043B40F8043B01
:1031D00051F8043B40F8043B51F8043B40F8043BF1
:1031E00051F8043B40F8043B51F8043B40F8043BE1
:1031F00051F8043B40F8043B51F8043B40F8043BD1
:1032000051F8043B40F8043B51F8043B40F8043BC0
:1032100051F8043B40F8043B51F8043B40F8043BB0
:1032200051F8043B40F8043B51F8043B40F8043BA0
:1032300051F8043B40F8043B51F8043B40F8043B90
:10324000403ABDD2303211D351F8043B40F8043B30
:1032500051F8043B40F8043B51F8043B40F8043B70
:1032600051F8043B40F8043B103AEDD20C3205D340
:1032700051F8043B40F8043B043AF9D2043208D038
:10328000D2071CBF11F8013B00F8013B01D30B88AA
:1032900003806046704700BF082A13D38B078DD088
:1032A00010F003038AD0C3F10403D21ADB071CBF5A
:1032B00011F8013B00F8013B80D331F8023B20F8C4
:1032C000023B7BE7043AD9D3013A11F8013B00F8FD
:1032D000013BF9D20B7803704B7843708B78837085
:1032E00060467047704700BF704700BFC36C70B541
:1032F00005460C464BB153F8240080B1026843F8F0
:1033000024200023C0E9033370BD2122042101F0F1
:1033100075FB0346E8640028EDD1002070BD012153
:1033200001FA04F6721D9200284601F067FB00289E
:10333000F3D0C0E90146E4E731B1C36C4A6853F801
:103340002200086043F82210704700BF2DE9F041C9
:103350000D6907460E461C4601F1140E0020DEF8EA
:1033600000108BB202FB03434FEA134C090C02FB23
:1033700001CC01309BB203EB0C4385424EF8043B79
:103380004FEA1C44EBDC3CB1B368AB4207DD06EB13
:10339000850301355C6135613046BDE8F0817168B7
:1033A00038460131FFF7A2FF8046A8B132690232E8
:1033B00006F10C0192000C30FFF7FAFEFB6C72680C
:1033C00053F82210316043F82260464606EB85032D
:1033D00001355C613561DFE7024B03484246B521A8
:1033E00001F0E6FA9CCF0008E4CF00082DE9F8438D
:1033F0000C4628491E46174603F1080281FB02319C
:10340000092E4FEAE2730546C3EB610339DD4FF045
:10341000010C00214FEA4C0C634501F10101F9DC7C
:103420002846FFF763FF014668B3089B4361092FF5
:103430004FF00103036112DC0A340927BE420BDDA1
:10344000F61B264414F8013B0A22303B2846FFF7BE
:103450007DFFA6420146F5D10846BDE8F88304F198
:103460000909C8463C4418F8013B0A22303B28466B
:10347000FFF76CFFA0450146F5D1A7F108044C44C5
:10348000DCE70021CCE70A46034B0448CE2101F0DB
:103490008FFA00BF398EE3389CCF0008E4CF0008D4
:1034A000020C12040346CAB90304102013F07F4F24
:1034B00004BF1B02083013F0704F04BF1B0104301F
:1034C00013F0404F04BF9B000230002B05DB13F0CC
:1034D000804F00F1010008BF202070470020E5E781
:1034E0000368024613F0070007D0D9071DD49807D8
:1034F0001FD55B0813600120704799B209B91B0CF6
:103500001020D9B209B908301B0A190704BF1B09DA
:103510000430990704BF9B080230D90703D45B0825
:1035200000F1010003D01360704700207047202095
:1035300070479B0813600220704700BF38B5C36C0A
:1035400004460D464BB15868B0B102685A6000227B
:103550000123C0E90435C26038BD2122042101F0F5
:103560004DFA0346E0640028EDD1094B09480022DA
:103570004FF4A07101F01CFA1C220121204601F039
:103580003DFA0028F1D001220223C0E90123DEE741
:103590009CCF0008E4CF00082DE9F04F0E691569B3
:1035A000AE4285B08846144605DB2A46234635469A
:1035B0000C4616469846A3686168AF19BB42B8BF6F
:1035C0000131FFF793FE0190002800F08780019BF6
:1035D00003F1140909EB870AD14505D24B460022B5
:1035E00043F8042B9A45FBD808F1140808EB860B26
:1035F00004F11403D8451A4603EB85055FD22B1B53
:10360000153B23F0030304331534A54238BF0423CC
:10361000CDE902A7AC461F46924605E0000C29D131
:10362000C34509F1040948D958F8040B85B2002DA7
:10363000F4D056464C46002356F8040B216882B25B
:103640001FFA81FE05FB02EE000C0A0C734405FB19
:10365000002202EB13429BB243EA0243B44544F812
:10366000043B4FEA1243E7D849F8073058F8040CF6
:10367000000CD5D0D9F80030544619464D460022EA
:103680002688090C00FB06110A449BB243EA024358
:1036900045F8043B54F8046B2968360C8BB200FBE8
:1036A000063303EB1243A4454FEA1342E8D8C3455F
:1036B00049F8073009F10409B6D8DDE902A7002F5F
:1036C00002DC05E0013F03D05AF8043D002BF9D09D
:1036D000019B18461F6105B0BDE8F08F034B0448FD
:1036E000019A40F25D1101F063F900BF9CCF000820
:1036F000E4CF000812F003032DE9F041144606461A
:1037000032D10D46A41020D0D6F84880B8F1000F71
:1037100033D0E3074FF0000707D4641015D0D8F872
:103720000000A8B18046E307F7D542462946304657
:10373000FFF732FFB5B16968F36C641053F82120CC
:103740002A6043F821500546E9D12846BDE8F081BA
:10375000424641463046FFF71FFFC8F800000760A9
:103760008046E0E70546D8E7013B0F4A52F82320A0
:103770000023FFF7EBFD0546C4E701213046FFF7C4
:10378000B5FD804640B1012340F27122C0E9043208
:103790000023B0640360BCE7044B054842464FF485
:1037A000A07101F005F900BF28CC00089CCF0008EB
:1037B000E4CF00082DE9F0470C4690462669A3683F
:1037C000496806EB6216751C9D4207464FEA62196E
:1037D00004DD5B009D4201F10101FADC3846FFF790
:1037E00085FD8446002851D0B9F1000F00F1140086
:1037F0000EDD09F105024FEA820E03460CEB820250
:10380000002143F8041B9342FBD1AEF1140318448A
:10381000216904F1140318F01F0803EB81012DD076
:10382000C8F1200986464FF0000A1A6802FA08F229
:1038300042EA0A024EF8042B53F8042B994222FA6A
:1038400009FAF2D80B1B153B23F00303043304F1F0
:103850001502914238BF0423BAF1000F18BF2E465B
:1038600040F803A0FB6C6268CCF8106053F822109B
:103870002160604643F82240BDE8F087043853F8E1
:10388000042B40F8042F9942F9D8EBE7034B044886
:10389000624640F2D91101F08BF800BF9CCF0008BE
:1038A000E4CF00080B6984460069C01A15D10CF1F9
:1038B000140C14310CEB830210B401EB830301E010
:1038C000944508D252F8044D53F8041D8C42F7D0A9
:1038D00004D24FF0FF3010BC70477047012010BC7D
:1038E000704700BF2DE9F84F0F691369FF1A002FC9
:1038F0000E4690467AD101F11405143202EB830290
:1039000005EB830301E09D4273D253F8041D52F886
:10391000044DA142F7D064D37168FFF7E7FC8146FC
:10392000002872D03569D8F81020C76008F1140E4D
:1039300006F1140009F1140A06F1100C0EEB8202D4
:1039400000EB8507564600215EF8044B5CF804BF87
:10395000A3B211FA8BF1CB1A210CC1EB1B4101EB85
:1039600023419BB243EA0143724546F8043B4FEAC8
:103970002141E9D8A2EB0804153C08F1150842459D
:1039800024F0030606F1040638BF0426304424F070
:10399000030238BF002287425244B24416D9564629
:1039A000044654F8043B11FA83F10A1402EB134263
:1039B00089B241EA0243A74246F8043B4FEA22415A
:1039C000EFD87A1E101A20F00302524423B952F89D
:1039D000043D013D002BFAD0C9F810504846BDE81F
:1039E000F88F334601274646984695E7F9DB0027CE
:1039F00092E70021FFF77AFC814668B1012200239B
:103A0000C9E904234846BDE8F88F074B07484A46F2
:103A10004FF4107100F0CCFF034B04484A4640F2CB
:103A2000322100F0C5FF00BF9CCF0008E4CF0008A2
:103A30000F4B0B40A3F15073002B02DD0020194601
:103A400070475B42B3F1A07F4FEA235205DA4FF48F
:103A50000023002043FA02F17047143A1E2ADABF0D
:103A60004FF0004323FA02F2012200211046704772
:103A70000000F07F2DE9F843066900F1140808EB17
:103A80008606A6F1040956F8047C3846FFF708FDBF
:103A9000C0F120030A280B6036DDC8451ED2B0F104
:103AA0000B0356F8082C26D0C3F1200C22FA0CF197
:103AB0009F400F43A6F1080147F07F55884545F424
:103AC00040153AD202FA03F056F80C3C23FA0CF3F4
:103AD00003431C4620462946BDE8F883B0F10B039A
:103AE00008D007FA03F343F07F55002345F440154F
:103AF0001C46EFE71A4647F07F5545F4401514463B
:103B000020462946BDE8F883C0F10B0327FA03F2EB
:103B1000C84542F07F553CBF56F8082CDA4000F10A
:103B2000150328BF002207FA03F345F4401543EAC2
:103B3000020420462946BDE8F88302FA03F31C4636
:103B4000C8E700BF70B5012182B016461D46FFF7D9
:103B5000CDFB044600284BD02B46C5F30A55C3F3D2
:103B600013030DB143F48013002E019322D0684655
:103B70000096FFF7B5FC002836D0019B0099C0F1F4
:103B8000200203FA02F20A43C34001936261002B50
:103B900014BF02210121A3612161ADB1069AA5F2F2
:103BA000334303441360079BC0F13500186020467F
:103BB00002B070BD01A8FFF793FC019B0121C4E98D
:103BC00004132030002DE9D104EB8102A0F232432E
:103BD0001069069A1360FFF763FC079BC0EB411165
:103BE0002046196002B070BDDDE900236261CEE7B6
:103BF000034B0448224640F20A3100F0D9FE00BFD0
:103C00009CCF0008E4CF00082DE9F04383B00F46B5
:103C100069468046FFF72EFF04460D46384601A947
:103C2000FFF728FFD8F810303A690F469A1ADDE9F5
:103C30000013CB1A03EB4213002B06460BDD05EBFA
:103C400003594D4632463B462046294603F0C2FE04
:103C500003B0BDE8F083C3EB033307EB03510F461A
:103C6000F0E700BF172870B506460ADD0849094D80
:103C70000020002422462B4603F082FD013EF9D1AC
:103C800070BD054B03EBC006D6E9040170BD00BF53
:103C90000000F03F0000244028CC00080139491101
:103CA00001F1010C116902F1140303EB81018B4254
:103CB00000EB8C0C16D210B5A0F1040E53F8044B97
:103CC0004EF8044F9942F9D88B1A153B23F00303A1
:103CD00004331844844504D9002340F8043B844548
:103CE000FBD810BD844505D9002340F8043B84452A
:103CF000FBD87047704700BF03694A11934200F137
:103D0000140009DA00EB830302E053F8042DC2B972
:103D10008342FAD80020704710DD11F01F010DD04A
:103D200010B450F8224000EB820324FA01F202FAA8
:103D300001F18C420BD0012010BC704700EB8203D4
:103D4000E6E70120704753F8042D002AF3D183429F
:103D5000F9D8002010BC704738B5074D0022044642
:103D600008462A6004F06CFC431C00D038BD2B6868
:103D7000002BFBD0236038BDF80A002000000000B3
:103D800090F800F06DE9024520F007016FF0000C9B
:103D900010F0070491F820F040F049804FF0000443
:103DA0006FF00700D1E9002391F840F000F108001E
:103DB00082FA4CF2A4FA8CF283FA4CF3A2FA8CF356
:103DC0004BBBD1E9022382FA4CF200F10800A4FABD
:103DD0008CF283FA4CF3A2FA8CF3E3B9D1E9042311
:103DE00082FA4CF200F10800A4FA8CF283FA4CF348
:103DF000A2FA8CF37BB9D1E9062301F1200182FA02
:103E00004CF200F10800A4FA8CF283FA4CF3A2FA07
:103E10008CF3002BC6D0002A04BF04301A4612BA15
:103E2000B2FA82F2FDE8024500EBD2007047D1E918
:103E3000002304F00305C4F100004FEAC50514F0A7
:103E4000040F91F840F00CFA05F562EA05021CBF78
:103E500063EA050362464FF00004A9E72DE9F04F3D
:103E6000936883B09146002B6DD017688D688046AB
:103E70000C460868083743E0A38913F4906F2ED0EE
:103E8000D4E90415A0EB010A05EB450505EBD57552
:103E90000AEB06006D100130A8422A4684BF054691
:103EA0002A465B0536D511464046FEF781FE0028BE
:103EB0003AD0524621690190FFF77AF9A289019B15
:103EC00022F4906242F08002A281A5EB0A0203EB89
:103ED0000A006561A260236120603546B2465946FA
:103EE000524600F099FFD9F80830A16820684D1BB0
:103EF00050449E1BA5602060C9F808601EB30837B7
:103F000057E902B6002EFAD0B542AA46B4D93546D2
:103F1000B246E4E7404600F0FBFF03460028D4D158
:103F20002169404600F00CFE0C23C8F80030A3893C
:103F3000002243F040034FF0FF30A381C9E9012282
:103F400003B0BDE8F08F0020C9F8040003B0BDE85D
:103F5000F08F00BF2DE9F04FABB0174606938B8969
:103F60001A068846834603D50B69002B00F0A5840A
:103F70001AAB0D930023CDE90E3309930DF16809B7
:103F800003935E463B78002B00F036813C4604E00C
:103F900014F8013F002B00F05781252BF8D1E51BC9
:103FA00040F054812378002B00F0268100214FF04F
:103FB000000263788DF82F20671C08464FF0FF3B06
:103FC00005918A460137A3F12002582A00F2588150
:103FD000DFE812F0AB0256015601A7025601560166
:103FE00056015601560156019D02990256013601AD
:103FF000800256017C0259005900590059005900AD
:1040000059005900590059005601560156015601F0
:1040100056015601560156015601560162025601DB
:1040200056015601560156015601560156015601D8
:1040300056012301560156015601560156016800EA
:1040400056015601160256015601560156015601F7
:1040500056015601560156015601070285015601C7
:10406000560156015E028501560156015402560161
:104070003E0225012D02E2015601C10156016A00EE
:1040800056015601E601A3F13002002417F8013B66
:1040900004EB840402EB4404A3F13002092AF5D9AD
:1040A000059490E74AF0100A1AF0200100F0098107
:1040B000069B073323F00703596853F8080B069350
:1040C00001234FF000028DF82F2000220792BBF150
:1040D000FF3F00F033822AF08002029250EA010290
:1040E00040F02A82BBF1000F40F00E84002B40F01C
:1040F0008A831AF00103049300F0878330238DF83C
:1041000067300DF16704049A079B5A45B8BF5A46B9
:10411000019213B1134601330193029B13F0020382
:10412000079302D0019B02330193029B13F0840397
:10413000089305D1059B019A9D1A002D00F3CB82AF
:10414000DDE90E219DF82F0080B101320DF12F0025
:104150000131C9F80000072A4FF00100CDE90E2116
:10416000C9F8040000F3F18209F10809079B7BB14B
:1041700001320CAB0231C9F80030072A4FF00203BC
:10418000CDE90E21C9F8043000F3EC8209F10809E9
:10419000089B802B00F00882049BABEB0305002DED
:1041A00000F34582049BC9F8004001321944072AF4
:1041B000CDE90E21C9F8043000F3788209F108092D
:1041C000029B5B0705D5059B019A9C1A002C00F306
:1041D000D682039B059A01988242ACBF9B181B189C
:1041E0000393002940F06E8200230E933B780DF17B
:1041F0006809002B7FF4CAAE0F9B002B40F0A08310
:10420000B8F80C3013F0400F039B18BF4FF0FF338A
:10421000039303982BB0BDE8F08F4AF0100A1AF010
:10422000200141D0069B073323F00703596853F858
:10423000080B0693002344E7059A5242CDE9052373
:104240003B784AF0040ABDE6E51BD5D00F9B2B4412
:104250000F930E9B0133072BC9E900750E9305DC04
:1042600009F10809039B2B4403939BE60DAA4146E1
:104270003046FFF7F3FD0028C2D10DF16809F1E7E0
:10428000002940F06383002BB6D08DF840304FF00A
:1042900000038DF82F3001230193049310ACCDF867
:1042A00008A04FF0000B38E71AF0100347D11AF0BE
:1042B000400144D0069A52F8040B0692194680B287
:1042C000FFE61AF0100340D11AF040013DD0069AE3
:1042D00052F8040B0692194680B20123F1E6002938
:1042E00040F04B831AF0200F069B00F0DF8007336D
:1042F00023F007031A465B6852F8080B069219462A
:10430000002BC0F28E82BBF1FF3F00F0F9829DF8D6
:104310002F30079350EA01032AF0800A00F06D82E3
:104320000A2871F1000380F09282303001238DF869
:104330006700CDF808A004930DF16704E3E6069B3F
:1043400053F8040B06930B46BBE6069B53F8040B8D
:1043500006930123B5E6069D55F8044B4FF0000384
:104360008DF82F30002C00F0E282BBF1FF3F00F00F
:1043700097825A4600212046FEF7CAFE002800F028
:10438000E882031B04939DF82F300695CDF808A012
:1043900007934FF0000BB6E63B784AF0200A11E68F
:1043A000002940F0ED82A74A09921AF020012FD08F
:1043B000069A073222F00702516852F8080B06925B
:1043C0001AF0010F0BD050EA010208D08DF83130FD
:1043D00030238DF830304AF0020A022371E60223BE
:1043E0006FE6069B4FF000028DF82F2053F8042B48
:1043F000069301238DF840200193049310AC4EE7FF
:10440000002940F0B182904A09921AF02001CFD1E0
:104410001AF0100240F0FB811AF0400100F0F78121
:10442000069C54F8040B0694114680B2C8E7069B1C
:1044300053F8040B069330238DF8303078238DF831
:104440003130804B09934AF0020A0021022338E6FA
:10445000002940F08C821AF0200F40F017821AF0E9
:10446000100F40F038821AF0400F00F03482069BA3
:10447000039953F8042B0693118083E53B786C2B4A
:1044800003BF7B784AF0200A01374AF0100A99E509
:104490003B784AF0400A95E5002940F06B824AF0EB
:1044A000100A1AF0200F069B7FF421AF53F8040B7B
:1044B00006931AF0100F40F0AF811AF0400F00F091
:1044C000AB8140F3C0310B4600B219E73B784AF0AC
:1044D000800A77E53C4614F8013B2A2B00F0538212
:1044E000A3F13002092A27464FF0000B3FF66BADCF
:1044F00017F8013B0BEB8B0B02EB4B0BA3F13002DC
:10450000092AF5D95FE53B7801212B205AE5069B66
:1045100053F8042B0592002AFFF68EAE06933B78E3
:1045200050E53B784AF0010A4CE53B7800287FF4DF
:1045300049AD0121202045E5DDF808A0012B3FF41D
:10454000EFAE022B1AAC12D1099A00F00F0300094A
:10455000D35C04F8013D40EA0170090950EA010307
:10456000F3D11AAB1B1BCDF808A00493CBE500F0E8
:104570000703C00840EA4170C908303350EA01051A
:10458000224604F8013DF2D11AF0010FE9D0302B98
:10459000E7D03023023A04F8013C1AAB9B1ACDF85D
:1045A00008A004931446AEE5059B01981D1A002D42
:1045B0007FF7F2AD102DDFF894A025DD50461023D3
:1045C000A246044604E0103D102D09F1080918DD4B
:1045D00001321031072AC9E90043CDE90E21F2DD8D
:1045E0000DAA414630460DF16809FFF737FC002857
:1045F0007FF406AE103D102DDDE90E214FF01003C3
:10460000E6DC234654469A4601322944072ACDE97E
:104610000E21C9F800A0C9F8045000F37B81049B67
:10462000ABEB0305002D09F108097FF7BBAD102D99
:10463000DFF818A02CDD0B4651464FF0100BA246B8
:104640000C460AE058CF00086CCF000860CD000887
:10465000103D102D09F1080916DD01321033072A2B
:10466000C9E9004BCDE90E23F2DD0DAA41463046E3
:10467000FFF7F4FB00287FF4C3AD103D102DDDE9FA
:104680000E230DF16809E8DC1946234654469A4684
:1046900001322944072ACDE90E21C9F800A0C9F842
:1046A000045000F3C78009F108097BE50DAA4146D3
:1046B0003046FFF7D3FB00287FF4A2AD0F990DF130
:1046C00068097DE50DAA41463046FFF7C7FB002883
:1046D0003FF48AAD94E5102DDDE90E21DFF8C8A284
:1046E00025DD50461023A246044604E0103D102D5F
:1046F00009F1080918DD01321031072AC9E9004320
:10470000CDE90E21F2DD0DAA414630460DF16809D2
:10471000FFF7A4FB00287FF473AD103D102DDDE9F9
:104720000E214FF01003E6DC234654469A46013230
:104730002944072ACDE90E21C9F800A0C9F8045080
:1047400000F3D18009F10809FCE40DAA4146304686
:10475000FFF784FB00287FF453ADDDE90E210DF156
:10476000680903E50DAA41463046FFF777FB0028AC
:104770007FF446ADDDE90E210DF1680908E5102C46
:104780000E9BDFF824A225DD0A4651461025B246CD
:104790000E4604E0103C102C09F1080916DD013327
:1047A0001032072BC9E90065CDE90E32F2DD0DAA02
:1047B00041465046FFF752FB00287FF421AD103CE4
:1047C000102CDDE90E320DF16809E8DC11463246A5
:1047D0005646924601332144072BC9E900A4CDE98E
:1047E0000E317FF7F6AC0DAA41463046FFF736FB97
:1047F00000287FF405AD0F99EBE4BBF1000F7FF4C7
:1048000094ADCDF808A0CDF810B01AAC7BE4069AB0
:1048100052F8040B0692D3E5C1170B46002BBFF6E6
:1048200072AD2D2340428DF82F30079361EB41018B
:1048300001234CE40DAA41463046FFF70FFB002848
:104840007FF4DEACDDE90E210DF16809AAE41AACB3
:10485000CDF804A00A22002382460D46FBF7F4FCA3
:10486000303204F8012D0023504629460A22FBF776
:10487000EBFCBAF10A0F75F10003EBD21AABDDF8CD
:1048800004A0CDF808A01B1B04933CE4069B0398EE
:1048900053F8041B0693C217C1E90002FFF772BB6D
:1048A00020460695CDF808A0FFF76AFA9DF82F304C
:1048B000049007934FF0000B25E44021FEF778F9B0
:1048C000C8F80000C8F81000002866D04023C8F8D7
:1048D0001430FFF74DBB069B039953F8042B11606E
:1048E0000693FFF74FBB0DAA41463046FFF7B6FAD5
:1048F00000287FF485ACDDE90E210DF1680921E483
:104900009DF82F3007930BE5012BDDF808A07FF40D
:1049100018AE0AE50DAA41463046FFF79FFA002877
:104920007FF46EACDDE90E210DF1680934E45B46DD
:10493000062B28BF06231D4C049306950193AEE475
:104940000DAA41463046FFF789FA59E48DF82F0049
:1049500099E49DF82F30CDF810B00695CDF808A059
:1049600083460793FFF7CFBB8DF82F004BE58DF8FB
:104970002F0070E58DF82F0091E58DF82F00B1E440
:104980008DF82F000FE5069A7B78274652F8044BE6
:10499000069244EAE47BFFF715BB0C23CBF800300A
:1049A0004FF0FF33039334E450CD000880CF00086C
:1049B00000B50B4C25681446EE681A4685B00346D0
:1049C0000D464CB107490095CDE901143046064922
:1049D00000F052F801F024FD04490C46F3E700BF53
:1049E0000000002018D0000828D0000824D00008BB
:1049F00008B513460022FFF7DBFF00BF10B502FB2E
:104A000001F1FEF7D5F8044668B150F8042C22F005
:104A10000302043A242A18D8132A06D8024600238F
:104A2000C2E900339360204610BD00231B2AC0E971
:104A300000330FD9242AC0E9023311BF00F110025C
:104A4000036100F118024361E9E70021FBF7C4FDAF
:104A5000204610BD00F10802E1E700BF0CB400B52C
:104A600083B004AB53F8042B019300F0FDFD03B0B9
:104A70005DF804EB02B070470EB410B583B005AB1F
:104A8000064C53F8042B01930146206800F0ECFD1E
:104A900003B0BDE8104003B0704700BF0000002025
:104AA000F8B5244F0C460646FEF71CFCBA6855685C
:104AB000C4F57E630F3325F003052B4423F47F6395
:104AC00023F00F03A3F58054B4F5805F07DB0021CA
:104AD0003046FFF741F9BB682B44984204D030467A
:104AE000FEF702FC0020F8BD61423046FFF734F9C2
:104AF00001300DD0104ABB682D1B45F001055D60EB
:104B0000136830461B1B1360FEF7EEFB0120F8BD57
:104B100000213046FFF720F9BA68831A0F2BDEDD3B
:104B200043F001035360054B03491B68C01A08603A
:104B3000D5E700BF30040020C80A00203808002054
:104B4000002961D0F8B50C460646FEF7CBFB54F8B9
:104B5000042C7B4FA4F1080522F0010105EB010CA8
:104B6000B868DCF80430604523F0030300F08B8064
:104B7000D207CCF8043032D454F8082CAD1A1144C2
:104B8000AA6807F1080082426AD00CEB0304D4F84B
:104B900004E0EC68D4601EF0010FA26000F0978082
:104BA00041F001036B60CCF80010B1F5007F35D205
:104BB0007A68CB08480901210133814011437960AB
:104BC00007EBC30257F83310083AC5E9021247F859
:104BD0003350CD603046BDE8F840FEF785BB0CEBA6
:104BE00003025268D00710D4194407F10800DCF81A
:104BF0000830834273D0DCF80C20DA60936041F017
:104C000001036B606950D0E7704741F00103B1F5D3
:104C1000007F44F8043CCCF80010C9D3B1F5206FF4
:104C20004FEA512348D28B0903F1390003F13802CE
:104C3000C300F818FB580838984259D05A6822F037
:104C400003028A4202D99B689842F7D1D868C5E925
:104C500002308560DD603046BDE8F840FEF744BBB9
:104C60000CEB03025268D20763D40B44DCE9021256
:104C7000CA60916043F001026A603046EB50BDE8C3
:104C8000F840FEF731BB0B44D10707D454F8082C89
:104C9000AD1A1344D5E90212CA60916043F00102D3
:104CA0006A60284ABD6012689A4293D8264B304603
:104CB0001968FFF7F5FE8DE7142B0AD9542B1FD87E
:104CC0000B0B03F16F0003F16E02C300B1E719444F
:104CD0008DE703F15C0003F15B02C300A9E741F03B
:104CE0000103C7E90455C5E902006B60695071E72B
:104CF00079689210012404FA02F20A437A60A6E766
:104D0000B3F5AA7F06D8CB0B03F1780003F1770245
:104D1000C3008EE740F25452934206D88B0C03F145
:104D20007D0003F17C02C30083E74FF47E737E2293
:104D30007FE741F001036B60CCF800104AE700BF49
:104D4000300400203C080020C40A002042B110B505
:104D50000B491046144600F0D7FA18B9094810BD9F
:104D6000084870470749204600F0CEFA0028F5D0E1
:104D70000549204600F0C8FA0028EFD0002010BDF9
:104D80005CD0000858D0000824D00008014B93F8EC
:104D9000280170474008002041B110B50C4620465C
:104DA0000A4900F0B1FA18B9094810BD084870471F
:104DB0000749204600F0A8FA0028F5D0054920460A
:104DC00000F0A2FA0028EFD0002010BD5CD000084F
:104DD00058D0000824D0000810B4034CD4F8E440A4
:104DE000A44610BC604700BF4008002082B049B113
:104DF0005AB16BB113780B601278101E18BF0120E6
:104E000002B0704701A9002AF3D1104602B07047E2
:104E10006FF00100F4E700BF88420DD98B18834280
:104E20000AD900EB020CBAB1624613F801CD02F8C0
:104E300001CD9942F9D170470F2A0ED8034602F1ED
:104E4000FF3C4AB10CF1010C013B8C4411F8012BE1
:104E500003F8012F6145F9D1704740EA01039B0730
:104E600050D1A2F1100370B501F1200C23F00F0511
:104E700001F1100E00F11004AC441B095EF8105C47
:104E800044F8105C5EF80C5C44F80C5C5EF8085C5E
:104E900044F8085C5EF8045C44F8045C0EF1100E03
:104EA000E64504F11004E9D1013312F00C0F01EBD7
:104EB000031102F00F0400EB031327D0043C24F08D
:104EC00003064FEA940C1E441C1F8E465EF8045BDA
:104ED00044F8045FB442F9D10CF1010402F003027A
:104EE00003EB840301EB840102F1FF3C4AB10CF1B6
:104EF000010C013B8C4411F8012B03F8012F614593
:104F0000F9D170BD02F1FF3C03469BE72246EBE777
:104F10002DE9F84F1746002900F0988007F10B059E
:104F200080460C46FEF7DEF9162D5DD810252A4680
:104F3000AF425ED854F8041C21F003069642A4F157
:104F4000080962DABC4BD3F808C009EB06008445B7
:104F500000F09780D0F804C02CF0010303445B6894
:104F6000DB0768D42CF0030C06EB0C03934247DA02
:104F7000CB0710D454F8083CA9EB030ADAF8043044
:104F800023F003018C44B444944580F211817318DA
:104F9000934280F2E88039464046FDF709FE074615
:104FA000E0B154F8043C23F001034B44A0F10802A3
:104FB000934200F0D280321F242A00F2F580132A97
:104FC00000F2AC80034622461168196051685960AE
:104FD00092689A6021464046FFF7B2FD4046FEF7D0
:104FE00083F93846BDE8F88F25F00705002D2A46DD
:104FF0009EDA0C23C8F8003000273846BDE8F88F49
:105000001E46D0E90223D3609A60731B0F2B22D86F
:10501000D9F8043003F0010333434E44C9F8043097
:10502000736843F00103736040462746FEF75CF95E
:105030003846BDE8F88FC907ADD454F8083CA9EB51
:10504000030ADAF8041021F00301A0E7BDE8F84FE5
:105050001146FDF7ADBDD9F8041001F00101294357
:10506000C9F8041009EB05014E4443F001034B60FD
:10507000736843F00103083173604046FFF760FD39
:10508000D2E7DCF8040020F0030B06EB0B0C05F173
:10509000100084454DDAC9073FF57DAF54F8081C70
:1050A000A9EB010ADAF8041021F003018B44B344A0
:1050B00058453FF76CAF5746DAF80C1057F8080F11
:1050C000321F242AC160886000F2DB80132A40F27C
:1050D000D6802168CAF808106168CAF80C101B2A2B
:1050E00000F2DF8008340AF1100221681160616863
:1050F0005160A16891600AEB0501ABEB050242F03B
:10510000010299604A60DAF8043003F001031D439C
:105110004046CAF80450FEF7E7F86EE723680360DC
:10512000636843601B2A68D804F1080200F1080391
:105130004AE709EB05029A60ACEB050343F0010373
:10514000536054F8043C03F001031D43404644F807
:10515000045CFEF7C9F827464FE750F8043C23F0FB
:1051600003031E4451E75746DAF80C1057F8080FAE
:10517000321F242AC16088604CD8132A48D921687C
:10518000CAF808106168CAF80C101B2A56D80834EF
:105190000AF110021E462368136063685360A36817
:1051A0009360D1463C4630E72146FFF735FE11E7D4
:1051B000D0E902135746CB60996057F8081FDAF818
:1051C0000C30CB60321F242A99602DD8132A29D99C
:1051D0002368CAF808306368CAF80C301B2A42D822
:1051E00008340AF1100322681A6062685A60A268E3
:1051F0009A606646D1463C4607E7A3688360E36849
:10520000C360242A26D004F1100200F11003DBE66B
:105210003A46BFE7214638461E46D146FFF7FCFD19
:105220003C46F2E63B46DEE7214638466646D14636
:10523000FFF7F2FD3C46E8E630040020A168CAF81A
:105240001010E168CAF81410242A20D010340AF192
:1052500018029FE7236903616169416104F1180243
:1052600000F11803B0E6A368CAF81030E368CAF882
:105270001430242A21D010340AF11803B3E73A4637
:1052800033E721463846FFF7C7FD164B33E722695F
:10529000CAF818206269CAF81C2018340AF12002E2
:1052A00078E7A168CAF81010E168CAF81410242A37
:1052B0000DD010340AF1180217E72369CAF8183024
:1052C0006369CAF81C3018340AF120038BE722699D
:1052D000CAF818206269CAF81C2018340AF12002A2
:1052E00003E700BF300400200000000000000000C1
:1052F00000000000000000000000000000000000AE
:10530000A2EB0300704700BF02780B78012A28BF88
:105310009A42F5D16DE9044540EA0104CDE90267FE
:105320006FF0000C4FEA447212B380EA010414F0EB
:10533000070F6AD100F0070420F0070004F003050E
:1053400021F007014FEAC505F0E8042314F0040F2B
:10535000F1E804670CFA05F462EA040266EA04065E
:105360000AD063EA0403624667EA0407664603E07C
:10537000F0E80423F1E8046782FA4CF582EA0604B7
:10538000A4FA8CF46CBB83FA4CF583EA0705A5FA02
:105390008CF595B950E9022351E9026782FA4CF580
:1053A00082EA0604A4FA8CF483FA4CF583EA070532
:1053B000A5FA8CF52543DBD09CB92DBAB5FA85F456
:1053C00024F0070427FA04F1DDE9026723FA04F365
:1053D00003F0FF0001F0FF01FDE80445A0EB010030
:1053E000704724BAB4FA84F424F0070426FA04F1CE
:1053F000DDE9026722FA04F202F0FF0001F0FF018A
:10540000FDE80445A0EB0100704714F0030F3CD108
:1054100010F0030428D150F8082B51F8083B82FA09
:105420004CF582EA0305A5FA8CF55DB950F8042C19
:1054300051F8043C82FA4CF582EA0305A5FA8CF592
:10544000002DE8D02DBAB5FA85F424F0070423FA2C
:1054500004F122FA04F202F0FF0001F0FF01FDE87E
:105460000445A0EB010070474FEAC40420F003009C
:1054700050F8082B21F0030151F8083B0CFA04F412
:1054800062EA040263EA0403C9E710F003041AD0D5
:10549000A1EB040120F00300E40750F8042B06D030
:1054A0000FD28B785FFAA2F4E41A06D12BB1CB7835
:1054B0005FFAB2F4E41A00D11BB920465DF8104B34
:1054C000704701F1040150F8042BCC0721F00301CF
:1054D00051F8043B48D824D222F07F4482FA4CF59C
:1054E00094EA1325A5FA8CF50AD165B951F8043B65
:1054F00084EA0204B4EB036F0ED150F8042BEBE7FF
:105500004FEA132355E035F07F454DD10878FDE88B
:105510000445C0F1000070474FEA126203F0FF0338
:1055200047E002EA1C4482FA4CF594EA1345A5FAD6
:105530008CF50AD165B951F8043B84EA0204B4EB56
:10554000034F0CD150F8042BEBE74FEA134330E044
:1055500015EA1C4528D10B884FEA124229E04FEA90
:10556000124203EA1C4324E002F0FF0482FA4CF5E5
:1055700094EA1365A5FA8CF50AD165B951F8043B94
:1055800084EA0204B4EB032F09D150F8042BEBE7B3
:105590004FEA13630DE015F0FF0F05D10B684FEADA
:1055A000122223F07F4304E04FF00000FDE80445A1
:1055B000704712BA1BBA82FA4CF482EA0304A4FAC6
:1055C0008CF5B5FA85F402FA04F203FA04F34FEA13
:1055D0001260FDE80445A0EB136070472DE9F84F19
:1055E0004B6E9C0490462DD59368126843B38B464E
:1055F000064602F1080959E9025A5FEA9A0715D0EE
:10560000043D002401E0A7420ED055F8041F5A467D
:10561000304601F03BF9431C04F10104F3D10023AF
:10562000C8E90133BDE8F88FD8F808302AF0030A3A
:10563000A3EB0A03C8F8083009F10809002BDAD1F6
:105640000020ECE701F054F90023C8E90133BDE87C
:10565000F88F00BF10B494680CB110BCBEE72046B0
:10566000546010BC704700BF2DE9F04FABB01C4632
:10567000884617460693834618B1836B002B00F0CB
:105680002582B8F90C1088048AB20AD4D8F864309C
:1056900041F4005223F40053A8F80C20C8F86430F9
:1056A00092B2130740F1A480D8F81030002B00F01C
:1056B0009F8002F01A020A2A00F0A8801AAB0D930C
:1056C0000023CDE90E3309930DF1680905933B786A
:1056D000002B00F00D813C4604E014F8013F002B44
:1056E00000F0E880252BF8D1E51B40F0E580237819
:1056F000002B00F0FD804FF0000200218DF82F20DC
:10570000637804914FF0FF32671C084602928A4684
:105710000137A3F12002582A00F2F780DFE812F0E7
:105720003302F500F5002F02F500F500F500F50055
:10573000F500F500E5012B02F500F001F401F5009C
:1057400027025900590059005900590059005900C1
:1057500059005900F500F500F500F500F500F500D9
:10576000F500F500F500F5000E02F500F500F50076
:10577000F500F500F500F500F500F500F5009400E2
:10578000F500F500F500F500F5008400F500F500E2
:105790004802F500F500F500F500F500F500F5000C
:1057A000F500F500F5003A02A701F500F500F50057
:1057B0008902A701F500F5007F02F5006902960055
:1057C000C902C502F500A402F5008600F500F50047
:1057D0008D02A3F13002002417F8013B04EB84048E
:1057E00002EB4404A3F13002092AF5D9049490E7AE
:1057F0004146584600F0AAFD002840F03985B8F827
:105800000C2002F01A020A2A7FF458AFB8F90E30C1
:10581000002BFFF653AF23463A46414658462BB07D
:10582000BDE8F04F00F044BD4AF0100A1AF0200124
:1058300000F00F81069B073323F00703596853F8E4
:10584000080B069301230EE04AF0100A1AF020011B
:1058500000F0F280069B073323F00703596853F8E2
:10586000080B069300234FF000028DF82F20002232
:105870000792029A541C00F02F822AF080040194AF
:1058800050EA010440F02682002A40F09584002B63
:1058900040F00E841AF00103039340F03E841AACEA
:1058A000DDE902639E42B8BF1E46079B002B3ED037
:1058B00001363CE0E51B1BD00E9B0F9A01332A44B6
:1058C000072BC9E900750F920E9305DC09F1080951
:1058D000059B2B4405930AE7002A00F0D1830DAA0B
:1058E00041465846FFF77AFE30B90DF16809EFE7F7
:1058F0000F9B002B40F08584B8F80C305B0600F15C
:10590000B78405982BB0BDE8F08F002940F075846E
:10591000002BEDD08DF8403001264FF000038DF8BC
:105920002F30039610AC0023CDF804A00293019B06
:1059300013F002030793019B18BF023613F0840390
:10594000089304D1049B9D1B002D00F3DB82DDE94D
:105950000E1001F1010C9DF82F3093B101300DF1C3
:105960002F030121BCF1070FCDE90EC0C9F80030AB
:10597000C9F8041000F3A682614609F108090CF188
:10598000010C079BEBB10CAB0230C9F80030BCF145
:10599000070F4FF00203CDE90EC0C9F8043040F301
:1059A000AB82002800F066830DAA41465846FFF7F7
:1059B00015FE0028A0D1DDE90E100DF1680901F1F6
:1059C000010C089B802B00F0C881DDE902329D1A92
:1059D000002D00F31C82039BC9F800401844BCF161
:1059E000070FCDE90EC0C9F8043040F3B381002899
:1059F00000F0D2820DAA41465846FFF7EFFD00287D
:105A00007FF47AAF0F980DF16809019B5A0704D50E
:105A1000049B9C1B002C00F3C982DDE90423B242E5
:105A2000ACBF9B189B190593002840F036820023D9
:105A30000E930DF168094AE61AF0100349D11AF0E5
:105A4000400146D0069A52F8040B0692194680B2DD
:105A500009E71AF0100342D11AF040013FD0069A2C
:105A600052F8040B0692194680B20123FBE6002986
:105A700040F0E5831AF0200F069B68D0073323F02F
:105A800007031A465B6852F8080B06921946002B6A
:105A9000C0F20483029B013300F08A839DF82F300B
:105AA000079350EA01032AF0800A00F054830A2881
:105AB00071F1000380F01283303001238DF867000C
:105AC000CDF804A003930DF16704E9E600F06AFE47
:105AD000D7E5069B53F8040B06930B46C3E6069BDB
:105AE00053F8040B06930123BDE6069B53F8042BE1
:105AF0000492002A80F20D83049A06935242049283
:105B00003B784AF0040A03E63C4614F8013B2A2B92
:105B100000F0B383A3F13002092A274698BF00247E
:105B200000F2938317F8013B04EB840402EB440476
:105B3000A3F13002092AF5D90294EAE5002940F0E0
:105B400088834AF0100A1AF0200F069B96D153F86A
:105B5000040B06931AF0100F40F09B821AF0400FCE
:105B600000F0978240F3C0310B4600B28FE73B78DC
:105B70004AF0800ACCE53B7801212B20C8E53B7830
:105B80004AF0010AC4E53B7800287FF4C1AD012149
:105B90002020BDE5069B4FF000028DF82F20012646
:105BA00053F8042B8DF840200693039610ACBAE608
:105BB000002940F05183BD4A09921AF0200144D0D7
:105BC000069A073222F00702516852F8080B069233
:105BD0001AF0010F0BD050EA010208D08DF83130D5
:105BE00030238DF830304AF0020A02233BE60223CC
:105BF00039E6002940F026831AF0200F40F09A82FF
:105C00001AF0100F40F0CC821AF0400F00F0C8825A
:105C1000069B059953F8042B0693118057E53B78B2
:105C20006C2B03BF7B784AF0200A01374AF0100A38
:105C30006EE53B784AF0400A6AE5002940F0FC82B4
:105C40009B4A09921AF02001BAD11AF0100240F0D2
:105C50001B821AF0400100F01782069C54F8040BD6
:105C60000694114680B2B3E7069D55F8044B4FF0F9
:105C700000038DF82F30002C00F0A482029B5E1CE4
:105C800000F072821A4600212046FDF741FA0028F2
:105C900000F0C282031B03939DF82F30079300236B
:105CA0000695CDF804A00293FAE53B784AF0200A65
:105CB0002EE5069B53F8040B069330238DF8303005
:105CC00078238DF831307A4B09934AF0020A00218B
:105CD0000223C8E5DDF804A0012B3FF4E8AE022B57
:105CE0001AAC12D1099A00F00F030009D35C04F832
:105CF000013D40EA0170090950EA0103F3D11AABF2
:105D00001B1BCDF804A00393CAE500F00703C008ED
:105D100040EA4170C908303350EA0105224604F8D0
:105D2000013DF2D11AF0010FE9D0302BE7D030233A
:105D3000023A04F8013C1AAB9B1ACDF804A0039375
:105D40001446ADE503981A9401231B900F900E930F
:105D50000DF1680909F1080957E6049B9D1B002D08
:105D60007FF733AE102D40F37F82DFF848A1524613
:105D70001023A246144607E001F1020E09F10809BA
:105D80001146103D102D1DDD4A1C1030072AC9E9AF
:105D90000043CDE90E20EFDD0DAA002800F08C8035
:105DA000414658460DF16809FFF718FC00287FF4BA
:105DB000A3ADDDE90E10103D102D01F1010E4FF0E5
:105DC0001003E1DC234654469A462844BEF1070FEF
:105DD000CDE90EE0C9F800A0C9F8045040F3A48151
:105DE000002800F0F8810DAA41465846FFF7F6FB5F
:105DF00000287FF481ADDDE90232DDE90E109D1A45
:105E0000002D01F1010C0DF168097FF7E4AD102DB3
:105E1000DFF8A0A02BDD52461023A246144607E06F
:105E200001F1020C09F108091146103D102D1BDD8E
:105E30004A1C1030072AC9E90043CDE90E20EFDDE6
:105E40000DAA414618B358460DF16809FFF7C6FB85
:105E500000287FF451ADDDE90E10103D102D01F149
:105E6000010C4FF01003E3DC234654469A462844C5
:105E7000BCF1070FCDE90EC0C9F800A0C9F8045065
:105E800000F3E38009F108090CF1010CA3E54FF0E0
:105E9000010C01460DF16809C7E70DAA41465846B5
:105EA000FFF79CFB00283FF4C2AD25E56CCF00084E
:105EB00058CF000880CD00084FF0010E01460DF1CB
:105EC00068095EE7002800F0D2800DAA41465846D6
:105ED000FFF784FB00287FF40FADDDE90E100DF114
:105EE000680901F1010C4CE502200CAB1B901A93E0
:105EF0004FF0010C0DF16809614609F1080901F143
:105F0000010C5EE5102D40F39181DFF804A3DDE97B
:105F10000EC052461023A2466146144607E001F126
:105F2000020C09F108091146103D102D1BDD4A1C19
:105F30001030072AC9E90043CDE90E20EFDD0DAA94
:105F400020B3414658460DF16809FFF747FB00288A
:105F50007FF4D2ACDDE90E10103D102D01F1010CE3
:105F60004FF01003E3DC2346614654469A4628442A
:105F70000729CDE90E10C9F800A0C9F8045000F3B4
:105F80009C8009F1080901F1010CE4E401464FF09D
:105F9000010C0DF16809C7E7019B0E9059074CD51C
:105FA000049B9C1B002C48DD0DF16809102C40F36C
:105FB0005681DFF85CA20E9A53461025B2461E4663
:105FC00006E0911C09F108091A46103C102C19DD55
:105FD000531C1030072BC9E90065CDE90E30F0DD08
:105FE0000DAA28B341465846FFF7F8FA00287FF477
:105FF00083ACDDE90E20103C102C02F101010DF103
:106000006809E5DC334656469A4620440729C9E923
:1060100000A4CDE90E107FF700AD70B10DAA414686
:106020005846FFF7DBFA00287FF466AC0F98F4E4DB
:10603000012102460DF16809C7E7DDE90423B242F8
:10604000ACBF9B189B190593F1E400283FF47AAE8E
:106050000DAA41465846FFF7C1FA00287FF44CAC20
:106060000E9B0F9803F1010C0DF16809B3E4079B37
:10607000002B69D14FF0010C01460DF16809A0E435
:106080000E920DF1680923E4069A52F8040B069269
:106090009EE5C1170B46002BBFF6FCAC2D234042FA
:1060A0008DF82F30079361EB41010123FFF7E1BB2E
:1060B000029B03931AACFFF7F3BB002862D00DAA32
:1060C00041465846FFF78AFA00287FF415ACDDE90F
:1060D0000E100DF1680901F1010C3CE41AAC0A2222
:1060E000002306460D46FAF7AFF8303204F8012DCA
:1060F0000023304629460A22FAF7A6F80A2E75F13F
:106100000003ECD21AAB1B1BCDF804A00393FFF7DE
:10611000C7BB06933B78FFF7FBBA30238DF8673097
:106120000DF16704FFF7BCBB09F108090EF1010C82
:1061300071464AE4DDE9050353F8041B0693C217D0
:10614000C1E90002FFF7C3BA02200CAB1B901A93FF
:106150000DF16809D1E6029B002B7FF4ADACCDF8C0
:1061600004A00393FFF79BBB20460695CDF804A03F
:10617000FDF706FE9DF82F3007930023039002934E
:10618000FFF78EBB9DF82F3063B301239C461B9312
:106190000DF12F031A930DF168096046FFF7ECBB70
:1061A000069B059953F8042B11600693FFF78FBAED
:1061B0009DF82F3007937AE4012BDDF804A07FF4DB
:1061C0008EAD79E4029E134C0695062E28BF062656
:1061D0000396FFF7A8BB4FF0010C01460DF16809CB
:1061E000FFF7F3BB079B002B7FF47EAE01464FF019
:1061F000010C0DF16809FFF7E8BB8DF82F00FFF7E0
:1062000087BB0DAA41465846FFF7E8F9FFF774BB74
:1062100070CD000880CF0008029B03939DF82F30BB
:106220000695CDE901A00793FFF73ABB0E990F98A9
:10623000DFF85CA001319AE68DF82F0000E58DF8BB
:106240002F0017E48DF82F00D6E400220292FFF70A
:1062500060BA8DF82F0074E48DF82F00ABE40E992E
:10626000DFF82CA00131D0E6DFF828A0E646ACE547
:106270004FF0FF330593FFF744BB069A7B78274620
:1062800052F8044B069244EAE4740294FFF740BAD1
:1062900070CD000880CD000810B4044C844613462D
:1062A000206810BC0A466146FFF7DEB900000020F6
:1062B00070B50C468989ADF58D6D21F00201ADF800
:1062C0000C10616E1991E189ADF80E10E16907912A
:1062D000616A09911AA9009104914FF480610291B9
:1062E00005910021069169460646FFF7BDF9051E96
:1062F00007DB6946304600F02BF9002818BF4FF045
:10630000FF35BDF80C305B0603D5A38943F040038D
:10631000A38128460DF58D6D70BD00BF10B4034CF0
:10632000D4F8E040A44610BC604700BF40080020FD
:1063300049B1FF2A02D80A70012070478A230360FE
:106340004FF0FF3070470846704700BF38B5334BF9
:106350001B6805460C460BB19A6B12B3B4F90C30AE
:1063600018079AB225D5216900292DD012F0010015
:1063700007D00020A06060694042A06139B10020D0
:1063800038BD950758BF6069A0600029F7D1120693
:1063900058BF0846F4D543F04003A3814FF0FF30C7
:1063A00038BD184600F0FEF9B4F90C3018079AB25F
:1063B000D9D4D1062AD5520714D4216943F0080351
:1063C000A3819AB20029D1D102F42070B0F5007FE8
:1063D000CCD02146284600F043FCB4F90C302169AA
:1063E0009AB2C3E7216B51B104F14002914204D04B
:1063F0002846FEF7A5FBB4F90C3000222263216980
:106400000022C4E9001223F02403D7E7092243F055
:1064100040032A604FF0FF30A38138BD0000002008
:1064200008B5062000F058FD012002F0D9F800BFA1
:10643000B1F90C20F8B50C461107074642D4636841
:1064400042F40062002BA28159DDA56A002D54D0D0
:1064500000233E683B6093B212F4805253D1E1694D
:1064600001233846A847421C63D0A389A56A5B076D
:1064700005D56368C01A236B0BB1E36BC01AE169E1
:10648000024600233846A847411C3ED13B68002BFA
:106490003BD01D2B01D0162B52D1A389226922603B
:1064A00023F4006300216160A381216B3E6021B36E
:1064B00004F14003994202D03846FEF741FB002028
:1064C0002063F8BD2669C6B193B2256826609A0795
:1064D0000CBF63690023AD1BA3600CE0D4F824C09B
:1064E000E1692B4632463846E047B0F1000CA5EB97
:1064F0000C05664416DD002DF0DC0020F8BDE36BD2
:10650000002BA2DCF9E7206DB1E7B4F90C30226969
:10651000226023F40063A3810022DB046260C4D5FF
:106520002065C2E7A38943F040034FF0FF30A38109
:10653000F8BD3B68002B98D01D2B06D0162B04D03D
:10654000A38943F04003A381F8BD3E60D5E700BFB7
:1065500038B50D46044608B1836B1BB1B5F90C0084
:1065600030B938BD00F01EF9B5F90C000028F8D09C
:1065700029462046BDE83840FFF75ABF38B5B8B1C4
:106580000F4B1D6804460DB1AB6B4BB1B4F90C0059
:1065900000B938BD21462846BDE83840FFF748BF5E
:1065A000284600F0FFF8B4F90C000028F1D0F1E71C
:1065B000044B05491868BDE8384000F02DBB00BF0A
:1065C0000000002000CC0008516500080020704742
:1065D000014900F021BB00BFF172000800207047A4
:1065E0002DE9F84F2D4A4668C26300240323C0E911
:1065F000B843074600F53B720423C0F8E822214661
:10660000C6E902430822C6E90044C6E904447466A8
:10661000B46106F15C00F9F7DFFFDFF884B0BD6814
:10662000DFF880A0DFF88090DFF88080204BC6F88C
:1066300024A0C6E9076BC6F82890C6F82C8008226B
:10664000EB60C5E90044C5E904446C66AC60AC612C
:10665000214605F15C00F9F7BFFFC5E9075BC5E915
:1066600009A9C5F82C80FD68124BEB60C5E9004410
:10667000C5E904446C66AC60AC612146082205F1B2
:106680005C00F9F7A9FF0123C5E9075BC5E90A9892
:10669000C5F824A0BB63BDE8F88F00BFD165000832
:1066A0005970000881700008C1700008E17000088E
:1066B000090001001200020070B568224D1E02FBA5
:1066C00005F50E4605F17401FCF772FA044640B177
:1066D00000210C30C4E90016A06005F16802F9F74A
:1066E0007BFF204670BD00BF274B2DE9F0411E689F
:1066F000B36B07465BB306F538764FF00408D6E96E
:106700000134013B04D51EE05A1C04F168041AD080
:10671000B4F90C50013B002DF6D11C4B6566C4E961
:106720000055C4E90253C4E90455A561082229466D
:1067300004F15C00F9F750FFC4E90C55C4E91155A8
:106740002046BDE8F08135682DB12E46D7E73046AA
:10675000FFF746FFCFE74FF4D6713846FCF728FA2B
:10676000044668B10560C0F804800C302946A0607A
:1067700025464FF4D072F9F72FFF34602E46BEE75E
:106780000C2330603B60DBE700CC00080100FFFF1A
:10679000024B0349186800F03FBA00BF00CC000864
:1067A000F1720008836B03B1704719E7704700BFAF
:1067B000704700BF704700BF704700BF024B0349DE
:1067C000186800F009BA00BF00000020CD6500087D
:1067D000024B0349186800F0FFB900BF0000002019
:1067E000DD6500082DE9F04383B00746884614466E
:1067F000FEF7CCFA012803D108F1FF33FE2B37D97D
:10680000424604F15C0301A9384600F0D1FC421C69
:10681000064633D038B39DF804C00DF105090025B4
:1068200009E023685A1C226083F800C00135B54294
:1068300019D219F801CBA368013B002BA360F0DA51
:10684000D4F818E0734561462246384602DBBCF1B5
:106850000A0FE6D100F048FC431CE7D1064630465B
:1068600003B0BDE8F0834646304603B0BDE8F08390
:106870005FFA88FC8DF804C00646CEE7A38930464F
:1068800043F04003A38103B0BDE8F083B2F90C30BC
:1068900013F4005F0AD110B4546E43F4005344F46F
:1068A00000545466938110BCFFF79CBFFFF79ABF5A
:1068B0000E4B70B51E6805460C460EB1B36B8BB11E
:1068C000B4F90C309A0406D4626E43F4005342F4D7
:1068D0000052A3816266224629463046BDE87040D8
:1068E000FFF780BF3046FFF75DFFE9E700000020BB
:1068F0009368002B00F081802DE9F04FB1F90C3046
:106900000C461907804683B0174698B223D52369F1
:106910000BB310F002033D682BD04FF0000ADFF8F4
:10692000B4B256465E453346524628BF5B464046A3
:10693000002E4FD0E169D4F824C0E047002852DD92
:10694000BB681B1A8244361ABB60002BEAD10020B8
:1069500003B0BDE8F08F21464046FFF7F7FC002862
:1069600040F03481B4F90C303D6898B210F0020365
:10697000D3D110F0010942D14E463EB38205D4F87E
:1069800008B040F18180B3455A4600F2B18010F45E
:10699000906F40F0BE80206801924946FEF73CFAB5
:1069A000A3682168019AA3EB0B030A44B246A360D3
:1069B00022600026B868A0EB0A00D144B860002825
:1069C000C5D0B4F90C0080B2002ED7D1D5E900961D
:1069D0000835D2E7D5E900A60835A3E721464046A9
:1069E000FFF7B6FD80B3B4F90C3043F040034FF02D
:1069F000FF30A38103B0BDE8F08F002070471E4632
:106A0000AA46994618461D4656B388B34A46D4E965
:106A100004132068B24228BF3246884205D9A168D3
:106A200003EB010B5A4500F3A780934264DCE16954
:106A3000D4F824C02A464046E047B0F1000BD2DD2E
:106A4000B9EB0B09CAD00120BB68A3EB0B035D4473
:106A5000A6EB0B06BB60002B3FF479AF002ED4D120
:106A60000AF1080353E902569A460833002EF9D07A
:106A700032460A212846FCF74BFB002800F09D8097
:106A80000130A0EB0509C1E720682369984217D8B7
:106A90006369B34214D86FF00042B24228BF324655
:106AA000E16992FBF3F2D4F824C002FB03F3404601
:106AB0004A46E047B0F1000A95DDA6EB0A0679E701
:106AC000B345DA4628BFB24652464946FEF7A4F916
:106AD000A3682268A3EB0A035244A3602260002B40
:106AE000EBD121464046FFF733FD0028E5D07AE799
:106AF0002068B34632464FE729460192FEF78CF9EB
:106B0000019AA3689B1AA3602368134423609346E9
:106B100096E723682169A3EB010B636903EB430A42
:106B20000AEBDA7A0BF101034FEA6A0A3344534560
:106B3000524684BF9A46524643052CD511464046DC
:106B4000FCF736F800283BD05A4621690190FCF743
:106B50002FFBA289019B22F4906242F08002A28165
:106B600003EB0B002361AAEB0B03C4F814A0A36092
:106B70002060B34632460FE729465A46FEF74CF9E5
:106B800023685B44236021464046FFF7E1FC002870
:106B90003FF456AF27E74046FEF7BAF90346002810
:106BA000DED121694046FDF7CBFFB4F90C300C2251
:106BB00023F08003C8F8002017E7721C914626E7EF
:106BC0000C22B4F90C30C8F800200EE74FF0FF306B
:106BD000BEE600BF00FCFF7F2DE9F041884600F5CE
:106BE00038770026D7E90154013D0FD4A389012B42
:106BF00005F1FF3506D9B4F90E300133204601D036
:106C0000C04706436B1C04F16804EFD13F68002FB6
:106C1000E8D13046BDE8F0812DE9F84307468846C3
:106C200000F538764FF00009D6E90154013D11D442
:106C3000A389012B05F1FF3508D9B4F90E300133D2
:106C4000214603D03846C04749EA00096B1C04F1CD
:106C50006804EDD13668002EE6D14846BDE8F883D9
:106C60002DE9F0418B890C46990796B008D504F1BF
:106C700043030122C4E90432236016B0BDE8F08169
:106C8000B4F90E100029064627DB6A4600F068FBBF
:106C9000002821DB019D05F47045A5F50055B5FAE6
:106CA00085F54FF480686D094FF400674146304622
:106CB000FBF77EFFB4F90C30F0B1204AF26343F0E9
:106CC0008003C4F81480A3812060206135BB3B435E
:106CD000A38116B0BDE8F081A38913F0800519D017
:106CE0004FF0400841463046FBF762FF0025B4F9FB
:106CF0000C302F460028E0D19A05BED423F00303C0
:106D000004F1430243F002030121C4E90421A381F9
:106D10002260B2E74FF480682F46C7E7B4F90E103F
:106D2000304600F033FB10B9B4F90C30CFE7A3893B
:106D300023F0030343F001031BB2C8E7D165000849
:106D400070B50C46B1F90E10002996B015461E46D6
:106D500014DB6A4600F004FB00280FDB019A02F402
:106D60007042A2F50052B2FA82F24FF480635209E7
:106D70004FF4006032602B6016B070BDB4F90C1097
:106D8000002311F08000336004D0402218462A60AE
:106D900016B070BD4FF480632B6016B070BD00BF9D
:106DA00038B5D0F8DC420CB1002038BD8021054652
:106DB000FBF7FEFE0246C5F8DC0230B1031F7C3251
:106DC00043F8044F9342FBD1EEE74FF0FF3038BD5C
:106DD0001F29F8B5054609D8D0F8DC620C461746DD
:106DE0004EB156F8240046F82470F8BD162303600F
:106DF0004FF0FF30F8BD8021FBF7DAFE0646C5F8FC
:106E0000DC0240B1031F00F17C05002143F8041FA0
:106E10009D42FBD1E5E74FF0FF30F8BD1F2938B5A3
:106E2000054621D8D0F8DC220C466AB152F8213050
:106E300053B1012B16D0591C10D00025204642F822
:106E400024509847284638BD284600F003F92246CA
:106E500001462846BDE8384000F0E6B81623036036
:106E6000012038BD002038BD162303604FF0FF30ED
:106E700038BD00BF1F292CD8D0F8DC2238B50C460D
:106E8000054682B152F8243002EB84024BB1591C02
:106E90001AD0012B16D000252046156098472846A9
:106EA00038BD012038BD8021FBF782FE0246C5F8BF
:106EB000DC0258B1031F00217C3043F8041F9842C4
:106EC000FBD1DFE7032038BD022038BD4FF0FF3093
:106ED00038BD4FF0FF30704738B5154B1F281D687F
:106EE00020D8D5F8DC22044662B152F820304BB1EC
:106EF000012B15D0591C0FD0002542F8205098477F
:106F0000284638BD284600F0A5F822460146284606
:106F1000BDE8384000F088B816232B60012038BD4A
:106F2000002038BD16232B604FF0FF3038BD00BF66
:106F300000000020134B1F2870B51E6809D80D46AD
:106F4000D6F8DC12044649B151F8240041F8245027
:106F500070BD162333604FF0FF3070BD8021304686
:106F6000FBF726FE0146C6F8DC0240B1031F00F124
:106F70007C0C002243F8042F6345FBD1E4E74FF07B
:106F8000FF3070BD0000002038B50C4B1D68D5F8EF
:106F9000DC420CB1002038BD80212846FBF708FEFA
:106FA000C5F8DC0238B1031F00F17C0243F8044F3E
:106FB0009342FBD1EEE74FF0FF3038BD00000020D8
:106FC00038B5184B1F281D6828D8D5F8DC22044690
:106FD00082B152F8243002EB84024BB1591C1BD011
:106FE000012B17D00025204615609847284638BD4C
:106FF000012038BD80212846FBF7DAFD0246C5F89E
:10700000DC0258B1031F00217C3043F8041F834287
:10701000FBD1DEE7032038BD022038BD4FF0FF3042
:1070200038BD00BF0000002070B50C46084D034677
:107030000026204611461C462E6001F0C9FA431C6A
:1070400000D070BD2B68002BFBD0236070BD00BF4B
:10705000F80A002001F0BABA10B50C46B1F90E10CA
:1070600000F0BCF9002803DB236D0344236510BD49
:10707000A38923F48053A38110BD00BF0020704773
:107080002DE9F0410C46B1F90C101F46CB05054621
:1070900016460BD421F48051A1813B46B4F90E1061
:1070A00032462846BDE8F04100F0C8B8B4F90E10E9
:1070B0000223002200F07CF9B4F90C10EAE700BFCB
:1070C00010B50C46B1F90E1000F072F9A389421CFC
:1070D0000EBF23F4805343F480532065A38110BD79
:1070E000B1F90E1000F0C0B8F8B50D4614460646CA
:1070F00010B1836B002B43D0B4F90C20A369A360BB
:10710000170790B21BD52369CBB1EDB281042F468E
:1071100022D522686169D31A994229DD0133A16819
:107120000139A160511C2160157062699A422AD010
:10713000A389DB0701D50A2D25D03846F8BD2146A5
:107140003046FFF703F920BBB4F90C20236990B255
:10715000EDB281042F46DCD442F40052A281626E6B
:10716000616922F4005262662268D31A9942D5DC22
:1071700021463046FFF7ECF958B922680123CEE7E3
:10718000FFF710FBB8E721463046FFF7E1F900288A
:10719000D3D04FF0FF37D0E710B4044C03460A4673
:1071A000206810BC1946FFF79FBF00BF00000020F9
:1071B00070B5054684B01C4639B10B4ED6F8E06078
:1071C000B047431C09D004B070BD0A460649D1F847
:1071D000E06001A9B047431CF5D100228A23226058
:1071E0002B6004B070BD00BF4008002070B5114B8B
:1071F00084B01D6814460B46014650B10E481A462D
:10720000D0F8E06023462846B047431C0BD004B0BA
:1072100070BD094A2346D2F8E06001A9024628461B
:10722000B047431CF3D100228A2322602B6004B0B4
:1072300070BD00BF000000204008002038B50C469B
:10724000084D8446114620461A4600232B606446AA
:1072500001F0DCF9431C00D038BD2B68002BFBD0BB
:10726000236038BDF80A002038B5074D00220446D7
:1072700008462A6001F0D8F9431C00D038BD2B68BD
:10728000002BFBD0236038BDF80A002070B50C46F7
:107290000646FFF7CDF8E36A054633B1E1693046AB
:1072A00098470028B8BF4FF0FF35A3891B0619D4B3
:1072B000216B41B104F14003994202D03046FDF701
:1072C0003FFC00232363616C21B13046FDF738FC9D
:1072D00000236364FFF76AFA0023A381FFF768FACB
:1072E000284670BD21693046FDF72AFCE0E700BF63
:1072F000B1B138B505460C4608B1836B4BB1B4F952
:107300000C300BB9002038BD21462846BDE8384076
:10731000BCE7FFF747FAB4F90C30002BF2D0F3E7E3
:1073200000207047C0B138B50C4B1D6804460DB144
:10733000AB6B4BB1B4F90C300BB9002038BD214612
:107340002846BDE83840A1E72846FFF72BFAB4F9F4
:107350000C30002BF1D0F2E7002070470000002035
:1073600070B50C46084D03460026204611461C46C3
:107370002E6001F05CF9431C00D070BD2B68002B1F
:10738000FBD0236070BD00BFF80A002038B5074D60
:107390000022044608462A6001F04EF9431C00D042
:1073A00038BD2B68002BFBD0236038BDF80A0020C5
:1073B00038B50C46084D8446114620461A4600232F
:1073C0002B60644601F03AF9431C00D038BD2B68AD
:1073D000002BFBD0236038BDF80A002038B50C46DE
:1073E000084D8446114620461A4600232B60644609
:1073F00001F0FCF8431C00D038BD2B68002BFBD0FB
:10740000236038BDF80A002081F0004102E000BF8F
:1074100083F0004330B54FEA41044FEA430594EA54
:10742000050F08BF90EA020F1FBF54EA000C55EA8F
:10743000020C7FEA645C7FEA655C00F0E2804FEA60
:107440005454D4EB5555B8BF6D420CDD2C4480EA42
:10745000020281EA030382EA000083EA010180EA72
:10746000020281EA0303362D88BF30BD11F0004FC0
:107470004FEA01314FF4801C4CEA113102D04042F6
:1074800061EB410113F0004F4FEA03334CEA133331
:1074900002D0524263EB430394EA050F00F0A78049
:1074A000A4F10104D5F1200E0DDB02FA0EFC22FA44
:1074B00005F2801841F1000103FA0EF2801843FA38
:1074C00005F359410EE0A5F120050EF1200E012A29
:1074D00003FA0EFC28BF4CF0020C43FA05F3C01867
:1074E00051EBE37101F0004507D54FF0000EDCF1E0
:1074F000000C7EEB00006EEB0101B1F5801F1BD389
:10750000B1F5001F0CD349085FEA30004FEA3C0C8C
:1075100004F101044FEA445212F5800F80F09A8082
:10752000BCF1004F08BF5FEA500C50F1000041EB86
:10753000045141EA050130BD5FEA4C0C404141EB8A
:107540000101013C28BFB1F5801FE9D291F0000F85
:1075500004BF01460020B1FA81F308BF2033A3F134
:107560000B03B3F120020CDA0C3208DD02F1140C2B
:10757000C2F10C0201FA0CF021FA02F10CE002F166
:107580001402D8BFC2F1200C01FA02F120FA0CFC5F
:10759000DCBF41EA0C019040E41AA2BF01EB0451A8
:1075A000294330BD6FEA04041F3C1CDA0C340EDCA6
:1075B00004F11404C4F1200220FA04F001FA02F3E9
:1075C00040EA030021FA04F345EA030130BDC4F1A7
:1075D0000C04C4F1200220FA02F001FA04F340EA9C
:1075E0000300294630BD21FA04F0294630BD94F04D
:1075F000000F83F4801306BF81F480110134013D34
:107600004EE77FEA645C18BF7FEA655C29D094EAA4
:10761000050F08BF90EA020F05D054EA000C04BF22
:107620001946104630BD91EA030F1EBF002100200D
:1076300030BD5FEA545C05D14000494128BF41F0AC
:10764000004130BD14F580043CBF01F5801130BD10
:1076500001F0004545F0FE4141F470014FF000009B
:1076600030BD7FEA645C1ABF194610467FEA655C4C
:107670001CBF0B46024650EA013406BF52EA0335EE
:1076800091EA030F41F4002130BD00BF90F0000FDC
:1076900004BF0021704730B54FF4806404F1320418
:1076A0004FF000054FF0000150E700BF90F0000FD1
:1076B00004BF0021704730B54FF4806404F13204F8
:1076C00010F0004548BF40424FF000013EE700BFC8
:1076D00042004FEAE2014FEA31014FEA02701FBF58
:1076E00012F07F4393F07F4F81F06051704732F08A
:1076F0007F4208BF704793F07F4F04BF41F40021E1
:10770000704730B54FF4607401F0004521F000413E
:107710001CE700BF50EA010208BF704730B54FF0C8
:1077200000050AE050EA010208BF704730B511F0C9
:10773000004502D5404261EB41014FF4806404F101
:1077400032045FEA915C3FF4D8AE4FF003025FEA87
:10775000DC0C18BF03325FEADC0C18BF033202EB0B
:10776000DC02C2F1200300FA03FC20FA02F001FA65
:1077700003FE40EA0E0021FA02F11444BDE600BF08
:1077800070B54FF0FF0C4CF4E06C1CEA11541DBFB7
:107790001CEA135594EA0C0F95EA0C0F00F0DEF882
:1077A0002C4481EA030621EA4C5123EA4C5350EA67
:1077B000013518BF52EA033541F4801143F48013B8
:1077C00038D0A0FB02CE4FF00005E1FB02E506F049
:1077D0000042E0FB03E54FF00006E1FB03569CF09E
:1077E000000F18BF4EF0010EA4F1FF04B6F5007FA4
:1077F00064F5407404D25FEA4E0E6D4146EB060616
:1078000042EAC62141EA55514FEAC52040EA5E509E
:107810004FEACE2EB4F1FD0C88BFBCF5E06F1ED848
:10782000BEF1004F08BF5FEA500E50F1000041EB7F
:10783000045170BD06F0004646EA010140EA02002C
:1078400081EA0301B4EB5C04C2BFD4EB0C0541EA4E
:10785000045170BD41F480114FF0000E013C00F363
:10786000AB8014F1360FDEBF002001F0004170BD87
:10787000C4F10004203C35DA0C341BDC04F11404A0
:10788000C4F1200500FA05F320FA04F001FA05F22C
:1078900040EA020001F0004221F0004110EBD370F9
:1078A00021FA04F642EB06015EEA430E08BF20EA25
:1078B000D37070BDC4F10C04C4F1200500FA04F3C8
:1078C00020FA05F001FA04F240EA020001F000415A
:1078D00010EBD37041F100015EEA430E08BF20EACD
:1078E000D37070BDC4F1200500FA05F24EEA020E15
:1078F00020FA04F301FA05F243EA020321FA04F044
:1079000001F0004121FA04F220EA020000EBD370FA
:107910005EEA430E08BF20EAD37070BD94F0000FFA
:107920000FD101F00046400041EB010111F4801F2E
:1079300008BF013CF7D041EA060195F0000F18BFDF
:10794000704703F00046520043EB030313F4801F1B
:1079500008BF013DF7D043EA0603704794EA0C0FD5
:107960000CEA135518BF95EA0C0F0CD050EA4106EB
:1079700018BF52EA4306D1D181EA030101F0004168
:107980004FF0000070BD50EA410606BF1046194690
:1079900052EA430619D094EA0C0F02D150EA01369C
:1079A00013D195EA0C0F05D152EA03361CBF1046DD
:1079B00019460AD181EA030101F0004141F0FE417C
:1079C00041F470014FF0000070BD41F0FE4141F400
:1079D000780170BD70B54FF0FF0C4CF4E06C1CEA00
:1079E00011541DBF1CEA135594EA0C0F95EA0C0FB5
:1079F00000F0A7F8A4EB050481EA030E52EA033570
:107A00004FEA013100F088804FEA03334FF0805590
:107A100045EA131343EA12634FEA022245EA1115BD
:107A200045EA10654FEA00260EF000419D4208BF6E
:107A3000964244F1FD0404F5407402D25B084FEA1B
:107A40003202B61A65EB03055B084FEA32024FF4C7
:107A500080104FF4002CB6EB020E75EB030E22BF24
:107A6000B61A754640EA0C005B084FEA3202B6EBE4
:107A7000020E75EB030E22BFB61A754640EA5C0093
:107A80005B084FEA3202B6EB020E75EB030E22BF23
:107A9000B61A754640EA9C005B084FEA3202B6EB24
:107AA000020E75EB030E22BFB61A754640EADC00E3
:107AB00055EA060E18D04FEA051545EA16754FEA45
:107AC00006164FEAC30343EA52734FEAC2025FEA63
:107AD0001C1CC0D111F4801F0BD141EA00014FF0F2
:107AE00000004FF0004CB6E711F4801F04BF0143C3
:107AF0000020B4F1FD0C88BFBCF5E06F3FF6AFAEDF
:107B0000B5EB030C04BFB6EB020C5FEA500C50F16E
:107B1000000041EB045170BD0EF0004E4EEA1131F1
:107B200014EB5C04C2BFD4EB0C0541EA045170BDF8
:107B300041F480114FF0000E013C90E645EA060E3C
:107B40008DE60CEA135594EA0C0F08BF95EA0C0F6A
:107B50003FF43BAF94EA0C0F0AD150EA01347FF4B2
:107B600034AF95EA0C0F7FF425AF104619462CE789
:107B700095EA0C0F06D152EA03353FF4FDAE1046EC
:107B8000194622E750EA410618BF52EA43067FF43D
:107B9000C5AE50EA41047FF40DAF52EA43057FF4CD
:107BA000EBAE12E74FF0FF3C06E000BF4FF0010CD8
:107BB00002E000BF4FF0010C4DF804CD4FEA410C3C
:107BC0007FEA6C5C4FEA430C18BF7FEA6C5C1BD009
:107BD00001B050EA410C0CBF52EA430C91EA030F8A
:107BE00002BF90EA020F0020704710F1000F91EAE7
:107BF000030F58BF994208BF90422CBFD8176FEAB5
:107C0000E37040F0010070474FEA410C7FEA6C5C82
:107C100002D150EA013C07D14FEA430C7FEA6C5C89
:107C2000D6D152EA033CD3D05DF8040B704700BFB5
:107C30008446104662468C461946634600E000BF03
:107C400001B5FFF7B7FF002848BF10F1000F01BDD5
:107C50004DF808EDFFF7F4FF0CBF012000205DF8A0
:107C600008FB00BF4DF808EDFFF7EAFF34BF012025
:107C700000205DF808FB00BF4DF808EDFFF7E0FFBE
:107C800094BF012000205DF808FB00BF4DF808ED0F
:107C9000FFF7CEFF94BF012000205DF808FB00BF76
:107CA0004DF808EDFFF7C4FF34BF012000205DF858
:107CB00008FB00BF4FEA410C7FEA6C5C02D150EA3E
:107CC000013C0AD14FEA430C7FEA6C5C02D152EAD4
:107CD000033C02D14FF0000070474FF001007047A5
:107CE0004FEA410212F5001215D211D56FF47873E4
:107CF000B3EB625212D94FEAC12343F0004343EA87
:107D0000505311F0004F23FA02F018BF4042704761
:107D10004FF00000704750EA013005D111F00040EB
:107D200008BF6FF0004070474FF00000704700BF81
:107D300030B589B000240394049405940694079404
:107D40000094194B1A6B42F004021A631A6B02F08A
:107D500004020092009A01941A6B42F080021A63A6
:107D60001A6B02F080020192019A02941A6B42F09F
:107D700001021A631B6B03F001030293029B0B4D7C
:107D800022464FF40051284601F018F84FF40053F2
:107D90000393012304930594069403A9284600F055
:107DA0002DFF09B030BD00BF00380240000802407E
:107DB00010B582B0002401940D4B1A6B42F40012EE
:107DC0001A631B6B03F400130193019B22462146A7
:107DD0000D2000F0FDFC0D2000F032FD22460221B6
:107DE000102000F0F5FC102000F02AFD02B010BDBC
:107DF0000038024072B6FEE700B58BB00023069350
:107E000007930893099304930593009301930293B6
:107E1000039323484FF080420260436083604FF039
:107E2000FF32C2600361836102F04AFB58BB4FF42A
:107E30008053069306A91A4802F06AFC28BB18482A
:107E400002F06AFB18BB502304930023059304A996
:107E5000134802F079FDE0B900220092012301935A
:107E60000292039269460E4802F0E4FB98B902239D
:107E70000093019304226946094802F0DBFB60B9D4
:107E80000BB05DF804FBFFF7B5FFFFF7B3FFFFF79B
:107E9000B1FFFFF7AFFFFFF7ADFFFFF7ABFF00BF8D
:107EA000100C002000B58BB00023069307930893B5
:107EB000099304930593009301930293039322483B
:107EC000224A0260436083604FF0FF32C260036168
:107ED000836102F0F5FA58BB4FF48053069306A96C
:107EE000194802F015FC28BB174802F015FB18BB17
:107EF000002304938023059304A9134802F024FD72
:107F0000E0B9002200920123019302920392694694
:107F10000D4802F08FFB98B90223009301930422CD
:107F20006946094802F086FB60B90BB05DF804FBB6
:107F3000FFF760FFFFF75EFFFFF75CFFFFF75AFFF9
:107F4000FFF758FFFFF756FF580C0020000C0040C9
:107F500008B50C480C4B03605F234360002383602B
:107F600042F21072C2600361836102F0A9FA28B97B
:107F70000821044802F0FCFA10B908BDFFF73AFFE7
:107F8000FFF738FFC80B00200048014008B509483A
:107F9000094B03600523436040F6FF73836000F0E4
:107FA00013FF28B9054A936843F48053936008BDD2
:107FB000FFF720FFBC0B002000300040002004E051
:107FC00000B595B03022002108A8F8F705FB002382
:107FD000039304930593069307930193214A116C2D
:107FE00041F080511164126C02F080520192019AAA
:107FF00002931D4B1A6842F440421A601B6803F456
:1080000040430293029B092308934FF48033099362
:1080100001230D9302230E934FF480020F92192235
:108020001092C022119212930423139308A801F016
:1080300065FD98B90F23039302230493002305934E
:108040004FF4805206920793032103A801F0AAFF80
:1080500030B901F04FFF15B05DF804FBFFF7CAFE21
:10806000FFF7C8FE003802400070004030B597B0FE
:1080700000F05CFBFFF7A4FF674B5B6F13F0005F42
:1080800057D0654A536F43F0807353670124FFF75D
:108090004FFEFFF78DFEFFF7AFFEFFF703FF04F083
:1080A00041FBFFF755FFFFF771FF5C4800F0B8FE9A
:1080B0005B4800F0CBF85B4800F0C8F84FF47A70EA
:1080C00000F060FB584B4FF000529A61002C32D008
:1080D00006AC564D0FCD0FC495E8070084E80700A5
:1080E0001B2106A804F070FB4F4B4FF400529A611D
:1080F0004A4800F095FE4E4C204602F099F80021C7
:10810000204602F093FB0421204602F08FFB2368F7
:108110000525DD60474C204602F08AF80021204604
:1081200002F084FB0421204602F080FB2368DD601E
:108130005AE00024ABE7404B06AC0FCB84E80F00BD
:108140000F21204604F040FBCEE7374C4FF00053A0
:10815000A361049B0093DDE90223384906A8F8F7E0
:10816000A9FA81B206A804F02FFB4FF40053A361D3
:1081700043E02B4B9A68002199602B4C4FF0005341
:10818000A3612F4906A8F8F795FA81B206A804F072
:108190001BFB4FF40053A36133E0234C4FF000531B
:1081A000A361049B0093DDE90223264906A8F8F7A2
:1081B00081FA81B206A804F007FB4FF40053A361D3
:1081C00025E0184B9A6800219960174C4FF0005336
:1081D000A3611D4906A8F8F76DFA81B206A804F05C
:1081E000F3FA4FF40053A3610C4800F019FE02A902
:1081F0000B4800F052F80028A7D1094B9B68002BD0
:10820000B7D102A9074800F048F80028C5D1054BAE
:108210009B68002BE8D0D4E700380240BC0B00205C
:10822000A00C0020B08C002000080240DCCE00082A
:10823000100C0020580C0020E8CE000894CE000856
:10824000A8CE0008B8CE0008CCCE000800230360FA
:10825000436083607047F9B100B584460A464368BD
:108260000133C3F30A0301688B4211D0DCF80430F8
:1082700003F1010E0CEB0E1E0FCA8EE80F00DCF8A6
:1082800004300133C3F30A03CCF804305DF804FB77
:10829000836801338360E9E77047036842689A4264
:1082A0000FD010B586460C4603F1010C00EB0C1301
:1082B0000FCB84E80F00CCF30A03CEF80030012086
:1082C00010BD00207047000082B0002100910B4BD0
:1082D0005A6C42F480425A645A6C02F48042009212
:1082E000009A01911A6C42F080521A641B6C03F0E0
:1082F00080530193019B02B0704700BF00380240D9
:1083000030B58BB00446002305930693079308937A
:1083100009930368B3F1804F08D0554A93424ED079
:10832000544A934200F090800BB030BD0025009578
:1083300003F50E331A6C42F001021A641A6C02F053
:1083400001020092009A01951A6B42F001021A6331
:108350001B6B03F001030193019B20230593022370
:1083600006930123099305A9434800F047FC4348BD
:10837000434B03604FF0C06343608560C5604FF4BA
:10838000806303614FF4805343614FF48043836102
:108390004FF48073C3610562456200F0DBFA58B99F
:1083A000364B63629C63002201211C2000F010FA0E
:1083B0001C2000F045FAB7E7FFF71CFDF0E70025A9
:1083C0000295304B1A6C42F008021A641A6C02F0E3
:1083D00008020292029A03951A6B42F001021A6394
:1083E0001B6B03F001030393039B012305930223FB
:1083F0000693099305A9204800F000FC2248234B6E
:1084000003604FF0406343608560C5604FF4806354
:1084100003614FF4805343614FF480438361C5612E
:108420000562456200F096FA58B9174B63629C6387
:1084300000220121322000F0CBF9322000F000FAB6
:1084400072E7FFF7D7FCF0E7002204920D4B596C5E
:1084500041F4802159645B6C03F480230493049BF2
:108460000F211A2000F0B4F91A2000F0E9F95BE7B7
:10847000000C00400048014000000240FC0A0020BF
:1084800088600240003802405C0B002040600240DF
:1084900008B501F03FFEFEE7FEE7FEE7FEE7FEE778
:1084A00070477047704708B500F05AF908BD0000E2
:1084B00008B5024800F0B4FA08BD00BF5C0B00200C
:1084C00008B5024800F0ACFA08BD00BFFC0A002065
:1084D00008B5024801F0E9FE08BD00BFC80B002046
:1084E0004FF08042136940F20661116113F0010FF1
:1084F00003D015490A6801320A6013F4C06F08D02E
:10850000124A9368013393604FF0804300221A614E
:10851000704713F0040F00D1704700B585B04FF0DD
:1085200080435A6B0092002101919B6B02939B1A2E
:108530000293054B1B68019369460448FFF78BFEC5
:1085400005B05DF804FB00BFC40C0120A00C0020A6
:10855000174A136940F20661116113F0010F03D04D
:1085600014490A6801320A6013F4C06F07D0124A36
:108570009368013393600E4B00221A61704713F029
:10858000040F00D1704700B585B0094B5A6B0092BB
:10859000002101919B6B02939B1A0293054B1B6870
:1085A000019369460448FFF756FE05B05DF804FBE9
:1085B000000C0040C00C0120B08C002008B502481F
:1085C00000F090FF08BD00BFB021012001207047DE
:1085D00008B5F7F7C1FF162303604FF0FF3008BD61
:1085E00008B54FF0FF31FFF7F3FFFEE770B50C461B
:1085F0001646002506E0AFF30080214601F8010B86
:1086000001350C46B542F6DB304670BD70B50C4600
:108610001646002504E014F8010BAFF30080013585
:10862000B542F8DB304670BD4FF0FF3070474FF475
:1086300000534B60002070470120704700207047B6
:1086400010B503460C4A0D490D48006840B10C486E
:1086500000680344521A934206D8094A136010BDB9
:108660000748084C0460F2E7F7F776FF0C23036035
:108670004FF0FF30F3E700BF0000022000040000CD
:10868000C80C0120E028012070470000DFF834D03A
:108690000D480E490E4A002302E0D458C45004335A
:1086A000C4188C42F9D30B4A0B4C002301E0136031
:1086B0000432A242FBD3FFF7E7FFF7F769FFFFF7AA
:1086C000D5FC70470000022000000020A40A002012
:1086D0007CD00008A80A0020DC280120FEE700006A
:1086E00010B504460E4B18784FF47A73B3FBF0F3D1
:1086F0000C4A1068B0FBF3F000F0B0F868B90F2C2A
:1087000001D901200AE0002221464FF0FF3000F09D
:108710005FF8054B1C60002000E0012010BD00BF89
:10872000B0090020AC090020B409002008B50B4BAB
:108730001A6842F400721A601A6842F480621A6081
:108740001A6842F480721A60032000F02FF80F209C
:10875000FFF7C6FFFFF7B8FD002008BD003C024050
:10876000034A1168034B1B780B441360704700BF2A
:10877000CC0C0120B0090020014B1868704700BFE5
:10878000CC0C012038B50446FFF7F6FF0546B4F1DE
:10879000FF3F02D0044B1B781C44FFF7EDFF401B4A
:1087A000A042FAD338BD00BFB0090020074AD36801
:1087B00023F4E0631B041B0C000200F4E06003439D
:1087C00043F0BF6343F40033D360704700ED00E033
:1087D00000B5194BDB68C3F30223C3F1070CBCF1EE
:1087E000040F28BF4FF0040C03F1040EBEF1060F76
:1087F00018D9033B4FF0FF3E0EFA0CFC21EA0C01A6
:1088000099400EFA03F322EA0303194300280BDB15
:108810000901C9B200F1604000F5614080F8001321
:108820005DF804FB0023E5E700F00F000901C9B281
:10883000024B1954F4E700BF00ED00E014ED00E036
:10884000002807DB00F01F02400901239340024A81
:1088500042F82030704700BF00E100E00138B0F17D
:10886000807F0BD24FF0E0235861054AF02182F857
:1088700023100020986107221A6170470120704779
:1088800000ED00E010B40368D9B210390B4AA2FB26
:10889000014212090A4CA25CC2655F2908D923F47F
:1088A0007F7323F0030304338365806D10BC70472E
:1088B00023F47F7323F003038365F6E7ABAAAAAA28
:1088C00008CF0008836A826992B9012B0AD0022B73
:1088D00002D00BB100207047C36A13F0807F28D10B
:1088E00000207047C36AB3F1C07F24D000207047D6
:1088F000B2F5005F09D0022B25D9032B25D1C36A1D
:1089000013F0807F23D100207047032B03D8DFE8CA
:1089100003F01404140A00207047C36A13F0807F28
:108920000DD100207047C36AB3F1C07F09D0002089
:1089300070470120704701207047012070470120D7
:1089400070470120704701207047002070470120C8
:108950007047000070B50446FFF70EFF002C5BD097
:108960000546022384F83530002384F83430226829
:10897000136823F00103136023681A6812F0010FD3
:108980000AD0FFF7F9FE431B052BF5D920236365B9
:10899000032084F8350070BD1A68204810406168D3
:1089A000A2680A43E1680A4321690A4361690A43EC
:1089B000A1690A43E1690A43216A0A430243616AE1
:1089C00004291ED01A602668756925F00705636AB8
:1089D0001D43042B07D1A36A1D43E36A1BB1204644
:1089E000FFF770FF90B975612046FFF74BFFE26D0E
:1089F0003F239340836000206065012384F8353075
:108A0000C9E7E16A206B01430A43DBE74023636562
:108A1000012084F83500BEE70120BCE73F8010F05C
:108A2000F0B583B0044600230193724B1D68724B6E
:108A3000A3FB0535AD0A876D3E68C26D08239340E0
:108A4000334210D003681A6812F0040F0BD01A6872
:108A500022F004021A60C26D08239340BB60436D8C
:108A600043F001034365E26D01239340334209D093
:108A70002268526912F0800F04D0BB60636D43F02E
:108A800002036365E26D04239340334209D02268F8
:108A9000126812F0020F04D0BB60636D43F0040350
:108AA0006365E26D10239340334224D0226812683C
:108AB00012F0080F1FD0BB6023681A6812F4802FD1
:108AC0000DD01B6813F4002F04D1236C9BB12046FA
:108AD000984710E0A36C73B1204698470BE01A68E2
:108AE00012F4807F03D11A6822F008021A60236C06
:108AF0000BB120469847E26D20239340334255D076
:108B00002268126812F0100F50D0BB6094F8353014
:108B1000DBB2052B0ED023681A6812F4802F33D0F5
:108B20001B6813F4002F2AD1636C002B3ED0204623
:108B300098473BE02268136823F01603136022680D
:108B4000536923F080035361236CA3B12268136837
:108B500023F008031360E26D3F239340BB600123C1
:108B600084F83530002384F83430236D002B3FD057
:108B7000204698473CE0A36C002BE7D1EBE7E36B82
:108B8000A3B12046984711E01A6812F4807F09D1FA
:108B90001A6822F010021A60012384F8353000238D
:108BA00084F83430E36B0BB120469847636DFBB11A
:108BB000636D13F0010F17D0052384F83530226858
:108BC000136823F001031360019B01330193AB424F
:108BD00004D823681B6813F0010FF5D1012384F832
:108BE0003530002384F83430E36C0BB120469847CD
:108BF00003B0F0BDAC090020B5814E1B00230F2B44
:108C000000F2D28070B582B060E085685E00032417
:108C1000B44025EA0405CC68B4402C438460456820
:108C200025EA02054C68C4F300129A402A434260C8
:108C30005AE0DC08083450F8246003F0070295007D
:108C40000F22AA4026EA020E0A69AA4042EA0E0250
:108C500040F824205CE0042200E0002202FA0EF238
:108C60002A430234514D45F82420514A94686FEA52
:108C70000C0224EA0C054E6816F4801F01D04CEA61
:108C800004054B4CA560E46802EA04054E6816F43E
:108C9000001F01D04CEA0405454CE560646802EA17
:108CA00004054E6816F4003F01D04CEA0405404C20
:108CB0006560246822404D6815F4803F01D04CEA7D
:108CC00004023B4C226001330F2B6BD801229A40E7
:108CD0000C6804EA020C32EA0404F4D14C6804F093
:108CE0000304013C012C90D94A6802F00302032AD4
:108CF00009D0C4685D000322AA4024EA02048A68FD
:108D0000AA402243C2604A6802F00302022A90D0BD
:108D100004684FEA430E032202FA0EF224EA020428
:108D20004A6802F0030202FA0EF2224302604A6825
:108D300012F4403FC7D0002201921E4A546C44F402
:108D400080445464526C02F480420192019A9C085F
:108D5000A51C164A52F8255003F003024FEA820E72
:108D60000F2202FA0EF225EA0205134A90423FF45E
:108D700074AF02F5806290420ED002F5806290429C
:108D80000CD002F5806290420AD002F580629042D7
:108D90003FF461AF072261E701225FE702225DE74E
:108DA00003225BE702B070BD704700BF003801408E
:108DB000003C014000380240000002400AB18161DD
:108DC000704709048161704740B338B504460368B1
:108DD0004CF6CC421A60036845F255521A6003689B
:108DE00042685A60036882689A60FFF7C5FC0546CE
:108DF0002368DA6812F0030F0BD0FFF7BDFC401BAD
:108E00003128F5D92368DB6813F0030FF0D0032075
:108E100003E04AF6AA221A60002038BD01207047FC
:108E200003684AF6AA221A60002070472DE9F04331
:108E300083B0D0F8008001EBC10300EB8303DA6D4F
:108E40005B6D9A4254D807460C469B1A01EBC1024F
:108E500000EB8202926C9A4200D31A4602F1030997
:108E60004FEA990915E006F103094FEA990904EB65
:108E7000C40507EB8505E96C3B7C0093B3B2E2B215
:108E8000404602F06DF9EB6C3344EB64EB6D334418
:108E9000EB6508EB441303F510639B699BB24B45EC
:108EA00012D304EBC40207EB8202D16D536D9942D9
:108EB0000AD24BB15B1A04EBC40207EB8202966C38
:108EC0009E42D0D31E46CEE704EBC40007EB8007DA
:108ED0007A6DFB6D9A420FD804F00F040123A34072
:108EE000D8F8344824EA0304C8F83448002000E0E5
:108EF000012003B0BDE8F0830020FAE770B58AB026
:108F0000002800F090800546046890F8BD343BB31B
:108F1000032385F8BD34E36B13F4807F01D1002374
:108F20002B61286801F036FE2C4654F8106BEC4695
:108F30000FCCACE80F000FCCACE80F0094E80300B6
:108F40008CE803002B1D0ECB304601F065FD044676
:108F500058B1022385F8BD34012420460AB070BD03
:108F600080F8BC3403F0E0FCD2E70021286802F06E
:108F70000EFB234616E003EBC30205EB8202012140
:108F800082F83D1082F83C30A2F84430002182F88B
:108F900040109164D16403EBC30205EB820251657A
:108FA0000133DBB269688B42E5D316E004EBC403FE
:108FB00005EB8303002283F87D2283F87C4283F84B
:108FC0008022C3F88822C3F88C2204EBC40305EB8B
:108FD0008303C3F894220134E4B2A142E6D82C46BC
:108FE00054F8106BEC460FCCACE80F000FCCACE89B
:108FF0000F0094E803008CE803002B1D0ECB3046D5
:1090000001F024FE044620B1022385F8BD3401247A
:10901000A3E7002385F83830012385F8BD3428689C
:1090200002F073FA99E7012497E7026890F8BC34DC
:10903000012B19D010B50446012380F8BC34836A93
:10904000012B09D0206801F09FFD206802F04FFA43
:10905000002084F8BC0410BD8369012BF2D0936B0F
:1090600043F480339363EDE70220704770B5044604
:109070000D460068066C00EB411303F530639A68F7
:109080002169012911D038498E4256D03DB905EBEE
:10909000C50304EB8303D3F89432002B5ED0E9B20E
:1090A000204603F08BFC002070BD12F0080F09D0A1
:1090B0002E498E42F7D912F4004FF4D04FF40042FB
:1090C0009A60F0E712F0200F02D020229A60EAE7BF
:1090D00012F0280FE7D125498E4206D912F4004F2D
:1090E00003D04FF400429A60DDE705EBC50204EBC4
:1090F0008202D2F898121B69C3F31203CB1AC2F88A
:109100009C327DB905EBC50204EB8202D2F89422B1
:109110006AB105EBC50204EB8202D2F88C120B4453
:10912000C2F88C32E9B2204603F048FCBBE704F2F7
:10913000C442012102F06CFAF4E712F4004F03D0AC
:109140004FF400429A60AEE712F0200F01D02022C7
:109150009A60E9B2204603F031FCA4E704F2C4426D
:10916000002102F055FA9AE70A31544F0A30544F61
:1091700038B5044603681D6C03EB4113D3F8081B94
:109180000E4A954207D903F5306311F4004F02D01F
:109190004FF400429A60204603F008FC074B9D42C2
:1091A00002D92369012B01D0002038BD04F2C4424A
:1091B0000121206802F02CFAF6E700BF0A30544F74
:1091C00090F8BC34012B0DD010B50446012380F873
:1091D000BC3480F83810006802F079F9002084F877
:1091E000BC0410BD0220704738B505468C4611F00E
:1091F000800F29D101F00F0E0EEBCE04A40004F570
:109200001E740444211D0EEBCE0E00EB8E0E0020CA
:109210008EF87D020CF00F0C81F800C0CA600B7153
:109220004A780AB1A1F808C0022B1DD095F8BC34C9
:10923000012B1CD0012385F8BC34286801F0DFFD28
:10924000002085F8BC0438BD01F00F0000EBC00120
:10925000890038312944043100EBC00005EB80005F
:10926000012480F83D40D5E700234B71DEE7022062
:10927000E9E710B504460A4611F0800F20D101F04D
:109280000F0000EBC0039B0003F51E732344191D60
:1092900000EBC00004EB8000002380F87D3202F078
:1092A0000F020A7094F8BC34012B19D0012384F802
:1092B000BC34206801F0F2FD002084F8BC0410BD2D
:1092C00001F00F0000EBC0039B0038332344191D4D
:1092D00000EBC00004EB8000012380F83D30DEE7A6
:1092E0000220ECE710B501F00F0404EBC401890083
:1092F00001F51E710144043104EBC40C00EB8C0C2D
:10930000CCF88C22CCF894320023CCF89C328CF828
:109310007D328CF87C420369012B06D064B9DAB245
:10932000006801F02BFE002010BD04EBC40C00EB24
:109330008C0CCCF89022F1E7DAB2006801F028FF3B
:10934000F1E701F00F0101EBC10100EB8101D1F860
:109350009C02704710B501F00F0404EBC4018900B2
:1093600038310144043104EBC40C00EB8C0CCCF814
:109370004C20CCF854300023CCF85C3001238CF81E
:109380003D308CF83C400369012B06D064B9DAB259
:10939000006801F0F3FD002010BD04EBC40C00EBED
:1093A0008C0CCCF85020F1E7DAB2006801F0F0FE46
:1093B000F1E738B501F00F054268954239D8044607
:1093C0000B4611F0800F1FD101EBC101890001F59F
:1093D0001E710144043103EBC30300EB830300223D
:1093E00083F87D2201238B700D7094F8BC34012B1F
:1093F00021D0012384F8BC34206802F00DF88DB12F
:10940000002084F8BC0438BD05EBC5018900383163
:109410000144043105EBC50300EB8303012283F80B
:109420003D20DFE704F2C442217C206802F0F0F81E
:10943000E6E70120E7E70220E5E701F00F034268D5
:10944000934231D810B5044611F0800F1ED103EBC2
:10945000C301890001F51E710144043103EBC3020D
:1094600000EB8202002082F87D0200228A700B70DD
:1094700094F8BC34012B19D0012384F8BC34206843
:1094800001F0F7FF002084F8BC0410BD03EBC3011A
:10949000890038310144043103EBC30200EB82023E
:1094A000012082F83D00E0E7012070470220ECE750
:1094B00008B511F0800F0CD101F00F0101EBC101D3
:1094C000890001F51E7101440431006801F0EAFDD4
:1094D00008BD01F00F0101EBC101890038310144E1
:1094E0000431F2E72DE9F04F83B0044605682846C1
:1094F00002F049F810B103B0BDE8F08F06462068CD
:1095000002F011F80028F6D005F50067BB68C3F338
:109510000D23C4F8FC34206802F005F810F0020FA7
:1095200004D02268536903F002035361206801F0FC
:10953000FAFF10F0100F13D02268936923F0100384
:109540009361D5F8208008F00F09C8F34343022B3C
:109550004BD0062B6FD02268936943F010039361C0
:10956000206801F0E0FF10F4002F76D1206801F0B0
:10957000DAFF10F4802F40F0E080206801F0D3FF84
:109580000028C0F26381206801F0CDFF10F4006F65
:1095900009D0BB6813F0010F40F070812268536955
:1095A00003F400635361206801F0BDFF10F4805F95
:1095B00040F06881206801F0B6FF10F4005F40F0D1
:1095C000B581206801F0AFFF10F0080F40F0C681B0
:1095D000206801F0A8FF10F0800F00F0D981AB697E
:1095E00023F08003AB610126C2E147F6F07318EA6D
:1095F000030FB0D04FEA181B4FEAC903019309EBE0
:10960000C90A04EB8A0AC8F30A12DAF88C1228464F
:1096100001F0D8FECBF30A0BDAF88C325B44CAF8BF
:109620008C32019B4B4404EB8303D3F89C325B44A4
:10963000CAF89C328FE7082204F2C441284601F0A0
:10964000C1FEC8F30A1809EBC90204EB8202D2F882
:109650009C324344C2F89C327DE7206801F067FFEA
:109660008046B14635E005EB49130122C3F8082BCB
:1096700049462046FFF7FAFC3CE005EB4913082277
:10968000C3F8082B49462046FFF772FD35E009EB89
:10969000C90304EB830393F87F32012B41D005EB20
:1096A00049130222C3F8082B1AF0200F04D005EB4F
:1096B00049132022C3F8082B1AF4005F05D005EBEC
:1096C00049134FF40052C3F8082B09F101094FEA7E
:1096D0005808B8F1000F3FF449AF18F0010FF4D06B
:1096E0005FFA89FB5946206801F031FF824610F08D
:1096F000010FB8D11AF0080FBFD11AF0100F04D023
:1097000005EB49131022C3F8082B1AF0020FCBD037
:109710006B6913F0800FBAD07B6843F480637B6081
:10972000B5E709EBC90304EB8303002283F87F222A
:109730005946204603F090F9B1E7206801F0FFFE9A
:109740008046B14625E05946204603F043F91AF019
:10975000080F04D005EB49130822C3F808291AF0B2
:10976000100F04D005EB49131022C3F808291AF092
:10977000400F04D005EB49134022C3F808291AF022
:10978000020F40D11AF0800F5BD109F101094FEAB5
:109790005808B8F1000F3FF4F0AE18F0010FF4D004
:1097A0005FFA89FB5946206801F0DAFE824610F024
:1097B000010FCCD009F00F03012101FA03F27B6BFA
:1097C00023EA02037B6305EB4913C3F808192369F5
:1097D0008B42B8D109EBC90304EB8303996CDA6CB3
:1097E0000A44DA64B9F1000FADD109EBC90304EB07
:1097F00083035B6D002BA6D104F2C44201212068D3
:1098000001F006FF9FE74946284601F0C9F909EB38
:10981000C90304EB830393F83F30012B05D005EB1C
:1098200049130222C3F80829ACE709EBC90304EB8A
:109830008303002283F83F205946204603F012F9A3
:10984000EDE749462046FFF7F1FA9EE77B6823F0F3
:1098500001037B6094F8F434012B08D0204603F018
:10986000F5F82268536903F0004353618BE6002149
:1098700084F8F414204600F040F9F2E7204603F0A3
:10988000CDF88BE67B6823F001037B601021206814
:1098900001F086F91AE005EB46134FF67F31C3F865
:1098A0000819D3F8002922F40012C3F80029C3F8DC
:1098B000081BD3F8002B22F40012C3F8002BD3F8B6
:1098C000002B42F00062C3F8002B01366368B342FC
:1098D000E1D8FB6943F00113FB61236BDBB1D7F8DF
:1098E000843043F00B03C7F884307B6C43F00B03E8
:1098F0007B64D5F8003823F4FE63C5F8003804F221
:10990000C442217C206801F083FE2268536903F47D
:10991000805353614EE67B6943F4005343F02B03BD
:109920007B613B6943F00B033B61E2E7206801F098
:109930005FFE206801F052FAE060266800F0E2FB6A
:109940000146227B304601F0ADF8204603F053F883
:109950002268536903F40053536132E6204603F052
:1099600044F82268536903F00803536130E6013676
:109970006368B3420CD906EBC60304EB830393F888
:109980007F32012BF3D1F1B22046FFF791FDEEE7D4
:10999000206801F0C8FD10F4801F27D1206801F075
:1099A000C2FD10F4001F5BD0012328E0013663687C
:1099B000B3421DD905EB4613D3F8002906EBC603C5
:1099C00004EB830393F84030012BEFD1002AEDDA4A
:1099D00006EBC60304EB8303012283F83F2066F005
:1099E0007F01C9B22046FFF763FDDFE70126DEE70E
:1099F0002268536903F480135361CFE7013362682F
:109A00009A4228D905EB4312D2F8001B03EBC3029C
:109A100004EB820292F88022012AEFD10029EDDACC
:109A200001F48031D4F8FC2402F001029142E5D126
:109A300003EBC30204EB8202012182F87F12AA69C0
:109A400042F08002AA616A6912F0800FD6D17B6869
:109A500043F400737B602268536903F4001353617D
:109A6000206801F060FD10F0804F10D1206801F0F7
:109A70005AFD10F0040F3FF43EAD23685D6815F009
:109A8000040F0DD1226853682B43536033E5204601
:109A900002F0EEFF2268536903F080435361E5E76B
:109AA000204602F0EBFFEDE710B40468606A29B9C4
:109AB00040EA0240A062002010BC70478C46A36AB6
:109AC00000EB1340002308E003F1400104EB8101A7
:109AD000496800EB11400133DBB20CF1FF318B42DE
:109AE000F2D340EA02400CF13F0104EB81014860EF
:109AF000E1E703685962002070477047002800F0D2
:109B0000E08170B582B00446036813F0010F3BD0CA
:109B10009F4B9B6803F00C03042B2CD09C4B9B6841
:109B200003F00C03082B21D06368B3F5803F4FD0BE
:109B3000B3F5A02F52D0964B1A6822F480321A60E7
:109B40001A6822F480221A606368002B50D0FEF756
:109B500013FE05468E4B1B6813F4003F14D1FEF72D
:109B60000BFE401B6428F5D90320B1E1884B5B68EC
:109B700013F4800FD8D0864B1B6813F4003F03D03A
:109B80006368002B00F09F81236813F0020F54D00C
:109B90007F4B9B6813F00C0F3ED07D4B9B6803F00E
:109BA0000C03082B33D0E368002B68D0794B0122DB
:109BB0001A60FEF7E1FD0546754B1B6813F0020FB6
:109BC00054D1FEF7D9FD401B0228F5D903207FE1CF
:109BD0006F4A136843F480331360B5E76C4B1A681F
:109BE00042F480221A601A6842F480321A60ABE7AD
:109BF000FEF7C2FD0546664B1B6813F4003FC3D059
:109C0000FEF7BAFD401B6428F5D9032060E1604BE4
:109C10005B6813F4800FC6D15D4B1B6813F0020F15
:109C200003D0E368012B40F05081594A136823F0B8
:109C3000F803216943EAC1031360236813F0080F96
:109C400042D063696BB3534B0122C3F8802EFEF7F9
:109C500093FD05464E4B5B6F13F0020F34D1FEF7B8
:109C60008BFD401B0228F5D9032031E1484A1368D7
:109C700023F0F803216943EAC1031360DDE7454B94
:109C800000221A60FEF778FD0546414B1B6813F071
:109C9000020FD2D0FEF770FD401B0228F5D9032039
:109CA00016E13C4B0022C3F8802EFEF765FD054609
:109CB000374B5B6F13F0020F06D0FEF75DFD401BC4
:109CC0000228F5D9032003E1236813F0040F77D0AD
:109CD0002F4B1B6C13F0805F33D1002301932C4B6F
:109CE0001A6C42F080521A641B6C03F0805301938B
:109CF000019B0125284B1B6813F4807F23D0A368A8
:109D0000012B34D0052B38D0214B1A6F22F00102E1
:109D10001A671A6F22F004021A67A368002B3DD05D
:109D2000FEF72AFD06461A4B1B6F13F0020F46D1B1
:109D3000FEF722FD801B41F288339842F3D90320BD
:109D4000C6E00025D6E7144A136843F48073136015
:109D5000FEF712FD0646104B1B6813F4807FCED130
:109D6000FEF70AFD801B0228F5D90320B0E0084A5F
:109D7000136F43F001031367CFE7054B1A6F42F0EF
:109D800004021A671A6F42F001021A67C5E700BFA2
:109D9000003802400000474200700040FEF7ECFC33
:109DA0000646524B1B6F13F0020F08D0FEF7E4FC7F
:109DB000801B41F288339842F3D9032088E0EDB943
:109DC000A369002B00F08380484A926802F00C02DD
:109DD000082A51D0022B17D0454B00221A66FEF7F5
:109DE000CBFC0446414B1B6813F0007F42D0FEF7CA
:109DF000C3FC001B0228F5D9032069E03B4A136C21
:109E000023F080531364DBE7394B00221A66FEF718
:109E1000B3FC0546354B1B6813F0007F06D0FEF7F8
:109E2000ABFC401B0228F5D9032051E0E369226A0C
:109E30001343626A43EA8213A26A5208013A43EA70
:109E40000243E26A43EA0263284A5360284B012234
:109E50001A66FEF791FC0446244B1B6813F0007F42
:109E600006D1FEF789FC001B0228F5D903202FE05C
:109E700000202DE000202BE0012B2BD01B4B5B683A
:109E800003F48001E269914226D103F03F02216A86
:109E90008A4223D1616A47F6C0721A40B2EB811F31
:109EA0001ED103F44031A26A5208013AB1EB024FCD
:109EB00018D103F07063E26AB3EB026F14D1002093
:109EC00006E001207047012002E0012000E00020B0
:109ED00002B070BD0120FBE70120F9E70120F7E7A0
:109EE0000120F5E70120F3E70120F1E70038024007
:109EF00000004742014B0122DA64704700004742EC
:109F000008B5254B9B6803F00C03042B3FD0082BAE
:109F10003FD1214B5A6802F03F025B6813F4800F77
:109F200012D01D4B5968C1F388111C480023A1FBB6
:109F30000001F6F789F9184B5B68C3F3014301335D
:109F40005B00B0FBF3F025E0134B5968C1F3881CAC
:109F50004FEA4C11B1EB0C006EEB0E0E4FEA8E1374
:109F600043EA90638101091A63EB0E03DB0043EAC5
:109F70005173C90011EB0C0C43F10003990200234B
:109F80004FEA8C2041EA9C51F6F75EF9D3E703488B
:109F900000E0034808BD00BF0038024040787D0162
:109FA0000024F400002800F09B8070B50D460446A4
:109FB0004F4B1B6803F007038B4208D2CBB24C4ACD
:109FC0001370136803F007038B4240F08B80236803
:109FD00013F0020F17D013F0040F04D0454A936812
:109FE00043F4E0539360236813F0080F04D0414A10
:109FF000936843F4604393603E4A936823F0F00310
:10A00000A1680B439360236813F0010F32D063689B
:10A01000012B21D09A1E012A25D9364A126812F046
:10A02000020F61D033498A6822F0030213438B6028
:10A03000FEF7A2FB06462F4B9B6803F00C036268F9
:10A04000B3EB820F16D0FEF797FB801B41F28833EB
:10A050009842F0D9032042E0264A126812F4003FE9
:10A06000E0D101203BE0234A126812F0007FD9D1F1
:10A07000012034E01E4B1B6803F00703AB4207D9F5
:10A08000EAB21B4B1A701B6803F00703AB422DD1D9
:10A09000236813F0040F06D0164A936823F4E053A4
:10A0A000E1680B439360236813F0080F07D0114A4F
:10A0B000936823F46043216943EAC1039360FFF787
:10A0C0001FFF0C4B9B68C3F303130B4AD35CD840B0
:10A0D0000A4B18600A4B1868FEF702FB002070BD9F
:10A0E000012070470120FAE70120F8E70120F6E798
:10A0F000003C024000380240F8CE0008AC090020C5
:10A10000B4090020014B1868704700BFAC0900205B
:10A110007047000008B5064BDB6813F0800F00D1D4
:10A1200008BDFFF7F5FF024B80229A73F8E700BFE6
:10A130000038024010B4036A046A24F00104046287
:10A14000846924F0F00C4CEA021223F00A030B435A
:10A150008261036210BC704730B4046A24F01004BA
:10A1600004628469056A24F4407C4CEA022C2CF4D5
:10A17000704C1B039BB243EA0C0325F0A0050901B8
:10A1800001F0A00129438361016230BC704710B423
:10A19000046A24F0100404628469036A24F4704C95
:10A1A0004CEA023223F0A00343EA01138261036206
:10A1B00010BC704730B4046A24F480740462C4692B
:10A1C000056A24F0030C4CEA020C2CF0F00C1B0185
:10A1D000DBB243EA0C0325F42065090201F4206197
:10A1E0002943C361016230BC704730B4046A24F46F
:10A1F00080540462C469056A24F4407C4CEA022C51
:10A200002CF4704C1B039BB243EA0C0325F420454D
:10A21000090301F420412943C361016230BC704746
:10A22000836823F070030B4343F007038360704798
:10A2300090F83D30DBB2012B2AD1022380F83D306B
:10A240000368154A934218D0B3F1804F15D0A2F598
:10A250007C42934211D002F5806293420DD002F508
:10A260008062934209D002F59A32934205D01A686F
:10A2700042F001021A60002070479A6802F007025B
:10A28000062A07D01A6842F001021A6000207047BF
:10A290000120704700207047000001407047704760
:10A2A0007047704770477047704710B504460368A1
:10A2B0001A6912F0020F11D0DA6812F0020F0DD0F5
:10A2C0006FF002021A610123037703689B6913F0A0
:10A2D000030F70D0FFF7E6FF0023237723681A6986
:10A2E00012F0040F12D0DA6812F0040F0ED06FF0E3
:10A2F00004021A610223237723689B6913F4407FC9
:10A300005FD02046FFF7CEFF0023237723681A692A
:10A3100012F0080F12D0DA6812F0080F0ED06FF0AA
:10A3200008021A61042323772368DB6913F0030F03
:10A330004ED02046FFF7B6FF0023237723681A6923
:10A3400012F0100F12D0DA6812F0100F0ED06FF06A
:10A3500010021A61082323772368DB6913F4407F16
:10A360003DD02046FFF79EFF0023237723681A691C
:10A3700012F0010F03D0DA6812F0010F36D1236812
:10A380001A6912F0800F03D0DA6812F0800F34D10E
:10A3900023681A6912F0400F03D0DA6812F0400FF8
:10A3A00032D123681A6912F0200F03D0DA6812F054
:10A3B000200F30D110BDFFF774FF2046FFF773FF69
:10A3C0008AE72046FFF76DFF2046FFF76CFF9BE70B
:10A3D0002046FFF766FF2046FFF765FFACE7204603
:10A3E000FFF75FFF2046FFF75EFFBDE76FF001025A
:10A3F0001A612046FFF754FFC1E76FF080021A612F
:10A40000204600F0E0FAC3E76FF040021A612046F0
:10A41000FFF74AFFC5E76FF020021A61204600F0FF
:10A42000D1FAC7E70368254A90420ED0B0F1804FB9
:10A430000BD0A2F57C42904207D002F58062904298
:10A4400003D002F58062904203D123F070034A6882
:10A4500013431A4A90421AD0B0F1804F17D0A2F598
:10A460007C42904213D002F5806290420FD002F5F8
:10A47000806290420BD002F59A32904207D002F5EA
:10A480008062904203D002F58062904203D123F4AF
:10A490004073CA68134323F080034A69134303607F
:10A4A0008B68C3620B688362044B984202D001231D
:10A4B000436170470B690363F9E700BF0000014087
:10A4C00040B310B5044690F83D30F3B1022384F850
:10A4D0003D30214651F8040BFFF7A4FF012384F817
:10A4E000463084F83E3084F83F3084F8403084F8B9
:10A4F000413084F8423084F8433084F8443084F8A2
:10A50000453084F83D30002010BD80F83C30FDF728
:10A51000F7FEDBE70120704740B310B5044690F822
:10A520003D30F3B1022384F83D30214651F8040B4D
:10A53000FFF778FF012384F8463084F83E3084F832
:10A540003F3084F8403084F8413084F8423084F859
:10A55000433084F8443084F8453084F83D3000209E
:10A5600010BD80F83C30FFF799FEDBE70120704713
:10A5700050B338B50D46044690F83D30FBB1022388
:10A5800084F83D30214651F8040BFFF74BFF226859
:10A59000136823F008031360236819680D431D60D6
:10A5A000012384F8463084F83E3084F83F3084F844
:10A5B000423084F8433084F83D30002038BD80F8C4
:10A5C0003C30FFF76CFEDAE70120704770B4046A94
:10A5D00024F0010404628469066A154DA84215D06E
:10A5E000B0F1804F12D0A5F57C45A8420ED005F5FC
:10A5F0008065A8420AD005F58065A84206D005F519
:10A600009A35A84202D044F0010202E024F003048B
:10A61000224322F0F0021B01DBB2134326F00A02B0
:10A6200001F00A0111438361016270BC704700BFF1
:10A630000000014038B590F83C30012B5AD0044658
:10A640000D46012380F83C3052B1042A1AD0082A62
:10A650002BD00C2A3BD00120002384F83C3038BD9D
:10A66000CB684A6809680068FFF7B0FF2268936901
:10A6700023F00C03936122689369A9680B439361EB
:10A680000020E9E7CB684A6809680068FFF764FDC5
:10A690002268936923F44063936122689369A968EF
:10A6A00043EA012393610020D6E7CB684A68096832
:10A6B0000068FFF77FFD2268D36923F00C03D361A4
:10A6C0002268D369A9680B43D3610020C4E7CB6833
:10A6D0004A6809680068FFF788FD2268D36923F497
:10A6E0004063D3612268D369A96843EA0123D36137
:10A6F0000020B1E70220B2E710B4846824F47F4C54
:10A7000042EA03220A4342EA0C02826010BC70470C
:10A7100090F83C30012B78D010B50446012380F826
:10A720003C30022380F83D300268936823F47F4375
:10A7300023F0770393600B68602B4CD029D8402B13
:10A7400054D00CD9502B22D1CA6849680068FFF751
:10A75000F1FC50212068FFF763FD002005E0202B6D
:10A760000DD009D9302B0AD00120012384F83D30C7
:10A77000002384F83C3010BD0BB1102B05D11946D5
:10A780002068FFF74DFD0020EFE70120EDE70120F5
:10A79000EBE7B3F5805F34D0B3F5005F0CD1CB6845
:10A7A0004A6889680068FFF7A7FF2268936843F446
:10A7B000804393600020D8E7702B24D1CB684A688F
:10A7C00089680068FFF798FF2268936843F0770371
:10A7D00093600020C9E7CA6849680068FFF7D7FCA2
:10A7E00060212068FFF71CFD0020BEE7CA684968A9
:10A7F0000068FFF79FFC40212068FFF711FD002053
:10A80000B3E70020B1E70120AFE70220704701F075
:10A810001F01012303FA01FC036A23EA0C0303620C
:10A82000036A02FA01F10B430362704710B5044654
:10A830000B46002937D190F83E00C0B2002B42D120
:10A8400094F84220D2B2012878D1012A77D1002B86
:10A8500049D1022284F83E20002B54D1022284F8F0
:10A860004220012219462068FFF7D1FF2368354AAC
:10A87000934258D0B3F1804F55D0A2F57C42934219
:10A8800051D002F5806293424DD002F5806293422E
:10A8900049D002F59A32934245D01A6842F001023B
:10A8A0001A6000204BE0042905D0082907D090F851
:10A8B0004100C0B2C2E790F83F00C0B2BEE790F8D6
:10A8C0004000C0B2BAE7042B05D0082B07D094F89B
:10A8D0004520D2B2B7E794F84320D2B2B3E794F858
:10A8E0004420D2B2AFE7042B05D0082B07D00222B8
:10A8F00084F84120B0E7022284F83F20ACE702222E
:10A9000084F84020A8E7042B05D0082B07D00222AA
:10A9100084F84520A5E7022284F84320A1E702221B
:10A9200084F844209DE79A6802F00702062A07D0BF
:10A930001A6842F001021A60002000E0012010BDF8
:10A940000020FCE70000014090F83C30012B34D09F
:10A9500010B4012380F83C30022380F83D300368B6
:10A960005A689C6822F0700C0A6842EA0C025A602D
:10A970000368134A934212D0B3F1804F0FD0A2F56F
:10A980007C4293420BD002F58062934207D002F5DD
:10A990008062934203D002F59A32934204D124F0AC
:10A9A00080044A6814439C60012380F83D300023F2
:10A9B00080F83C30184610BC70470220704700BF3A
:10A9C000000001407047704782B000230193019B53
:10A9D00001330193019A0F4B9A4215D80369002B5A
:10A9E000F5DA00230193036943F001030361019B3E
:10A9F00001330193019A074B9A4208D8036913F077
:10AA0000010FF4D1002000E0032002B070470320C2
:10AA1000FBE700BF400D030084B010B5044603A857
:10AA200080E80E00089B012B1FD1A36B23F4803319
:10AA3000A363E36823F4840323F04003E360E36843
:10AA400023F44013E3600F9B012B09D02046FFF74E
:10AA5000BBFF069B012B1BD0BDE8104004B0704724
:10AA6000E36843F48013E360F0E7E36843F04003F6
:10AA7000E3602046FFF7A8FF0C9B23B9A36B43F4C8
:10AA80008033A363E5E7A36B23F48033A363E0E79C
:10AA9000A36843F00603A360A36843F02003A36008
:10AAA000DAE70000022A0AD00921C26822F47052B3
:10AAB000C260C36843EA8123C36000207047234B10
:10AAC0000B44234A93422FD9224B0B44224A9342F0
:10AAD0002CD9A1F57403A3F51053204A934227D92A
:10AAE000A1F18373A3F5E7431D4A934222D31D4B83
:10AAF0000B441D4A93421FD91C4B0B441C4A9342E2
:10AB00001CD31C4B0B441C4A934219D3A1F1B773BD
:10AB1000A3F55853194A934214D3194B0B44194ABD
:10AB2000934211D20721C0E70F21BEE70E21BCE7F7
:10AB30000D21BAE70C21B8E70B21B6E70A21B4E7EB
:10AB40000921B2E70821B0E70621AEE7405327FF0D
:10AB5000FF340C00401E1BFF3F420F007F4F1200CE
:10AB600020D6130060B6E5FE5FE3160000D3CEFEEC
:10AB700040771B00C05BB3FEC091210020753800F8
:10AB8000E05459FEE09C4100836843F00103836078
:10AB900000207047836823F0010383600020704722
:10ABA00082B000230193019B01330193019A0F4B63
:10ABB0009A4215D80369002BF5DA00230193890125
:10ABC00041F020010161019B01330193019A074B80
:10ABD0009A4208D8036913F0200FF4D1002000E056
:10ABE000032002B070470320FBE700BF400D0300C5
:10ABF00082B000230193019B01330193019A0E4B14
:10AC00009A4213D80369002BF5DA0023019310232D
:10AC10000361019B01330193019A074B9A4208D8C3
:10AC2000036913F0100FF4D1002000E0032002B0FC
:10AC300070470320FBE700BF400D0300D0F8003849
:10AC40001943C0F8001800207047000084B02DE9B7
:10AC5000F041044607A880E80E00002306E003F157
:10AC6000400204EB82020021516001330E2BF6D921
:10AC7000119F27BBD4F8043843F00203C4F804380A
:10AC8000A36B43F40013A363A36B23F40023A36318
:10AC9000A36B23F48023A3630023C4F8003E04F5D0
:10ACA0000065D4F80038C4F800380C9B012B14D18F
:10ACB000099B6BB900212046FFF7C0FF11E0A36B91
:10ACC00023F40013A363A36B43F40023A363E3E71C
:10ACD00001212046FFF7B2FF03E003212046FFF7E2
:10ACE000ADFF10212046FFF75BFF804608B14FF013
:10ACF00001082046FFF77CFF08B14FF00108002350
:10AD00002B616B61EB610AE0C3B94FF00060C2F8E0
:10AD1000000900220A614FF67F328A6001330799E9
:10AD2000994210D904EB431202F51061D2F80009E0
:10AD30000028E9DB0020C2F80009EAE74FF0904064
:10AD4000C2F80009E5E700230AE0C3B14FF0904CD8
:10AD5000C2F800CB002202614FF67F3282600133DD
:10AD6000994211D904EB431202F53060D2F8006B1E
:10AD7000002EEADB4FF0000CC2F800CBEAE74FF000
:10AD8000006CC2F800CBE5E72B6923F480732B61DC
:10AD90000023A3616FF0804363610A9B1BB9A36921
:10ADA00043F01003A361A2690B4B1343A3610D9BF6
:10ADB0001BB1A36943F00803A361012F04D04046EF
:10ADC000BDE8F04104B07047A36943F0804343F00D
:10ADD0000403A361F3E700BF00383C80D0F80838D3
:10ADE00013F0060307D0022B07D0062B01D00F204B
:10ADF000704702207047002070470220704710B54E
:10AE000091F800C04B78012B23D000F5006ED0F8EC
:10AE10001C380CF00F040122A24043EA0243C0F8A0
:10AE20001C3800EB4C10D0F8003B13F4004F0ED14F
:10AE3000D0F8003BCA68C2F30A02097942EA8142AB
:10AE4000134343F0805343F40043C0F8003B002019
:10AE500010BDD0F81C280CF00F0E03FA0EF39BB2B5
:10AE60001343C0F81C3800EB4C10D0F8003913F431
:10AE7000004FECD1D0F80039CA68C2F30A02097950
:10AE800042EA814242EA8C5C43EA0C0343F080537D
:10AE900043F40043C0F80039D9E7000030B40B7820
:10AEA0004A78012A26D000EB4313D3F8002B002A5E
:10AEB00052DBD0F83C480A7802F00F024FF0010C48
:10AEC0000CFA02F224EA0242C0F83C28D0F81C280E
:10AED000097801F00F010CFA01FC22EA0C42C0F8DB
:10AEE0001C28D3F8001B234A0A40C3F8002B00207B
:10AEF00030BC704700EB4313D3F80029002A1EDB57
:10AF0000D0F83C580A7802F00F02012404FA02F249
:10AF100092B225EA0202C0F83C28D0F81C28097831
:10AF200001F00F018C40A4B222EA0404C0F81C48CE
:10AF3000D3F80019104A0A40C3F80029D7E7D3F81C
:10AF4000002942F00062C3F80029D3F8002942F03A
:10AF50008042C3F80029D3E7D3F8002B42F0006207
:10AF6000C3F8002BD3F8002B42F08042C3F8002B2B
:10AF70009FE700BF0078F3EF007833EC30B40B7834
:10AF80004C78012C29D000EB431000F530631C698C
:10AF9000E40CE4041C611C6924F0FF5424F4C01484
:10AFA0001C618C690CB1CC688C61CC68CC611C696B
:10AFB00044F400241C611C69CD69C5F3120C44EAF9
:10AFC0000C041C61012A68D0D0F8003B43F0044314
:10AFD000C0F8003B002030BC70478C696CBB00EBB4
:10AFE0004314D4F8105925F0FF5525F4C015C4F8C2
:10AFF0001059D4F8105945F40025C4F81059D4F864
:10B000001059ED0CED04C4F81059012A36D000EBAC
:10B010004313D3F8002942F00442C3F800298B6996
:10B02000002BD7D0D0F834380A7802F00F01012273
:10B030008A401343C0F83438CCE700EB431404F5DE
:10B0400010642569ED0CED042561256925F0FF5597
:10B0500025F4C0152561CD68D1F818C0AC4500D9DC
:10B060008D61256945F4002525612569D1F818C051
:10B07000CCF3120C45EA0C052561C6E74A691AB102
:10B0800000EB4311C1F8142900EB4310D0F800295C
:10B0900042F00442C0F800299CE70A69002A93D0D4
:10B0A0005A6191E710B483B00246002301934878B7
:10B0B00001280AD00B7802EB4313D3F8000B0028C9
:10B0C0002CDB002003B010BC70470B7802EB43135D
:10B0D000D3F80049002C01DB0020F3E7D3F8004946
:10B0E00044F00064C3F800490B7802EB4313D3F833
:10B0F000004944F08044C3F80049019B01330193A7
:10B10000019C42F210739C42DCD80B7802EB431393
:10B11000D3F80039002BF0DB0020D3E7D3F8000B85
:10B1200040F00060C3F8000B0B7802EB4313D3F838
:10B13000000B40F08040C3F8000B019B01330193EA
:10B14000019842F21073984208D80B7802EB43132F
:10B15000D3F8003B002BF0DB0020B3E70120B1E780
:10B1600010B59DF8084084B903334FEA930E4FF0B1
:10B17000000C08E000EB023303F5805351F8044B58
:10B180001C600CF1010CF445F4D3002010BD00004C
:10B19000F0B583B00B784C78012C33D000EB43131F
:10B1A00003F5306CDCF81040E40CE404CCF81040FB
:10B1B000DCF8104024F0FF5424F4C014CCF8104004
:10B1C0008C69002C40F0C780DCF81040CD68C5F3D6
:10B1D00012052C43CCF81040DCF8104044F4002455
:10B1E000CCF81040012A00F0D0800A79012A00F042
:10B1F000D380D3F8002B42F00442C3F8002B002088
:10B2000003B0F0BD8C6984BB00EB4314D4F8105933
:10B2100025F0FF5525F4C015C4F81059D4F810597D
:10B2200045F40025C4F81059D4F81059ED0CED047C
:10B23000C4F81059012A4CD000EB4313D3F800494D
:10B2400044F00444C3F800490C79012C6AD08B699E
:10B25000002BD4D0D0F834380A7802F00F01012244
:10B260008A401343C0F83438C9E700EB4314D4F8DC
:10B270001059ED0CED04C4F81059D4F8105925F00C
:10B28000FF5525F4C015C4F81059D4F810698D691C
:10B29000CF683D44013DB5FBF7F5494F07EAC54589
:10B2A0003543C4F81059D4F810598E69C6F3120604
:10B2B0003543C4F8105904F510640D79012DB9D146
:10B2C000256925F0C0452561256945F000552561B2
:10B2D000B0E74A691AB100EB4314C4F814290A799B
:10B2E000012A08D000EB4313D3F8002942F00442AE
:10B2F000C3F8002983E7D0F8082812F4807F08D12A
:10B3000000EB4311D1F8002942F00052C1F80029A6
:10B31000E8E700EB4311D1F8002942F08052C1F870
:10B320000029DFE7D0F8084814F4807F0CD1D3F867
:10B33000004944F00054C3F8004900920B8B0A788E
:10B340000969FFF70DFF5AE7D3F8004944F080542C
:10B35000C3F80049F1E7CD682C44013CB4FBF5F497
:10B36000A4B204FB05F5CD61DCF81050144E06EADA
:10B37000C4442C43CCF81040DCF81040CD69C5F330
:10B3800012052C43CCF810402CE70A69002A3FF440
:10B390002CAFCCF8142028E7D0F8082812F4807FCE
:10B3A00006D1D3F8002B42F00052C3F8002B20E75F
:10B3B000D3F8002B42F08052C3F8002B19E700BFEE
:10B3C0000000F81F00B583B0844608464FEA920E8D
:10B3D00002F00302002305E00CF58051096840F8F3
:10B3E000041B01337345F7D39AB10CF5805CDCF88C
:10B3F000003001934FF0000C5FFA8CF3D900019BF1
:10B40000CB4000F8013B0CF1010C013A92B2002A4A
:10B41000F2D103B05DF804FB0B784A78012A14D00E
:10B4200000EB4310D0F8002B002A06DB2BB1D0F83C
:10B43000003B23F08043C0F8003BD0F8003B43F4CE
:10B440000013C0F8003B0020704700EB4310D0F819
:10B450000029002A06DB2BB1D0F8003923F0804305
:10B46000C0F80039D0F8003943F40013C0F80039AF
:10B47000E9E70B784A78012A0ED000EB4310D0F8A8
:10B48000003B23F40013C0F8003B0B79023BDBB216
:10B49000012B15D90020704700EB4310D0F800397C
:10B4A00023F40013C0F800390B79023BDBB2012B07
:10B4B000F0D8D0F8003943F08053C0F80039E9E7FC
:10B4C000D0F8003B43F08053C0F8003BE2E7D0F8EF
:10B4D000003823F4FE63C0F80038D0F800380901C2
:10B4E00001F4FE611943C0F8001800207047D0F83D
:10B4F000003E23F00303C0F8003ED0F8043823F0E8
:10B500000203C0F8043800207047D0F8003E23F052
:10B510000303C0F8003ED0F8043843F00203C0F83B
:10B520000438002070474269806910407047D0F8A5
:10B53000183800F50060C0691840000C7047D0F85A
:10B54000183800F50060C069184080B2704700EB01
:10B550004111D1F8082B00F5006040691040704798
:10B5600010B4D0F81048D0F8343801F00F02D340AE
:10B57000DB01DBB2234300EB411000F51060806873
:10B58000184010BC7047406900F00100704738B5A2
:10B590000546C36823F0C043C360012913D019BB1B
:10B5A000C36843F08043C36000240120FDF7EAF83C
:10B5B00001342846FFF7E7FF08B1312CF5D9322CCA
:10B5C00014D0002038BDC36843F00053C36000248A
:10B5D0000120FDF7D7F801342846FFF7D4FF0128F2
:10B5E000EDD0312CF4D9EAE70120EBE70120E9E7BF
:10B5F000D0F8003923F4FF6323F00703C0F80039C3
:10B60000D0F8043843F48073C0F804380020704741
:10B6100010B4046C144B9C4203D9D0F8003B002BAF
:10B6200016DB0024C0F8104BD0F8104B44F4002473
:10B63000C0F8104BD0F8104B44F01804C0F8104B71
:10B64000D0F8104B44F0C044C0F8104B012902D090
:10B65000002010BC7047C0F8142BD0F8003B43F01A
:10B660008023C0F8003BF3E70A30544F10B5D0F800
:10B67000D43203F1B00250F822408CB100EB8200CA
:10B6800043687BB194F80002FF280DD09B6894F8C2
:10B69000012221469847FF2384F80032002010BD84
:10B6A0000320FCE70020FAE70020F8E70A230380E4
:10B6B00000487047340A0020F8B506460F4F822133
:10B6C000384600F03CFC05460121384600F037FCC6
:10B6D00004468121384600F032FC0DB11022AA71D7
:10B6E0001CB1402222710022627118B14022027105
:10B6F00000224271432333800048F8BDF009002046
:10B70000F8B506460F4F8221384600F018FC054672
:10B710000121384600F013FC04468121384600F030
:10B720000EFC0DB11022AA711CB140222271002220
:10B73000627118B1402202710022427143233380AA
:10B740000048F8BDF0090020F8B506460F4F8221E9
:10B75000384600F0F4FB05460121384600F0EFFBC7
:10B7600004468121384600F0EAFB0DB11022AA718F
:10B770001CB1002222710222627118B100220271F2
:10B7800002224271432333800048F8BDF0090020B3
:10B7900038B5D0F8D432B03350F8235095B10446C0
:10B7A00001F0BDF9C5F80C02D4F8D432B03304EB83
:10B7B00083046368DB6805F50371D5F804029847D4
:10B7C000002038BD0320FCE738B5D0F8C852D0F8C7
:10B7D000D432B03350F8234084B301F00F0303EBAD
:10B7E000830200EB820292694AB103EBC30C05EBC2
:10B7F0008C05AD6CB2FBF5FC05FB1C2292B100235D
:10B80000C4F81432D0F8D432B03300EB830043686C
:10B810001B69ABB10A4604F50471D4F808029847D5
:10B82000002038BD03EB830300EB830300249C61FD
:10B830002346224601F0BCF92046F2E70320F0E758
:10B840000020EEE7F0B583B0D0F8D43203F1B002B7
:10B8500050F8227000228DF80720ADF80420002F48
:10B860007BD004460D46097811F0600634D0202EB6
:10B870006CD1EA882AB311F0800F07D16B7887F872
:10B880000032EA883F2A13D8D2B212E0B03300EB7C
:10B8900083035B689B68394668789847EA88072A7B
:10B8A00028BF07223946204600F0FAFE002651E064
:10B8B000402287F801223946204600F006FF002684
:10B8C00048E0B03300EB830463689B68002229469C
:10B8D0006878984700263DE06F780B2F31D8DFE875
:10B8E00007F006393030303030303030162690F8DE
:10B8F0009C32DBB2032B04D0294600F05DFB03260B
:10B9000028E0022201A900F0CBFE3E4622E090F89A
:10B910009C32DBB2032B04D0294600F04DFB0326FA
:10B9200018E001220DF1070100F0BAFE12E090F8D4
:10B930009C32DBB2032B0DD0294600F03DFB0326E1
:10B9400008E0294600F038FB032603E0294600F012
:10B9500033FB0326304603B0F0BD0326FAE738B5C3
:10B960000446812101F004F90025258701212046A4
:10B9700001F0FEF8A4F878518221204601F0F8F891
:10B98000A4F84C50A4F84E50D4F8D43203F1B002CD
:10B9900054F822209AB1B03304EB83035B685B68F0
:10B9A0009847D4F8D432B03354F8230001F0C2F8E9
:10B9B000D4F8D432B03344F82350C4F8BC52002039
:10B9C00038BD70B504464FF4077001F0AFF8002899
:10B9D00049D005464FF407720021F4F7FDFDD4F875
:10B9E000D432B03344F82350C4F8BC52237C002B2B
:10B9F00041D14FF4007302228121204601F0ADF8BD
:10BA0000012626874FF4007302223146204601F0BA
:10BA1000A4F8A4F878611023A4F84E300823032278
:10BA20008221204601F099F80123A4F84C30002629
:10BA3000C5F80462D4F8D432B03304EB83035B68F6
:10BA40001B689847C5F81462C5F81862D5F8042237
:10BA500062B3257C1DBB4FF400730121204601F029
:10BA6000AFF8284670BDD4F8D432B033002244F881
:10BA700023200225F5E7402302228121204601F000
:10BA80006CF801262687402302223146204601F029
:10BA900064F8A4F878611023A4F84E30BEE7402380
:10BAA0000121204601F08CF80025DAE70225D8E7CD
:10BAB00039B1D0F8D432B03300EB830041600020BC
:10BAC000704703207047D0F8D432B03350F8233099
:10BAD0002BB1C3F80812C3F81022002070470320CE
:10BAE0007047D0F8D432B03350F823301BB1C3F8CC
:10BAF0000412002070470320704708B5D0F8D432F4
:10BB0000B03350F823209AB1D2F814320BB101208F
:10BB100008BD0123C2F81432D2F81032C362D2F841
:10BB20001032D2F80822812101F042F80020EFE71C
:10BB30000320EDE710B5D0F8D432B03350F823200D
:10BB400092B1047C44B94FF40073D2F8042201216D
:10BB500001F036F8204610BD4023D2F8042201211E
:10BB600001F02EF80024F5E70324F3E798B108B5B7
:10BB700003460020C3F8B802C3F8C402C3F8D002D9
:10BB800009B1C3F8B412012183F89C121A70184647
:10BB900000F07AFF08BD0320704710B582B0002383
:10BBA000ADF8063089B10446C0F8B812CB6A23B1AB
:10BBB0000DF106009847C4F8D002D4F8D83201330A
:10BBC000C4F8D832002002B010BD0320FBE708B54E
:10BBD00000F0BBFF08BD08B5D0F8B83213B11B6840
:10BBE000984708BD0020FCE708B5D0F8B8325B687C
:10BBF000984700B908BD0320FCE738B5044600F2B9
:10BC0000AA25284600F0C4F90123C4F89432B4F8F8
:10BC1000B032C4F8983294F8AA1201F01F03012B35
:10BC20000DD0022B10D02BB101F08001204600F086
:10BC3000A7FF03E02946204600F080FB38BD2946D7
:10BC4000204600F0B6FBF9E72946204600F0F3FB5A
:10BC5000F4E7F8B50446012380F89C320023C0F8CD
:10BC600094324360C0F8A43280F8A032D0F8B832E1
:10BC7000DBB15B68DBB1002198470746C8B94023B8
:10BC800000221146204600F068FF0126A4F86461F6
:10BC90004025C4F860512B4600228021204600F048
:10BCA0005CFFA68425623846F8BD0027E7E7002739
:10BCB000E5E70327E3E701740020704790F89C3222
:10BCC000DBB280F89D32042380F89C32002070475C
:10BCD00090F89C32DBB2042B01D00020704790F822
:10BCE0009D32DBB280F89C32F7E708B590F89C32C1
:10BCF000DBB2032B01D0002008BDD0F8B832002BF6
:10BD0000F9D0DB69002BF6D09847F4E708B5D0F8F6
:10BD1000D432AE3350F823205AB190F89C32DBB2C3
:10BD2000032B01D0002008BD136A23B198470020DF
:10BD3000F9E70320F7E70020F5E708B5D0F8D4329B
:10BD4000AE3350F823205AB190F89C32DBB2032B6B
:10BD500001D0002008BD536A23B198470020F9E7BD
:10BD60000320F7E70020F5E70020704708B501231E
:10BD700080F89C32D0F8B83223B15B6801799847DB
:10BD800010B908BD0020FCE70320FAE70020704747
:10BD90000020704738B504460D46002943D11346AC
:10BDA000D0F89422032A01D0084638BDD0F85C119F
:10BDB000D0F86021914212D890F8AA3203F01F0304
:10BDC000012B17D0022B1CD0284694F89C32DBB2F2
:10BDD000032B1BD0204600F08FFC2846E5E7891A8C
:10BDE000C0F85C118A4228BF0A46194600F07CFC64
:10BDF0002846DAE790F8AE12FFF7C8FF0028E9D12D
:10BE0000E3E790F8AE12FFF7C3FFF7E700F1AE03E8
:10BE100054F823301A69002ADCD0C4F8D4021B6914
:10BE200020469847D6E701F07F01FFF7B1FF90B9B0
:10BE300094F89C32DBB2032BB7D100F1AE0354F877
:10BE400023309A69002AB0D0C4F8D4029B692946ED
:10BE500020469847A9E70020A7E738B504460D46D5
:10BE600000294BD11346D0F89422022A07D094F827
:10BE7000A00218B1002384F8A032284638BDC26958
:10BE8000016A8A420ED88A4218D094F89C32DBB2FA
:10BE9000032B27D08021204600F072FE204600F0C0
:10BEA00036FCE4E7521AC261194600F006FC002392
:10BEB0001A461946204600F083FED8E78369994266
:10BEC000E3D8D0F898229342DFD20022114600F046
:10BED000F4FB0021C4F898120B460A46204600F0F5
:10BEE0006FFEC4E7D4F8B832DA68002AD2D0002254
:10BEF000C4F8D422DB6820469847CBE741F08001A4
:10BF0000FFF746FF90B994F89C32DBB2032BB5D112
:10BF100000F1AE0354F823305A69002AAED0C4F8B9
:10BF2000D4025B69294620469847A7E70020A5E789
:10BF300003780A8813440B800378184470474288BA
:10BF400003789A4218D930B583B004460D46ADF84F
:10BF500006306288BDF806309A420AD90DF1060112
:10BF6000FFF7E6FF4378052BF3D18378AB42F0D19E
:10BF700000E0002003B030BD0020704703460020E1
:10BF800002E00130C0B201331A78002AF9D17047BB
:10BF90000B7803704B7843708B78CA7843EA02239E
:10BFA00043800B794A7943EA022383808B79CA79EB
:10BFB00043EA0223C380704710B50446802100F095
:10BFC000DFFD0021204600F0DBFD10BD30B583B061
:10BFD00004460D460023ADF806304A88130A013B9B
:10BFE000062B00F2AB80DFE803F0041F33A9A98D14
:10BFF0009A00D0F8B4321B680DF10601007C984716
:10C00000EA88002A00F0A380BDF80630002B00F07B
:10C0100099809A4228BF1A46ADF80620014620466C
:10C0200000F03EFB03B030BD037C43B9D0F8B8321A
:10C030009B6A0DF10600984702234370E0E7D0F8B1
:10C04000B832DB6A0DF10600984702234370D7E748
:10C05000D2B2052A52D8DFE802F003101D2A374475
:10C06000D0F8B4325B6823B10DF10601007C98472B
:10C07000C6E72946FFF7A0FFD4E7D0F8B4329B68A3
:10C0800023B10DF10601007C9847B9E72946FFF777
:10C0900093FFC7E7D0F8B432DB6823B10DF1060196
:10C0A000007C9847ACE72946FFF786FFBAE7D0F84F
:10C0B000B4321B6923B10DF10601007C98479FE75C
:10C0C0002946FFF779FFADE7D0F8B4325B6923B1B9
:10C0D0000DF10601007C984792E72946FFF76CFFB7
:10C0E000A0E7D0F8B4329B6923B10DF10601007CC2
:10C0F000984785E72946FFF75FFF93E72946FFF753
:10C100005BFF8FE7037C33B9D0F8B8325B6B0DF17E
:10C110000600984774E72946FFF74EFF82E7037C45
:10C1200043B9D0F8B8321B6B0DF1060098470723CE
:10C13000437065E72946FFF73FFF73E72946FFF79E
:10C140003BFF6FE729462046FFF736FF6AE72046A8
:10C1500000F0D2FA66E738B504468B88FBB9CB8885
:10C16000EBB94B887F2B1AD803F07F0590F89C32EF
:10C17000DBB2032B0CD080F89E52294600F010FD54
:10C18000204600F0B9FA35B1022384F89C3209E068
:10C19000FFF712FF06E0012384F89C3202E02046FC
:10C1A000FFF70AFF38BD000070B504460E468D78D3
:10C1B0002F4B1D70012D10D890F89C32DBB2022B52
:10C1C0000FD0032B26D0FFF7F7FE294B1978204616
:10C1D000FFF70AFD0325284670BDFFF7EDFE032596
:10C1E000F9E7A5B145602946FFF7F5FC054638B1EA
:10C1F00031462046FFF7E0FE022384F89C32EAE74E
:10C20000204600F079FA032384F89C32E3E700F03B
:10C2100073FAE0E7CDB141688D4225D0C9B2FFF78E
:10C22000E3FC134B197861602046FFF7D4FC054608
:10C23000B0B131462046FFF7BFFE21792046FFF717
:10C24000D3FC022384F89C32C5E7022380F89C3299
:10C2500045602946FFF7C8FC204600F04DFABAE7D2
:10C26000204600F049FAB6E700F046FA0025B2E7AA
:10C27000D00C012008B5CB88012B0BD190F89C3253
:10C28000DBB2022B09D9032B09D10122011D00F0D9
:10C2900007FA01E0FFF790FE08BD5BB213B9FFF7A4
:10C2A0008BFEF9E70146002341F8083F012200F028
:10C2B000F7F9F1E708B590F89C32013B022B12D850
:10C2C000CB88022B0CD10123C360D0F8A4320BB170
:10C2D0000323C360022200F10C0100F0E1F908BD64
:10C2E000FFF76AFEFBE7FFF767FEF8E708B54B8844
:10C2F000012B04D0022B07D0FFF75EFE08BDC0F86B
:10C30000A43200F0F9F9F9E78B881B0A80F8A03213
:10C3100000F0F2F9F2E708B590F89C32013B022BED
:10C3200009D84B88012B00D008BD0023C0F8A432E7
:10C3300000F0E2F9F8E7FFF73FFEF5E738B50C78D3
:10C3400004F06004202C06D0402C04D06CB1FFF720
:10C3500033FE002407E0D0F8D432AE3350F8233057
:10C360009B6898470446204638BD4D78092D1DD856
:10C37000DFE805F012191C161C08051C0F0BFFF74F
:10C3800025FEF0E7FFF7E7FEEDE7FFF70DFF0446B8
:10C39000E9E7FFF76FFFE6E7FFF78CFF2C46E2E7E0
:10C3A000FFF7A4FFDFE7FFF7B6FFDCE7FFF704FEC8
:10C3B000D9E770B505460C460B7803F06003202BD7
:10C3C00007D0402B05D023B1FFF7F6FD00263046FD
:10C3D00070BD95F89C32013B022B26D821790129AA
:10C3E00005D921462846FFF7E7FD0026EFE7284656
:10C3F000FFF7CCFC68B900F1AE0255F82220916835
:10C4000089B1C5F8D4029368214628469847064664
:10C4100000E00326E388002BD9D1002ED7D128468F
:10C4200000F06AF9D3E70326F4E721462846FFF730
:10C43000C3FD0026CBE72DE9F04106460D468B886B
:10C44000DFB20C7804F06004202C08D0402C06D019
:10C45000DCB1FFF7B1FD00242046BDE8F08139468C
:10C460003046FFF795FC0446002840F0F880C6F8F7
:10C47000D40200F1AE0356F823309B68002BEBD0BA
:10C480002946304698470446E6E791F80180B8F11E
:10C49000010F31D0B8F1030F05D0B8F1000F67D00C
:10C4A000FFF78AFDD8E790F89C32DBB2022B04D06C
:10C4B000032B12D0FFF780FDCEE70FB1802F04D100
:10C4C00029463046FFF778FDC6E7394600F058FBAD
:10C4D0008021304600F054FBBEE74B8823B91FB1E2
:10C4E000802F01D0CB881BB1304600F005F9B3E7AF
:10C4F000394600F045FBF7E790F89C32DBB2022B9F
:10C5000004D0032B12D0FFF757FDA5E70FB1802F02
:10C5100004D129463046FFF74FFD9DE7394600F02C
:10C520002FFB8021304600F02BFB95E74B88002B3A
:10C5300092D117F07F0F17D1304600F0DDF8394661
:10C540003046FFF725FC002886D1C6F8D40200F15A
:10C55000AE0256F822209268002A00F08280294616
:10C5600030469047044677E7394600F011FBE3E791
:10C5700090F89C22D2B2022A05D0032A27D0FFF7D6
:10C580001BFD444668E70FB1802F13D113F0800FD5
:10C5900014D107F07F0707EB8707B90001F5A871F1
:10C5A0003144043100230B600222304600F078F859
:10C5B000444651E7FFF700FD44464DE707F07F078B
:10C5C00007EB8707B900103131440431EAE75BB269
:10C5D000002B1FDB07F00F0202EB820200EB82024E
:10C5E000B2F864211AB3002B25DB07F07F0303EBBD
:10C5F00083039C0004F5A874344404340FB1802FE5
:10C6000022D10023236002222146304600F048F860
:10C61000444621E707F00F0202EB820200EB8202A0
:10C62000928C002ADFD1FFF7C7FC444614E7FFF7DE
:10C63000C3FC444610E707F07F0303EB83039C0031
:10C64000103434440434D9E73946304600F050FA07
:10C6500010B101232360D6E700232360D3E7002431
:10C66000FAE60446F8E6D0B170B50D461646044623
:10C67000FFF784FC431C5B009BB233802B700323C9
:10C680006B70022307E0EA5401345A1CD2B2002135
:10C69000A9540233DBB22278002AF4D170BD70476E
:10C6A00008B513460222C0F894228361C3610A468A
:10C6B000002100F07DFA002008BD08B513460A46A7
:10C6C000002100F075FA002008BD08B513460322CA
:10C6D000C0F89422C0F85831C0F85C310A460021F5
:10C6E00000F06EFA002008BD08B513460A46002186
:10C6F00000F066FA002008BD08B50422C0F89422B4
:10C7000000231A46194600F053FA002008BD08B568
:10C710000522C0F8942200231A46194600F050FA68
:10C72000002008BD08B500220F491048FFF71EFA87
:10C7300070B90F490D48FFF730FA60B90D490B4841
:10C74000FFF7B6F950B90948FFF741FA48B908BDF3
:10C75000FBF750FBEDE7FBF74DFBEFE7FBF74AFB81
:10C76000F1E7FBF747FBF2E7540A0020D40C012065
:10C77000B8090020400A00200020704700207047C0
:10C780000020704710B50146044C2046FFF7A9F978
:10C790002046FFF7CFF9002010BD00BFD40C0120C8
:10C7A00010B5064C002206492046FFF78CF90549D2
:10C7B0002046FFF796F9002010BD00BFD40C0120E1
:10C7C000B0170120B00F0120094BD3F8BC32D3F8C9
:10C7D00014320BB10120704710B5054C0A460146D2
:10C7E0002046FFF770F92046FFF787F910BD00BF1C
:10C7F000D40C012012230B8000487047700A0020DF
:10C8000004230B8000487047840A002000239342D1
:10C810001ED200B510E00CF1370C01F813C0000176
:10C820004FEA430C0CF1010C4FF0000E01F80CE044
:10C830000133DBB2934209D24FEA107CB0F1204FB2
:10C84000E9D20CF1300C01F813C0E8E75DF804FB05
:10C850007047000038B50B4BD3F8100AD3F8144AD0
:10C86000D3F8183AC01800D138BD074D0822A91CCA
:10C87000FFF7CCFF042205F112012046FFF7C6FFA7
:10C88000F2E700BF0070FF1F880A002008B51A23D6
:10C890000B80FFF7DFFF014808BD00BF880A0020BA
:10C8A00008B50A4628B905490548FFF7DCFE0348E4
:10C8B00008BD02490248FFF7D6FEF8E7B01F012085
:10C8C00010CF000810B50A46034C21460348FFF775
:10C8D000CAFE204610BD00BFB01F01201CCF0008BB
:10C8E00008B50A4628B905490548FFF7BCFE0348C4
:10C8F00008BD02490248FFF7B6FEF8E7B01F012065
:10C900002CCF000808B50A4628B905490548FFF7A5
:10C91000AAFE034808BD02490248FFF7A4FEF8E753
:10C92000B01F012038CF000870B588B000230393F2
:10C9300004930593069307930368B3F1A04F01D0C6
:10C9400008B070BD00250195164C236B43F0010320
:10C950002363236B03F001030193019B4FF4C05346
:10C96000039302230493032306930A26079603A93D
:10C970000D48FCF743F9636B43F080036363029552
:10C98000636C43F480436364636C03F480430293F9
:10C99000029B2A4631464320FBF71AFF4320FBF750
:10C9A0004FFFCDE7003802400000024008B500F21A
:10C9B000C441D0F80805FFF720F908BD08B501EB20
:10C9C000C10300EB8303D3F88C22D0F80805FFF7EE
:10C9D000E1F908BD08B501EBC10300EB8303DA6C94
:10C9E000D0F80805FFF739FA08BD08B5D0F80805F2
:10C9F000FFF77BF908BD10B50446C368022B09D1C7
:10CA00000121D4F80805FFF756F9D4F80805FFF717
:10CA100020F910BDFBF7EEF9F2E7000010B504466F
:10CA2000D0F80805FFF74AF92268D2F8003E43F033
:10CA30000103C2F8003E236A23B1034A136943F09D
:10CA40000603136110BD00BF00ED00E008B5D0F88B
:10CA50000805FFF73DF908BD08B5D0F80805FFF750
:10CA60006CF908BD08B5D0F80805FFF74FF908BD07
:10CA700008B5D0F80805FFF777F908BD08B5D0F874
:10CA80000805FFF773F908BD02780AB10020704766
:10CA900010B503461548C0F80835C3F8C8024FF072
:10CAA000A0430360042343600222C26000230361A9
:10CAB0008261C36103624362C3620363FCF71EFACF
:10CAC00080B90A4C80212046FDF713F8402200214E
:10CAD0002046FCF7E9FF802201212046FCF7E4FF15
:10CAE000002010BDFBF786F9EBE700BFB021012065
:10CAF000D0F8C83211F0800F08D101F07F0101EBAE
:10CB0000C10103EB810191F87E02704701F07F01C2
:10CB100001EBC10103EB810191F83E00704708B5BC
:10CB2000D0F8C802FCF70DFC08BD000000487047B3
:10CB3000BC2601207047032805D8DFE800F0050473
:10CB40000205012070470320704708B5D0F8C802DD
:10CB5000FCF76BFAFFF7EFFF08BD08B594461A46DD
:10CB60006346D0F8C802FCF73FFBFFF7E4FF08BDBF
:10CB700008B5D0F8C802FCF77CFBFFF7DCFF08BD66
:10CB800008B5D0F8C802FCF714FCFFF7D4FF08BDC5
:10CB900008B5D0F8C802FCF750FCFFF7CCFF08BD81
:10CBA00008B5D0F8C802FCF70BFBFFF7C4FF08BDBF
:10CBB00008B5D0F8C802FCF7CDFBFFF7BCFF08BDF5
:10CBC00008B5D0F8C802FCF78DFBFFF7B4FF08BD2D
:10CBD000024B13B10248F3F7B9BC704700000000E4
:10CBE00065050008F8B500BFF8BC08BC9E46704754
:0CCBF000F8B500BFF8BC08BC9E467047BA
:10CC0000080000202020202020202020202020207C
:10CC10002020202030303030303030303030303054
:10CC20003030303000000000050000001900000026
:10CC30007D00000000000000000000000000F03F48
:10CC400000000000000024400000000000005940E7
:10CC50000000000000408F40000000000088C3403A
:10CC600000000000006AF8400000000080842E41AF
:10CC700000000000D01263410000000084D79741FB
:10CC80000000000065CDCD41000000205FA0024201
:10CC9000000000E876483742000000A2941A6D4276
:10CCA000000040E59C30A2420000901EC4BCD64269
:10CCB00000003426F56B0C430080E03779C3414314
:10CCC00000A0D8855734764300C84E676DC1AB438A
:10CCD000003D9160E458E143408CB5781DAF1544A8
:10CCE00050EFE2D6E41A4B4492D54D06CFF0804483
:10CCF000F64AE1C7022DB544B49DD9794378EA4498
:10CD0000BC89D897B2D29C3C33A7A8D523F6493921
:10CD10003DA7F444FD0FA5329D978CCF08BA5B2543
:10CD2000436FAC642806C80A0080E03779C34143EA
:10CD3000176E05B5B5B89346F5F93FE9034F384D81
:10CD4000321D30F94877825A3CBF737FDD4F15752D
:10CD500020202020202020202020202020202020D3
:10CD600030303030303030303030303030303030C3
:10CD700020202020202020202020202020202020B3
:10CD800030303030303030303030303030303030A3
:10CD9000002020202020202020202828282828208B
:10CDA0002020202020202020202020202020202083
:10CDB00020881010101010101010101010101010EB
:10CDC00010040404040404040404041010101010DB
:10CDD00010104141414141410101010101010101A5
:10CDE00001010101010101010101010110101010F7
:10CDF0001010424242424242020202020202020277
:10CE000002020202020202020202020210101010CA
:10CE100020000000000000000000000000000000F2
:10CE20000000000000000000000000000000000002
:10CE300000000000000000000000000000000000F2
:10CE400000000000000000000000000000000000E2
:10CE500000000000000000000000000000000000D2
:10CE600000000000000000000000000000000000C2
:10CE700000000000000000000000000000000000B2
:10CE800000000000000000000000000000000000A2
:10CE90000000000044313B3078256C6C582C307811
:10CEA000256C580D0A00000044314F56523B307833
:10CEB000256C580D0A00000044323B3078256C6C1C
:10CEC000582C3078256C580D0A00000044324F561B
:10CED000523B3078256C580D0A00000052455345EE
:10CEE000545F495744470D0A494E49545F434F4DDB
:10CEF000504C4554450D0A000000000000000000A1
:10CF000001020304060708090006101600061016A1
:10CF100050756C73655375636B6572004863635439
:10CF20006563682E20496E6300000000434443207F
:10CF3000436F6E666967000043444320496E746521
:10CF40007266616365000000494E4600696E6600C6
:10CF50004E414E006E616E0030313233343536371B
:10CF60003839616263646566000000003031323335
:10CF700034353637383941424344454600000000D5
:10CF8000286E756C6C290000300000004E614E0068
:10CF9000496E66696E6974790000000042616C6CCC
:10CFA0006F632073756363656564656400000000EA
:10CFB0002E2E2F2E2E2F2E2E2F2E2E2F2E2E2F2E8C
:10CFC0002E2F2E2E2F2E2E2F6E65776C69622F6CD2
:10CFD0006962632F7374646C69622F64746F612E6D
:10CFE000630000002E2E2F2E2E2F2E2E2F2E2E2FB2
:10CFF0002E2E2F2E2E2F2E2E2F2E2E2F6E65776C4F
:10D0000069622F6C6962632F7374646C69622F6D3F
:10D01000707265632E6300002C2066756E63746900
:10D020006F6E3A2000000000617373657274696F5F
:10D030006E2022257322206661696C65643A206641
:10D04000696C6520222573222C206C696E65202571
:10D0500064257325730A000043000000504F5349B4
:08D06000580000002E00000042
:08D068001032FF7F01000000FF
:08D07000D1CB000829020008E1
:04D0780001020008A9
:10D07C00080000200000000000000000F402002066
:10D08C005C030020C403002000000000000000002E
:10D09C000000000000000000000000000000000084
:10D0AC000000000000000000000000000000000074
:10D0BC000000000000000000000000000000000064
:10D0CC000000000000000000000000000000000054
:10D0DC000000000000000000000000000000000044
:10D0EC000000000000000000000000000000000034
:10D0FC000000000000000000000000000000000024
:10D10C000000000000000000000000000000000013
:10D11C000000000000000000000000000000000003
:10D12C0001000000000000000E33CDAB34126DE6A0
:10D13C00ECDE05000B000000000000000000000009
:10D14C0000000000000000000000000000000000D3
:10D15C0000000000000000000000000000000000C3
:10D16C0000000000000000000000000000000000B3
:10D17C0000000000000000000000000000000000A3
:10D4AC0000000000000000003004002030040020C8
:10D4BC0038040020380400204004002040040020E0
:10D4CC004804002048040020500400205004002090
:10D4DC005804002058040020600400206004002040
:10D4EC0068040020680400207004002070040020F0
:10D4FC0078040020780400208004002080040020A0
:10D50C00880400208804002090040020900400204F
:10D51C009804002098040020A0040020A0040020FF
:10D52C00A8040020A8040020B0040020B0040020AF
:10D53C00B8040020B8040020C0040020C00400205F
:10D54C00C8040020C8040020D0040020D00400200F
:10D55C00D8040020D8040020E0040020E0040020BF
:10D56C00E8040020E8040020F0040020F00400206F
:10D57C00F8040020F804002000050020000500201D
:10D58C0008050020080500201005002010050020CB
:10D59C00180500201805002020050020200500207B
:10D5AC00280500202805002030050020300500202B
:10D5BC0038050020380500204005002040050020DB
:10D5CC00480500204805002050050020500500208B
:10D5DC00580500205805002060050020600500203B
:10D5EC0068050020680500207005002070050020EB
:10D5FC00780500207805002080050020800500209B
:10D60C00880500208805002090050020900500204A
:10D61C009805002098050020A0050020A0050020FA
:10D62C00A8050020A8050020B0050020B0050020AA
:10D63C00B8050020B8050020C0050020C00500205A
:10D64C00C8050020C8050020D0050020D00500200A
:10D65C00D8050020D8050020E0050020E0050020BA
:10D66C00E8050020E8050020F0050020F00500206A
:10D67C00F8050020F8050020000600200006002018
:10D68C0008060020080600201006002010060020C6
:10D69C001806002018060020200600202006002076
:10D6AC002806002028060020300600203006002026
:10D6BC0038060020380600204006002040060020D6
:10D6CC004806002048060020500600205006002086
:10D6DC005806002058060020600600206006002036
:10D6EC0068060020680600207006002070060020E6
:10D6FC007806002078060020800600208006002096
:10D70C008806002088060020900600209006002045
:10D71C009806002098060020A0060020A0060020F5
:10D72C00A8060020A8060020B0060020B0060020A5
:10D73C00B8060020B8060020C0060020C006002055
:10D74C00C8060020C8060020D0060020D006002005
:10D75C00D8060020D8060020E0060020E0060020B5
:10D76C00E8060020E8060020F0060020F006002065
:10D77C00F8060020F8060020000700200007002013
:10D78C0008070020080700201007002010070020C1
:10D79C001807002018070020200700202007002071
:10D7AC002807002028070020300700203007002021
:10D7BC0038070020380700204007002040070020D1
:10D7CC004807002048070020500700205007002081
:10D7DC005807002058070020600700206007002031
:10D7EC0068070020680700207007002070070020E1
:10D7FC007807002078070020800700208007002091
:10D80C008807002088070020900700209007002040
:10D81C009807002098070020A0070020A0070020F0
:10D82C00A8070020A8070020B0070020B0070020A0
:10D83C00B8070020B8070020C0070020C007002050
:10D84C00C8070020C8070020D0070020D007002000
:10D85C00D8070020D8070020E0070020E0070020B0
:10D86C00E8070020E8070020F0070020F007002060
:10D87C00F8070020F807002000080020000800200E
:10D88C0008080020080800201008002010080020BC
:10D89C00180800201808002020080020200800206C
:10D8AC002808002028080020FFFFFFFF00000200CE
:10D8BC004300000000000000000000000000000019
:10D8CC00000000000000000000000000000000004C
:10D8DC0043000000000000000000000000000000F9
:10D8EC00000000000000000000000000000000002C
:10D8FC0043000000000000000000000000000000D9
:10D90C00000000000000000000000000000000000B
:10D91C0043000000000000000000000000000000B8
:10D92C0000000000000000000000000000000000EB
:10D93C004300000000000000000000000000000098
:10D94C0000000000000000000000000000000000CB
:10D95C004300000000000000000000000000000078
:10D96C0000000000000000000000000000000000AB
:10D97C004300000000000000000000000000000058
:10D98C00000000000000000000000000000000008B
:10D99C0031630008ED4D00080000000090CD000838
:10D9AC0064D0000824D0000824D0000824D000083B
:10D9BC0024D0000824D0000824D0000824D000086B
:10D9CC0024D0000824D00008FFFFFFFFFFFFFFFF5B
:10D9DC00FFFFFFFFFFFF00000100415343494900D7
:10D9EC00000000000000000000000000000000002B
:10D9FC0000000000000000000000415343494900B2
:10DA0C00000000000000000000000000000000000A
:10DA1C000000000000000000000000000024F400E2
:10DA2C000100000010000000C3B900085FB9000835
:10DA3C0045B80008000000006DB60008C9B7000822
:10DA4C0091B700080000000000000000000000007A
:10DA5C0049B7000801B70008B9B60008ADB6000810
:10DA6C0009024300020100C0320904000001020255
:10DA7C000100052400100105240100010424020208
:10DA8C0005240600010705820308001009040100A3
:10DA9C00020A000000070501024000000705810290
:10DAAC00400000000A0600020000004001000000D7
:10DABC00A1C7000879C700087DC7000885C7000802
:10DACC0081C70008F5C7000801C80008C5C80008D0
:10DADC00A1C800088DC80008E1C8000805C90008E5
:10DAEC0012010002020200408304405700020102AE
:10DAFC0003010000040309041A03000000000000E5
:10DB0C000000000000000000000000000000000009
:04DB1C000000000005
:040000050800868DDC
:00000001FF
